:020000040000FA
:040000006FD00400B9
:101000006F00107E00000000000000009020002013
:10101000AA220020A9BDF9F56C23002000000000E1
:10102000000000006C230020902000200000000041
:101030000000000090200020000000009020002010
:101040000000000090200020902000209020002030
:101050009020002090200020502F00208A24002083
:101060000000000090200020902000201424002088
:1010700090200020D22300209020002090200020EB
:101080009020002090200020902000209020002020
:101090009020002001A04111B7170040985F3AC688
:1010A000945F3247E39CE6FE3245410182800111A4
:1010B00013078008F337078093F787083EC20100C3
:1010C0000100B7170040930570052380B70413068D
:1010D00080FA2380C7040100010083C6B70493F699
:1010E000F60DA385D704238007049246F3A6068055
:1010F0000100010093760502D5CEF336078093F602
:10110000860836C4010001002380B7042380C70489
:1011100001000100B70614007D89558D88C70100C4
:1011200001000100010023800704A246F3A6068007
:101130000100010073370780137787083AC6010062
:1011400001002380B7042380C704010001000100CF
:1011500001003727004093061005A303D7802380A2
:101160000704B247F3A70780010001009307800836
:10117000F3B7078093F787083ECE01000100B71749
:101180000040130770052380E704130780FA2380CB
:10119000E7040100010003C7B70413670708A3852C
:1011A000E70423800704F247F3A70780010001004A
:1011B0000561828093760504BDC6F336078093F6F9
:1011C000860836C8010001002380B7042380C704C5
:1011D00001000100B7061400938606047D89558D31
:1011E00088C7010001000100010023800704C246F6
:1011F000F3A6068001000100733707801377870884
:101200003ACA010001002380B7042380C70401000B
:1012100001003727004093062005A303D7802380D1
:101220000704D24781B773370780137787083ACC12
:10123000010001002380B7042380C70401000100DE
:1012400098471367070C98C723800704E24719BF24
:101250000111814601468145114506CE97000000E7
:10126000E780C05793078008F3B7078093F7870894
:101270003EC601000100B717004013077005238028
:10128000E704130780FA2380E7040100010003C785
:101290006704136717002383E70423800704B2471A
:1012A000F3A7078001000100F2400561828041112F
:1012B000814601468145114597000000E7800052B4
:1012C00013078008F337078093F787083EC40100AF
:1012D0000100B7170040130670052380C70493066A
:1012E00080FA2380D70401000100FD552396B70240
:1012F00023800704A245F3A5058001000100733790
:101300000780137787083AC6010001002380C704CD
:101310002380D7040100010003C767041367170087
:101320002383E70423800704B247F3A70780010063
:10133000010001A0B1473305F50201007D1575FDDF
:101340008280411122C426C206C6AA8401446317C2
:101350009400B24022449244410182800504130566
:10136000803E420497000000E78000FD4180C5B741
:101370009305000273A04580824573901534924016
:101380002242B2424243D2436244F2440255925551
:101390002256B2564257D2576258F25806499649D9
:1013A000264AB64A464BD64B664CF64C065D965DD1
:1013B000265EB65E465FD65F09617300203041113C
:1013C000B7170040985F3AC6945F3247E39CE6FE49
:1013D000324541018280B71700401307000323887C
:1013E000E702854717170000232EF75C73002030B3
:1013F000411122C406C637040020976000E0E78050
:101400000077975000E0E780009F1C40829797602C
:1014100000E0E780C075D5B7373700408347470005
:101420009146BD8B639ED702B73600401306F00F7E
:1014300097350000938505369737000083D7874599
:1014400003C7A6001377F70F1DE3B7E70400BC4FEF
:101450000946894517150000034585F7829731A095
:1014600099466394D700834757007300203003C721
:1014700086001377F70FE365F6FC13851700AE9728
:10148000173800002318A8402380E70075B7B787F6
:10149000004003C76700098B6309071003C7770083
:1014A0009306000313770703630DD708174800005E
:1014B0000348D8A1174600001306469E0547B30609
:1014C00006012380E60083C5770017470000130755
:1014D000E79E429793F5F50F2300B70003C58700F9
:1014E000974500009385859CC2951375F50F238061
:1014F000A5000347070089451377F703630CB70C72
:1015000063E7E50A6306071A8545630CB712974738
:10151000000083C7B79B3307F60003470700137724
:10152000F70F19CB850793F7F70F3D476363F71A5A
:1015300017470000A30CF798B7870040094723839B
:10154000E700B787004083C77700E207E18763DEE3
:1015500007049747000083C77797174700001307D2
:10156000E7933E9785462300D700174700001307EF
:10157000E7943E97930600032300D7001747000027
:101580001307C7923E97A14685072300D70093F71C
:10159000F70F3D476364F71417470000A308F7925D
:1015A000B787004009472383E70073002030930684
:1015B00010026300D70E930620026305D706930638
:1015C0000002E316D7F403C727021377C70F136788
:1015D0002700D5A803C767001377070465CB03C7A7
:1015E000A702173800001308E86C17350000130530
:1015F0002564134707082385E70203C7A70213776B
:10160000370F136787002385E7028147130700041C
:10161000B305F5008C41B306F80091078CC2E3993D
:10162000E7FEF5B503C7A702134707042385E702C2
:1016300003C7A7021377C70F136727002385E702A5
:10164000F9B503C767001377070449C303C76702E7
:10165000173800001308C859173500001305055145
:10166000134707082383E70203C767021377370F7F
:10167000136787002383E702814713070004B3053C
:10168000F5008C41B306F80091078CC2E399E7FEA0
:10169000BDBD03C76702134707042383E70203C7DF
:1016A00067021377C70F136727002383E70285B507
:1016B00003C767001377070411CB03C7270213770B
:1016C000370F136787002381E70291B52380060057
:1016D0003DBD97370000A38B077EB9BD973700004B
:1016E000A386077E75BD2303048015472303E4808A
:1016F00001002302A480828083076480E3CE07FE7A
:1017000023030480828083076480E3CE07FE0345C1
:101710004480828083076480E3CE07FE2302A48096
:101720008280411126C44AC24EC006C61377F50B0B
:10173000AD47AA892E899544630CF7001945970097
:101740000000E78080FA97000000E78020FB8D44CE
:101750004E8597000000E78040F9FD59FD1463981D
:101760003401B240A244124982494101828013559A
:1017700009011375F50F97000000E780E0F92209D1
:10178000F1BF011126CC06CEB70408009700000077
:10179000E780C0F6154597000000E78000F5970048
:1017A0000000E78080F697000000E78000F62AC678
:1017B00097000000E78080F432459377150089EBAD
:1017C000136515001375F50FF240E2440561828040
:1017D000FD14E9F00145CDBF397126DC4ADA4ED857
:1017E00052D656D45AD25ED006DE62CE66CCB7E769
:1017F00000E07D5783AA070022C603AA470023A062
:10180000E71823A2E718B7170040130770052380D5
:10181000E704130780FA2380E70483C74704930B88
:1018200075FFB684E20793FBFB0F8546AA892E8BD2
:10183000328937240040E187015763FA7601630853
:10184000D5008946130700026313D5000157D98FCD
:1018500093F7F70FB71C00402382FC0411472303C2
:10186000E4801305F00F97000000E78000E8094CC2
:1018700097000000E78080E863657C15B7050700E6
:10188000DA9537870700795563FEE504B38795003D
:10189000636AF704370B0800A94733EB65016395CA
:1018A000F90881E8814497000000E78020E526855B
:1018B00015A8DA85094597000000E780C0E605090C
:1018C0000345F9FFFD14050B97000000E780C0E415
:1018D00081C49377FB0FE5F797000000E780A0EA4B
:1018E00069F17D55B7170040130770052380E704A1
:1018F000130780FA2380E70403C74704418B238240
:10190000E704F250B7E700E023A0571123A24711E4
:10191000E25432445259C259325AA25A125B825B83
:10192000724CE24C21618280A547639BF906856970
:101930001309F00FB3069900B3742B01B694134941
:10194000F9FFB3749900856B33796901416B938713
:10195000F9FFB3F7270199E363FC340193D94900F8
:10196000C147E3E637FF3DBF0569C1697D19D9B7B6
:101970001305800D638869011305000263847901F2
:1019800013051008CA8597000000E780C0D99700AA
:101990000000E78040DF31D54E99B38434416DBFFC
:1019A000DA852D4597000000E780E0D7CA94E30B65
:1019B00099EE050997000000E78020D5A30FA9FE46
:1019C000FDB79387F9FF93F7F70F636DFC0C83C79F
:1019D0001C04130730086315F70637070800636116
:1019E000EB06B3079B00B706100063FBD704334B2D
:1019F000EB0089476399F9068980D549E38404EAB5
:101A0000DA85094597000000E780E0D11109032736
:101A1000C9FF91472320E48003076480E34E07FE5B
:101A200023033481FD17EDFBFD14110B81C4937763
:101A3000FB0FE9FF97000000E780E0D461F155B5A6
:101A4000B717004003C75704B7070800137707020A
:101A500019E3B78707007955E376FBE833079B0066
:101A6000E3F9E7F841B58547E380F9F0DA852D45DC
:101A700097000000E78020CB9389F4FFE38404E221
:101A800097000000E78060C893F7390091EB832648
:101A900004800327090093074900E396E6E03E89A6
:101AA000CE84D9BFB5476399F9001305900B970011
:101AB0000000E78080C3FDB3B1471305B00AE38897
:101AC000F9FE99476397F904B7050800B365BB00B1
:101AD0002D4597000000E78000C581448D4BA1494A
:101AE00097000000E78060C263967401832704803A
:101AF0002320F9008504E39534FF8327048013171E
:101B00002B01635507002312F90069BB2322F9005A
:101B100051BB9D47639FF90281451305B0049700AF
:101B20000000E78040C0BD442320090023220900B3
:101B3000FD5997000000E78040BD93F77400CA97F5
:101B400003C70700FD14398D2380A700E39334FFFA
:101B500091BBA1476397F90697000000E780A0C2F8
:101B60008144630D0B008D479304C0036308FB00A1
:101B70009304000563048B01930440041375C507A7
:101B8000E30295D2194597000000E78000B6970060
:101B90000000E780A0B6054597000000E780E0B4AC
:101BA000268597000000E78020B7094597000000D0
:101BB000E78080B697000000E780E0BCE31405CE24
:101BC0000DB39147639FF90013056006970000006D
:101BD000E780A0B197000000E78040B213059009AC
:101BE000F9B5E38109CCF1547DB9BD6601471736DB
:101BF00000001306264B938606A6854583470600FC
:101C000093F7F70F91C382800507E3F9E6FE973754
:101C100000002389B748DDB77D16620661869317F9
:101C20008601E18763D4070001458280931726006F
:101C30003307F500AE9718439C4363E7E7007D1632
:101C4000E37FF7FC7D55828005458280FD15E20526
:101C5000E18513978501618793F7F50F63480700C6
:101C6000FD15139725002A97584365D7138517004C
:101C70006205618582803308B5021C4283A8060094
:101C8000B335B502C29733B50701AE98469585487E
:101C90006367B5006394A50063E3070181480C43C3
:101CA000C6950CC388C21CC28280814713978701E6
:101CB00061876343B7008280139727002A97232008
:101CC00007008507E5B78147014793968701E186BD
:101CD00063C5B60013351700828093962700AA9635
:101CE00094428507558FD5B793D755408A07AA9751
:101CF0009C4305453315B5007D8D828017F3FFDFCA
:101D0000E702A33D2A8497000000E78060F405C540
:101D1000931725003E940327C4FF814711EB7D15DF
:101D200016053E954205418517F3FFDF6700233D09
:101D300005838507E5B70145C5BF8147139787012F
:101D400061876343C700828013972700B386E5004D
:101D500094422A97850714C3D5B77D16620661861B
:101D6000014793178601E18763D5070013351700F4
:101D7000828093172600B306F500AE9794429C43E9
:101D80007D16B58F5D8FF1BF8A05AA950147636304
:101D9000B500828083A6C5FFF11593D71600D98FB1
:101DA0009CC11397F601E5B72A8301480147014515
:101DB0006343D7008280B387050183A80700B30778
:101DC00006019C43C697AA976384F80033B51701B0
:101DD0000507B3080301620723A0F8006187110813
:101DE000C1BF2A8301478147014563C3D700828071
:101DF0003388E50083280800330EE600032E0E002A
:101E00003388A8403308C8416384080133B508010A
:101E10008507B308E300E20723A00801E187110763
:101E2000E9B717F3FFDFE702432B0111B286B28453
:101E30002E86AA850A8597000000E780C0FA2A84CA
:101E4000A6850A8597000000E78020E833348000EB
:101E5000060413351500018D056117F3FFDF6700D8
:101E6000032A17F3FFDFE702C3244111AA89AE8AD0
:101E7000328BB68402C202C402C60144131C840120
:101E8000135C8C4163499C02939B1400FD1B054924
:101E9000138CF4FFF15C33048901620461846340B4
:101EA000740792478E04CE9423AEF4FE410117F3DB
:101EB000FFDF6700832313192400B30B2B01014AB2
:101EC00093172A00D69783A50B0088437800340027
:101ED000500097000000E78040DA050A93178A0156
:101EE000E187F11BE35EFCFC92474E990504232039
:101EF000F900A2473EC2B24702C63EC441B7131A18
:101F00008901135A8A41131D240093178A01E1871E
:101F100063CF970092470A044E941CC0A24705095C
:101F20001379F90F3EC2B24702C63EC4ADB7B3073C
:101F30009A0313152A005695084178003400500082
:101F4000050AEA97DA978C4397000000E780E0D211
:101F50006DBF0000197106C212C416C61AC81ECA87
:101F600022CC26CE2AD02ED232D436D63AD83EDA59
:101F700042DC46DECAC0CEC2D2C4D6C6DAC8DECA89
:101F8000E2CCE6CEEAD0EED2F2D4F6D6FAD8FEDA39
:101F900097150000938585A28841E70005009240CF
:101FA0002242B2424243D2436244F2440255925525
:101FB0002256B2564257D2576258F25806499649AD
:101FC000264AB64A464BD64B664CF64C065D965DA5
:101FD000265EB65E465FD65F096173002030000062
:101FE0009721002093810102175100201301818164
:101FF00017F5FFFF13054501970500209385850020
:10200000171600201306C6FD63FAC50083220500DB
:1020100023A0550011059105E3EAC5FE171502003E
:10202000130505D0971500209385C5FB17160020D2
:102030001306467C63FAC5008322050023A05500E1
:1020400011059105E3EAC5FE171500201305857AF1
:1020500097450020938505516377B500232005003F
:102060001105E36DB5FEFD42739002BC8D42739085
:102070004280B722000093828288739002309702D8
:102080000020938222F893E23200739052309752EC
:1020900000009382428C739012346FB07476730098
:1020A0002030397101436EC619A0397141536AC895
:1020B00066CA62CC5ECE19A0397101535AD056D28D
:1020C00052D44ED64AD826DA22DC06DE33016140ED
:1020D000828241114AC026C222C406C68282B24D03
:1020E0004101024D924C224CB24B4101024B924AAB
:1020F000224AB2494101024992442244B24041017C
:1021000082803D432A876373C3029377F700BDEF54
:10211000ADE5937606FF3D8ABA960CC34CC30CC757
:102120004CC74107E36BD7FE11E28280B306C34080
:102130008A069702000096966780A6002307B700DC
:10214000A306B7002306B700A305B7002305B70011
:10215000A304B7002304B700A303B7002303B70009
:10216000A302B7002302B700A301B7002301B70001
:10217000A300B7002300B700828093F5F50F939674
:102180008500D58D93960501D58D61B7939627006F
:102190009702000096968682E78086FA9680C1179D
:1021A0001D8F3E96E374C3F8A5B73367B500FD53A2
:1021B0000D8B79E7B7877F7F9387F7F710419441BD
:1021C000B372F6003363F600BE92B3E26200639727
:1021D000720C6318D6065041D441B372F6003363D3
:1021E000F600BE92B3E262006398720A631BD604E3
:1021F00010459445B372F6003363F600BE92B3E225
:1022000062006391720A631ED6025045D445B372D0
:10221000F6003363F600BE92B3E26200639A72087E
:102220006311D60210499449B372F6003363F60085
:10223000BE92B3E26200639372085105D105E30FC9
:10224000D6F61317060193970601631CF700135780
:10225000060193D706013305F7409375F50F91E911
:1022600082804183C1833305F7409375F50F91E177
:1022700082801377F70F93F7F70F3305F7408280CB
:102280000346050083C60500050585056313D600D2
:1022900065FA3305D640828011059105E312D6FE1A
:1022A000014582802105A105E31CD6FC0145828001
:1022B0003105B105E316D6FC014582804105C10513
:1022C000E310D6FC01458280B717004003C77705AD
:1022D0001377E70FA38BE704130700F8A38DE70438
:1022E0003D47238CE70413075003A38CE70403C77F
:1022F000A7051377D70F238DE7048280B717004017
:1023000003C7E7020D8941111377C70F498F930661
:102310008008F3B6068093F6860836C601000100F1
:10232000930670052380D704930680FA2380D70490
:10233000010001002387E70223800704B247F3A7C7
:102340000780010001004101828041112A83014E72
:10235000930E407E130F0019930F400663E56E1233
:102360009308001913034006B3781503854E0D4FEB
:10237000A14F337365020D891335150063EFBE124B
:102380001308F6FF7946729842081358080133077C
:10239000C70213D61700BE0732976146B3F6C602CE
:1023A00013068070B386C6023697A166F58F420782
:1023B0005D8FB716004083C7F60293F70708A303A3
:1023C000F1000346710083C7F60293F70708E39410
:1023D000C7FE83477100B716004093F7F70F638875
:1023E000071293078008F3B7078093F787083EC466
:1023F00001000100B7170040930670052380D70441
:10240000930680FA2380D7040100010023AA070362
:1024100083C6170393E60608A388D7022380070420
:10242000A247F3A70780010001001166B71700401B
:102430007D16D45BC85F93854703A98EF18EF5FAAC
:1024400093068008F3B6068093F6860836C6010028
:102450000100930670052380D704930680FA238039
:10246000D7040100010098C103C7170313670704CD
:10247000A388E70223800704B247F3A7078001007F
:102480000100410182807D133368E3039308E01665
:10249000630E08003368F3039308D016630808003E
:1024A0009378330093B818009388D81633081E0128
:1024B000131E0801135E0E0155B56393E50305482D
:1024C000638608000148630303002A887108729834
:1024D000FD15131E0801C205135E0E01C18179BDF1
:1024E00013F8150063F4BF007908D5B71338180046
:1024F000E5BF83C7F60293F70708A303F10003467D
:10250000710083C7F60293F70708E394C7FE834779
:10251000710093F7F70FF1DFE9B531714AD966CB56
:1025200006DF22DD26DB4ED752D556D35AD15ECFF9
:1025300062CD6AC96EC7AA8C02D897100000E780E6
:1025400020B12A8993078008F3B7078093F787089B
:102550003EDA01000100B717004013077005238021
:10256000E704130780FA2380E7040100010003C792
:10257000F7021377770FA387E70203C7F702136702
:102580008700A387E70223800704D257F3A70780B9
:1025900001000100054597000000E78060D61307A1
:1025A00080C13347E902116A93070AE89306500293
:1025B000BD69930BA004814A014B13048008930466
:1025C00070057D1AB347F9023307D7023EC0FD8775
:1025D0003ECC938709A69309803E3347F7023AC25F
:1025E0007D873AC4334739038549B399990193D913
:1025F0003940B306D702B30B7703B3C6F602B3CBA9
:10260000FB0236C6FD8636C893D6FB4136CEB746AA
:102610000F00938606243349D9028566938606FA0D
:10262000B3969601B389E902130760553309D902BD
:1026300093060010B389E9023349D902B3C9F902FC
:102640009316390036CA37190040FD8636D0930DEF
:10265000090493D7F9413ED2F336048093F68608F5
:1026600036DC01000100930770052380FD0093060E
:1026700080FA2380DD00010001008346390593F6CE
:10268000860FA309D9048346390593E61600A309EA
:10269000D90423800D00E256F3A606800100010054
:1026A000130C80FA116DF336048093F6860836DE3B
:1026B00001000100930770052380FD0023808D0138
:1026C0000100010083463905216693E60602A3094D
:1026D000D90483560905B3E6A6012318D904835605
:1026E0000905D18E2318D90423800D00F256F3A6D4
:1026F0000680010001008346390593F606026381D6
:10270000061A03463905218A6DDE08189710000065
:10271000E78000987336048013768608B2C2010001
:10272000010023809D0023808D0101000100B71767
:10273000004003C637051376F60DA389C70403C608
:10274000370513660602A389C70483560905216667
:10275000B3E6A6012318D90483560905D18E2318A0
:10276000D90423800D009646F3A6068001000100DF
:102770008346390593F60602638B061483463905B2
:10278000A18AEDFE97000020E780E090AA8636D46B
:1027900097000020E7802090A256E30AD5FE8356DA
:1027A00009054255B3E6A6012318D9049710000085
:1027B000E780C08F83463905A18AEDDE03560905FF
:1027C0008346290582473376CA00B306DA0293D5D9
:1027D000F641B296B388F640E24733B8C6002E9869
:1027E0003308F840A247B3B616013308D84063C790
:1027F0000701631DF800924763FA1701C247634F50
:10280000F80E63950701B24763EAF80E894663E95B
:10281000660FF2469315180013D3F8015E861395E0
:102820001800B365B30042D646D497C00100E780D4
:10283000A0123258050B137BFB0F63470001631A8C
:102840000838A2586387083813081500B336A80063
:10285000B69513D6F5013298B336C800AE96135824
:102860001800FE06B3E60601733604801376860868
:10287000B2C60100010023809D0023808D0101006C
:1028800001000356C902B296C206C1822316D902BC
:1028900023800D00B646F3A606800100010021B595
:1028A000F336048093F68608B6C001000100238049
:1028B0009D0023808D01010001008346390593E6C8
:1028C0000602A309D90423800D0086460DB5F33610
:1028D000048093F68608B6C40100010023809D00A1
:1028E00023808D01010001008346390593E606022D
:1028F000A309D90423800D00A646BDB5E30B0BF058
:10290000F336048093F68608B6C8010001009306EA
:1029100080FA23809D002380DD00010001008346B2
:10292000390593F5FC0F93F6860FA309D904834666
:102930003905CD8EA309D90423800D00C646F3A620
:10294000068001000100130580FA0346390593064D
:1029500039051D8A631C9629733604801376860810
:10296000B2CC01000100130680FA23809D00238071
:10297000CD000100010003C606001376F60D23808A
:10298000C60003C60600136606022380C6008356EF
:1029900009051166D18E2318D904835609052166CD
:1029A000D18E2318D90423800D00E646F3A60680B5
:1029B00001000100130680FA8346390593F60602EA
:1029C0006380062683463905130C3905A18AFDDA92
:1029D000081897000000E780A06BF336048093F698
:1029E0008608B6D001000100930680FA23809D007E
:1029F0002380DD000100010083460C00116693F680
:102A0000F60D2300DC0083460C0093E6060223004B
:102A1000DC0083560905D18E2318D9048356090595
:102A20002166D18E2318D90423800D008656F3A683
:102A3000068001000100130680FA8346390593F6EB
:102A40000602638A062083463905A18AEDFE97F0C7
:102A5000FF1FE78040642A8C97F0FF1FE780A06388
:102A6000E30C85FF8356090511664255D18E231864
:102A7000D90497000000E780606383463905130698
:102A80003905A18AFDDAF336048093F68608B6D4B8
:102A900001000100930680FA23809D002380DD0061
:102AA000010001008346060093F6F60D2300D600D0
:102AB00023800D00A656F3A6068001000100835670
:102AC000090503462905D247B376DA003306CA0260
:102AD0001305800C9355F6413696330DF640825718
:102AE000333CD6002E9C3336A601330CFC40330C0D
:102AF000CC403308850392564E86B335A503330583
:102B0000A503C29597C00100E78000E563468001F8
:102B1000631E0C16630C0D16130615003335A60044
:102B20002E959356F5013696B335D600AA95939611
:102B3000F50105828585D18E6346B000639D051A37
:102B4000638B061A0356C90215823305D600333645
:102B5000C500B2956348B000639105241306F00FD9
:102B6000637DA622894663F3561593078008F3B761
:102B7000078093F78708BED6010001003717004091
:102B8000930770052300F704930780FA2300F704E6
:102B9000010001008356C70289678117D58FC207DC
:102BA000C1832316F70223000704B657F3A7078053
:102BB00001000100FA506A54DA544A59BA592A5AA3
:102BC0009A5A0A5BFA4B6A4CDA4C4A4DBA4D296163
:102BD00082801308F5FF3335A800FD152E95135696
:102BE000F5013298B336C800AA9695B9F336048039
:102BF00093F68608B6CA0100010023809D00238059
:102C0000AD000100010083463905CD8EA309D9042A
:102C100023800D00D646F3A606800100010035B3DF
:102C2000F336048093F68608B6CE010001002380B7
:102C30009D002380CD00010001008346390593E605
:102C40000602A309D90423800D00F646F3A60680E8
:102C50000100010095B3F336048093F68608B6D2DE
:102C60000100010023809D002380CD0001000100B0
:102C70008346390593E60602A309D90423800D0093
:102C80009656F3A606800100010045BB9306F5FFAA
:102C900033B5A600FD152E959355F501AE96B3B547
:102CA000B600AA951396F501858269B5F3360480BE
:102CB00093F68608B6D801000100930680FA2380B7
:102CC0009D002380DD00010001008356C9020566D6
:102CD000011693F6F60FD18EC206C1822316D902D1
:102CE00023800D00C656F3A6068001000100850A68
:102CF00093FAFA0F95B233E6B60045C20356C902FD
:102D00003305D0403338A000B305B040B38505414A
:102D100015826345B000D1E16371A608894663F06E
:102D2000560593078008F3B7078093F78708BEDA44
:102D300001000100B7170040130770052380E70466
:102D4000130780FA2380E7040100010003D7C702BC
:102D50007D8B2396E70223800704D65781BDF33687
:102D6000048093F68608B6DC01000100930680FA21
:102D700023809D002380DD00010001008356C902ED
:102D80000566011693F6F60FD18EC206C182231690
:102D9000D90223800D00E656B9B793078008F3B730
:102DA000078093F78708BEDE010001003717004057
:102DB000930770052300F704930780FA2300F704B4
:102DC000010001000356C70293975600B297C2074D
:102DD000C1832316F70223000704F657C1BB9147AE
:102DE00063EEB70217E70100130787C68A05BA9595
:102DF0009C41BA978287B717004003A7470B13453A
:102E0000F5FF698F23AAE70A03A7070B698F23A899
:102E1000E70A03A7070A798D23A0A70A8280B717BC
:102E2000004083A6470B1347F5FFF98E23AAD70A64
:102E300083A6070B558D23A8A70A83A6070A758FBB
:102E400023A0E70A8280B717004003A7470B498FEA
:102E500023AAE70A03A7070B1345F5FF45BFB717DA
:102E6000004083A6470B1347F5FF758F23AAE70A97
:102E700003A7070A598D4DB7B717004003A7470BA3
:102E8000498FEDB7914763EEB70217E701001307CB
:102E900067BD8A05BA959C41BA978287B7170040EB
:102EA00003A7470D1345F5FF698F23AAE70C03A776
:102EB000070D698F23A8E70C03A7070C798D23A0C2
:102EC000A70C8280B717004083A6470D1347F5FF74
:102ED000F98E23AAD70C83A6070D558D23A8A70C1E
:102EE00083A6070C758F23A0E70C8280B7170040DC
:102EF00003A7470D498F23AAE70C03A7070D134526
:102F0000F5FF45BFB717004083A6470D1347F5FFF0
:102F1000758F23AAE70C03A7070C598D4DB7B71778
:102F2000004003A7470D498FEDB7797122D43714BC
:102F3000004026D24AD0035924028354040206D604
:102F40004209C2044ECE52CC56CA13590901C1805F
:102F50002DE11379F9F793F4F49F4209C204135950
:102F60000901C18093078008F3B7078093F78708AA
:102F70003EC401000100930770052300F404930789
:102F800080FA2300F404010001002311240323101C
:102F9000940223000404A247F3A707800100010064
:102FA000B250225492540259F249624AD24A4561BF
:102FB0008280B7F5070081463000B10519459700BA
:102FC0000020E7806081A24713972701E34A07FCAE
:102FD0001369090893E4044093098008F3B7098052
:102FE00093F787083EC001000100930A7005230093
:102FF0005405130A80FA230044050100010023113F
:10300000240323109402230004048247F3A70780BB
:1030100001000100294597F0FF1FE780A031F3B9B7
:10302000098093F989084EC201000100230054056C
:1030300023004405010001008357040293E70720A1
:103040002310F402230004049247B9B7B7170040D5
:103050008847420541819377050491EB9377F50109
:103060003755E801130505803345F50282809377D3
:10307000050C130700046397E7009377F5013745C4
:103080009C1CCDB72165130505D0828037E700E091
:103090001C435443A183E206D58F1CC1FD57232056
:1030A000F7182322F718828013178500B7E700E08E
:1030B00023A0E710618123A2A7108280B7F700E068
:1030C0008847CC478280814737370040A14663C498
:1030D000C700328582800345B740E38EA6FE338564
:1030E000F5000345050085072304A740CDB79707E2
:1030F0000020938727EF9C4317370020130787464C
:103100003E95636EE500173700201307A74F6368ED
:10311000A700170700202327A7EC3E858280FD57D4
:10312000EDBF8280411122C406C62A8497000000A8
:10313000E78000F22947B307E502B2408D83B3D799
:10314000870222449507B3D7E70237370040C2070A
:10315000C1832316F70041018280411137150E000B
:1031600006C697000000E78020FCB7370040130731
:1031700070F82381E7000D47A381E70013070004DF
:10318000A380E70005472387E700B2404101828022
:10319000B737004003C7170019C9D98DA380B700FE
:1031A00003C70700136787002380E700828093C569
:1031B000F5FFF98DA380B7008280AE872A87B736E6
:1031C000004021463738004089E7170300006700B8
:1031D00083F583C8B600E30916FF05078348F7FFA8
:1031E000FD17C20723041801C183F9BF411122C48E
:1031F00006C62A8497000000E78080E52947B307C8
:10320000E502B2408D83B3D7870222449507B3D736
:10321000E70237370040C207C1832316F740410158
:103220008280716541111305052006C697000000D4
:10323000E78000FCB7370040130770F82381E740B0
:103240000D47A381E74013070004A380E74005472B
:103250002387E740B24041018280CC41411106C63C
:10326000328503C6150083C5050022064D8E420631
:103270008D654186138875A2630C0611634BC804E3
:10328000138845A26300060D634AC800938535A2E2
:103290006301B6082390060029464DA0138855A265
:1032A0006305060D938565A2E316B6FE8D451D46A2
:1032B00063E6E5081146198E63F3C7003E86B7E75B
:1032C00004002390C600FC4797D501009385C57B79
:1032D0009DA0138895A263030611634E060D138803
:1032E000A5A263000613938505A5E315B6FA9945D3
:1032F0001D4663E5E504198E63F3C7003E86B7E714
:1033000004002390C600FC47970500209385C5D78D
:103310001DA09D451D4663E3E5022146198E63F31A
:10332000C7003E86B7E70400FC472390C600970518
:1033300000209385A54CBA9582970146B24032850C
:1033400041018280AD451D46E3EAE5FE3146198E16
:1033500063F3C7003E86B7E704002390C600FC472E
:1033600097D501009385C574F9B7B1451D46E3E7CC
:10337000E5FC3546198E63F3C7003E86B7E70400C7
:103380002390C600FC4797D501009385657365B708
:103390008D451D46E3E4E5FA1146198E63F3C70037
:1033A0003E86B7E704002390C600FC4797D501008E
:1033B0009385456E49B78D451D46E3E1E5F8114615
:1033C000198E63F3C7003E86B7E704002390C6005A
:1033D000FC4797D5010093856570B1BFA5451D4693
:1033E000E3EEE5F42946198E63F3C7003E86B7E79E
:1033F00004002390C600FC4797D501009385456AD9
:103400001DBFB5451D46E3EBE5F23946198E63F362
:10341000C7003E86B7E704002390C600FC4797D557
:1034200001009385656501BFB7E7040003A3071397
:1034300097060020938646C44146A54517050020FF
:10344000130585BA02832D455DE703C505000947CD
:10345000631FE50803A84500411106C6034718008D
:1034600032850346080022074168518F930828FEE1
:103470006307170563E9E800051863030703239052
:103480000600294591A8130648FE630AC7041518CB
:10349000E31707FF15463E87637BF600154701A833
:1034A000130600023E876374F60013070002B7E7B5
:1034B00004002390E600FC471316070111A83E867E
:1034C00091C30546B7E70400FC472390C6004206B7
:1034D000CC45418282970145B2404101828013066A
:1034E00000083E87E375F6FC13070008C9B7239070
:1034F0000600054582808280416779176304E504F0
:10350000411122C406C685472A84639FF500B7E7A8
:10351000040022852244B24003A3871397050020AC
:10352000938505484101028389476399F500B7E710
:10353000040083A7070B8545829771D9B2402244C6
:10354000410182808280797126D252CCAE842A8A4F
:1035500097D501009385855A17D501001305855C21
:1035600006D63AC622D44AD0368432894ECE97C087
:103570000100E780A089A28517D501001305855BAE
:1035800097C00100E7808088294597C00100E78047
:10359000C08C83C7840093F70702F9E383C9040052
:1035A0008947054532476396F908D44083C716001A
:1035B00083C60600A207D58FC166138616FE638CEC
:1035C000C7028D16638FD7068D6693862690294590
:1035D0006391D706B7E70400A286225403A34714D9
:1035E000B250F2494A86A685025992545285624ADF
:1035F0008547456102832D450DEF93070002354550
:1036000063E98702B7E70400FC47C84413060002D9
:10361000CA858297814997070020938727399C4361
:10362000014581CB9C4391C74E852286CA858297EE
:103630000145B250225492540259F249624A4561FE
:1036400082802D457DF79307700F3545E3E387FEB4
:10365000B7E70400FC47C8442286CA85829765BF45
:103660002145C1BF411122C437E4040083278413DC
:1036700026C2AA84416506C6970500209385453277
:103680007D1582978327C40A17050000130505E7F7
:103690008588829795C0032304132244B240924444
:1036A000970600209386C6AF4146C5451705002002
:1036B0001305059E41010283B24022449244014514
:1036C0004101828019C59707002023A1A72E01453B
:1036D0008280454582801147636AA70A97D6010018
:1036E000938686400A0536951841411106C63697DD
:1036F000AE87B2850287130700026145639DE7002C
:10370000B7E70400FC471306000217050020130565
:10371000650F82970145B2404101828005476145AE
:10372000E39BE7FEB7E70400FC47054617050020CA
:103730001305450FF9BF1307700F6145E39DE7FCC3
:10374000B7E70400FC471306700F170500201305A8
:10375000A50DC1B7130700086145E39EE7FAB7E777
:103760000400FC4713060008170500201305451B3D
:103770004DB715476145E390E7FAB7E70400FC470A
:103780001546170500201305E52161B7094582801C
:10379000411126C2B7E4040083A7C41322C44AC05F
:1037A00006C62E84970500209385851F2A89829757
:1037B000058905C5970700209387878D83D7A70BB9
:1037C000A28503A3440D2310F4002244B240924486
:1037D0004A850249014641010283B2402244924493
:1037E0000249494541018280970700202382071C36
:1037F0009707002023A0071CB717004003A7070C5A
:10380000B706C0FFFD16758F23A0E70C03A7070DB1
:10381000B7064000558F23A8E70C03A7070C3D9B74
:1038200023A0E70C03A7070D1367070123A8E70CE4
:103830008280B717004003A5470C83A7470C598126
:1038400013451500C18B058999E31365250097077A
:10385000002083C7E7156380A7029707002023890C
:10386000A71411C9970700209387C71403A3070063
:103870006303030002838280114517F3FFFF670093
:1038800003CA411193962500AA852D4506C697F0D7
:10389000FF1FE78060F4B2400145410182800111C1
:1038A00022CC06CE3714004026CA4AC84EC652C49F
:1038B00083447405034AB405834984050349940588
:1038C00097F0FFFFE78080A08347A40593F4F40FEF
:1038D000137AFA0F93E71700230DF40493F9F90F05
:1038E0001379F90FB717004003C7A705058B6DFFC4
:1038F00003D5C705A38D4705238C3705A38C270562
:10390000A38B9704F2406244D2444249B249224A0E
:103910000561828041119397050122C406C626C223
:10392000C1872E8463DC0700B7E40400FC5482974F
:1039300019C1BC5482972165218D15A893F71500F4
:1039400013C515008DE793F725009DC7970000006C
:10395000E78060EEB7E70400BC4F1306000A894514
:103960001705002003458505829713452400B240C2
:1039700022449244410182809397250163D8070233
:10398000B7E4040083A7C41E829797000000E78075
:10399000E0EEBC4C37560700130606308965170564
:1039A00000200345A5018297096579B79397150112
:1039B0000145E3DE07FA17D501001305A51F97B0EF
:1039C0000100E780805CB7E70400BC4F1306006489
:1039D000916517050020034565FE82971165A9BF13
:1039E0002D71232A9110FD74E98C232C811023283A
:1039F0002111232631112A84AE89328993060010C1
:103A00000A86A6852D45232E111097F0FF1FE7800B
:103A1000A0DC13154401B7E70400FC4751810A05F7
:103A200013962900CA850A958297A6858566014660
:103A3000254597F0FF1FE78020DA0A86A6859306C2
:103A40000010294597F0FF1FE78000D98320C1119E
:103A50000324811183244111032901118329C110F9
:103A600015618280B7F7070003C70701411106C639
:103A700022C426C24AC0A547631DF7009700000074
:103A8000E78040F6B2402244924402490145410198
:103A9000828013942500AA843289A286AA850146D1
:103AA000254597F0FF1FE78020D3A2864A86A6858A
:103AB000294597F0FF1FE78020D2E9B71D71A2CCFE
:103AC00037E404005C5C485886CE494697D501002F
:103AD0009385C509829711E917D501001305450A99
:103AE00097B00100E780604A01A0B7F600E079577F
:103AF00098CAFD57DCCA0567B7E700E023A0E710C6
:103B00001306F00290C223A0E71801000100370756
:103B1000002018471306000481459706002023ADB6
:103B2000E6E84157A38AE7403C4408088297971784
:103B300000209387A7853EC8856713870740231A0F
:103B4000E1001D673ACC37070105130707103ACE8D
:103B5000938757D11307B00F2310E1022312F1020C
:103B6000054797F7FFFF9387A7552301E1023ED84A
:103B700017070000130727D197070000938767D224
:103B8000B7F50700BAC23EDC170700001307C7ED00
:103B900097070000938787CE81463000E1051945DD
:103BA000BAC43EDE97F0FF1FE78000C318088147C4
:103BB000994630003E960346060085070507A30B8D
:103BC000C700E398D7FEC24791C7035741018567F5
:103BD0006373F70001A0B7E7040083A7470A08084A
:103BE0008297AA8511C917D501001305A5FA97B0C8
:103BF0000100E780A02101A0F64066442561828093
:103C0000411126C2B7E4040083A7040806C622C4F3
:103C100017050000130545D08297170400201304F0
:103C2000E4D92300A40097000000E78080029700F9
:103C30000000E780A0BB03450400224403A38405E1
:103C4000B2409244130600328965410102837971C2
:103C500006D622D413078008F337078093F7870826
:103C60003EC201000100B717004093057005238094
:103C7000B704130680FA2380C7040100010083C63D
:103C8000F70293F6A60FA387D70223800704924674
:103C9000F3A60680010001007337078013778708B9
:103CA0003AC4010001002380B7042380C704010047
:103CB000010003C7F70213672700A387E7022380E9
:103CC0000704A247F3A7078001000100054597E01C
:103CD000FFFFE780E06297000000E78020BA01471D
:103CE00081468147054685451305407E97E0FFFFE5
:103CF000E780E06537E404003C44680051468145B4
:103D00008297B707C0A83EC8B787E803938707D054
:103D10003ECA97E7FF1F9387876A3EC67C586800B4
:103D20008297B250225445618280411197D501009B
:103D30009385455017D501001305C5DE06C697B01B
:103D40000100E780A00C17D501001305656997B045
:103D50000100E780A00BB2402945410117B30100E3
:103D60006700A30F411197D501009385E54D17D545
:103D70000100130525DB06C697B00100E7800009A6
:103D800017D501001305856497B00100E78000088E
:103D9000B2402945410117B301006700030C4111EE
:103DA00022C406C6834705002A849DC797D5010013
:103DB0009385454F17D501001305C5D697B001006F
:103DC000E780C0044C4017D501001305A56F97B0DC
:103DD0000100E780A0033DA058410DEF97D50100F9
:103DE0009385454C17D501001305C5D397B0010045
:103DF000E780C00117D501001305456E97B001009B
:103E0000E780C0002244B2402945410117B30100B8
:103E10006700A304A1679386D7036313D70297D5DE
:103E200001009385254817D501001305A5CF97B04C
:103E30000100E780A0FD17D501001305256B7DBFAC
:103E4000ED0797D501009385E54517D501001305CA
:103E500065CD631BF70097B00100E78020FB17D505
:103E600001001305E56959BF97B00100E78000FA2A
:103E70004C4017D501001305A56A91BF411197D594
:103E800001009385A53D17D501001305A5C906C6F8
:103E900097B00100E78080F7B2402945410117B390
:103EA0000100670083FB797122D426D24AD02E8488
:103EB0002A898145B2844800714606D697E0FFFF03
:103EC000E780602497F7FF1F9387474EDC4783D72F
:103ED0000700231421012313F10097500000E7800D
:103EE00040139547A305F1009307401F3EC6FD57B9
:103EF0002305A100230AF10097500000E780A025C8
:103F00002686A285480097500000E7806013B250D3
:103F10002254925402594561828097270020239AA7
:103F200007969727002023830786B7E70400BC473E
:103F3000411106C64146814517050020130545334A
:103F4000829797200000E780807397200000E78029
:103F50008052014597600000E78080A0170700208D
:103F6000034707339307F00A6315F7029307F0F846
:103F70008945170500201305A531170700202309DF
:103F8000F73097070020A385073097600000E7808F
:103F9000C0C797600000E78020F481453705040022
:103FA0009707002023A4072C97070020239E072AA9
:103FB00097070020238B072A97070020239C0722BE
:103FC00097070020239A072097070020239D0728A2
:103FD000970700202396072A97300000E780205A91
:103FE000014597600000E78040CB97D5010093859D
:103FF000652917D501001305E5B297B00100E780E8
:10400000E0E017D501001305E55797B00100E78000
:10401000E0DFB2402945410117B301006700E3E347
:10402000411122C406C626C293F715002E84638F61
:104030000710814617F6FF1F1306863485451705BE
:1040400000200355251997C00000E780E04D15C9F1
:1040500097D501009385C52317D50100130585ACBD
:1040600097B00100E78080DA17D50100130505C578
:1040700097B00100E78080D9294597B00100E7801B
:10408000C0DD97D501009385A52017D50100130544
:1040900065A997B00100E78060D717D50100130527
:1040A00025C397B00100E78060D6294597B001008D
:1040B000E780A0DA17F5FF1F1305452F5C4505477C
:1040C0002390E70097400100E78060FE97D501004C
:1040D0009385051C17D501001305C5A497B00100F1
:1040E000E780C0D217D501001305C5BF97B0010006
:1040F000E780C0D1294597B00100E78000D693073B
:1041000010F8170700202305F7189707002083D71A
:10411000270C17070020A30DF7161705002013051D
:104120002517A1839145170700202304F716970749
:104130000020A380071697600000E78000AD1345BC
:104140001400B240224492444101828093F725003A
:10415000E1C3170700200357271145CB970600201E
:104160009386C610944297D701009387A7431706FA
:1041700000200346860F8145170500201305450FD3
:1041800097700000E780A059AA8441C197D501002B
:104190009385C51817D501001305C59897B0010080
:1041A000E780C0C6A68517D50100130525B597B0D1
:1041B0000100E780A0C5294597B00100E780E0C96C
:1041C000970700202392070A930710F8170700208B
:1041D0002300F70C9707002083D787FF17070020DD
:1041E000A308F70AA183170700202304F70A9145C3
:1041F0008D47170500201305A50917070020A30AFE
:10420000F70897600000E78040A01345240015BF21
:1042100093F74500D1C397D501009385251017D595
:1042200001001305259097B00100E78020BE17D547
:104230000100130565AE97B00100E78020BD294558
:1042400097B00100E78060C1930720F817070020AE
:104250002300F7049707002083D7C7F9170700202A
:10426000A308F702A183170700202304F70285475C
:1042700017070020A30FF70097500000E780A0ED7C
:10428000170500201305C500914597600000E780E1
:10429000C0971345440075B593F78500A9C797D516
:1042A00001009385A50717D501001305A58797B0D1
:1042B0000100E780A0B517D50100130525A797B029
:1042C0000100E780A0B4294597B00100E780E0B87D
:1042D00097070020239A07F897700000E7800054A2
:1042E00013458400B9BD93F70501D1C38545170572
:1042F0000020035525F097600100E780200697D540
:1043000001009385A50117D501001305A58197B07C
:104310000100E780A0AF17D50100130565A297B093
:104320000100E780A0AE294597B00100E780E0B228
:10433000930730F817070020230CF7F497070020A5
:1043400083D747EB17070020A304F7F417050020D5
:10435000130505F4A1838D4517070020230BF7F201
:1043600097600000E780608A13450401D9BB93F78A
:104370000502D1C797D50100938545FA17C50100FD
:104380001305457A97B00100E78040A817D50100D2
:104390001305459D97B00100E78040A7294597B0D8
:1043A0000100E78080AB930740F817070020230146
:1043B000F7EE9707002083D727E217070020A3090D
:1043C000F7ECA183170700202305F7EC85471707B3
:1043D0000020A300F7EC97070020239F07DE9750EB
:1043E0000000E78040D717050020130565EA9145D6
:1043F00097600000E78060811345040299B393F74A
:104400000504FDC397D50100938545F117C501004B
:104410001305457197B00100E780409F17D5010053
:104420001305C59597B00100E780409E294597B0D8
:104430000100E78080A29707002083C767E5130784
:10444000700A6386E7061307800A638CE708130780
:10445000600A6393E704930760F8170700202309B5
:10446000F7E29707002083D707E017070020A30192
:10447000F7E2A18317070020230DF7E08547170710
:104480000020A30CF7E0B14517050020130545E017
:1044900097500000E780607797500000E780A0CB3E
:1044A0001345040497070020239F07DA59B993079F
:1044B00070F817070020230DF7DC9707002083D73B
:1044C00087DA17070020A305F7DCA1831707002070
:1044D0002301F7DC854717070020A30DF7DA99457C
:1044E00065B7930780F8F1B793F705080145E38AAC
:1044F00007C497D50100938565E217C50100130530
:10450000656297B00100E780609017D50100130540
:10451000658897B00100E780608F294597B001005A
:10452000E780A0939307A0F8170700202302F7D68F
:104530009707002083D7C7D417070020A30AF7D412
:10454000A183170700202306F7D48547170700200B
:10455000A301F7D497070020239407D297500000B7
:10456000E78060BF17050020130585D2914597505D
:104570000000E780806913450408E1B6411122C4B8
:1045800097D50100938545D32A8417C501001305EB
:10459000655906C697B00100E78040874C4017D5A3
:1045A00001001305A5EF97B00100E780208629459B
:1045B00097B00100E780608A034704009307F00F7B
:1045C000631FF70297D50100938505CF17C501003A
:1045D0001305455597B00100E78040834C4017D53F
:1045E00001001305A5EC97B00100E780208222446A
:1045F000B2402945410117B3010067000386B2406C
:10460000224441018280B1C1411122C417C5010079
:10461000130545512E8497D501009385E5C406C640
:1046200097A00100E780807EA28517D501001305C1
:1046300025F397A00100E780607D2244B240294520
:10464000410117B30100670043818280411122C4F8
:1046500026C22E84AA8497D501009385A5C117C5CB
:1046600001001305254C06C697A00100E780007ADB
:1046700017D50100130585EF97A00100E7800079A9
:10468000294597A00100E780407D97D501009385DB
:1046900065BE97070020239F97B217C50100130539
:1046A0006548854497070020239487B29707002028
:1046B000239197B297170020239D871C97A0010094
:1046C000E780C0749715002083D5A51C17D501007D
:1046D000130545EA97A00100E7804073294597A09C
:1046E0000100E7808077971700202381970A9720A1
:1046F0000000E78040D8228597500000E7804026E0
:10470000054597500000E780405997F7FF1F9387B2
:10471000E7C9DC4703D70700C167FD176312F7023B
:104720002244B7E70400B240924403A3870517F57B
:10473000FF1F034525291306000A85454101028311
:10474000B2402244924441018280011122CC37E4DC
:1047500004005C5C06CE354697D50100938585C97B
:1047600017E50100130585B0829711E917C501000F
:104770001305054197B00100E780208101A097F75C
:10478000FF1F9387E7243EC4B7F50700856793872B
:104790000780814617F6FF1F13060623E10519451A
:1047A0003EC697E0FF1FE78020037C44194697F53B
:1047B000FF1F93856521170500201305E5A3829748
:1047C000340017F6FF1F1306262097D501009385A6
:1047D000651217D501001305651397700000E78077
:1047E00000C92A841DCD97D50100938525B017C532
:1047F00001001305253397A00100E7802061A28501
:1048000017D50100130505C097A00100E7800060DF
:10481000294597A00100E7804064F24062440561A9
:10482000828097E00000E780602B17D50100130518
:1048300065B497600000E78040BD97A00000E78066
:10484000A07F97600100E78020E417F5FF1F1305A4
:1048500065B297600100E780C0CC17D50100130551
:1048600065B297600100E780A0E42A8497600000A9
:10487000E780802397100100E78000BC978001004B
:10488000E780205597700000E780C07B977000009C
:10489000E780809997300100E780607D97D501001F
:1048A0009385C5A417C501001305C52719C897A08E
:1048B0000100E780A055A28517D501001305C5B6F4
:1048C000A1B797A00100E780605417D50100130538
:1048D000E5B797A00100E7806053294597A0010044
:1048E000E780A05797300100E780405997F000001B
:1048F000E780007855C985453705040097300000EA
:10490000E780E0C797D501009385459E17C5010054
:104910001305452197A00100E780404F17D50100FE
:10492000130545B497A00100E780404E294597A0A4
:104930000100E780805297F7FF1F9387E79683D7A0
:104940000700171700202316F7F4854717170020D4
:10495000230EF7E297200000E78020CB972000008D
:10496000E78060B1171500200355A5F297500000AD
:10497000E78000FF054597500000E780003297D59B
:1049800001009385A59617C501001305A51997A0E9
:104990000100E780A04717D501001305E5AE97A0F9
:1049A0000100E780A046ADB597D501009385059439
:1049B00017C501001305051797A00100E780004502
:1049C00017D50100130505BC97A00100E78000443E
:1049D000294597A00100E7804048014569BF411182
:1049E00022C437E404008327041A06C6829797502E
:1049F0000000E780A0FA8327040817F5FFFF1305DE
:104A00006562829797F7FF1F238EA7FA17F5FF1F9E
:104A10001305C59997500000E78080A62244B24054
:104A2000410117030000670083D2411106C622C46A
:104A300026C299C1AA8415ED97D501009385058CEE
:104A400017C501001305050E97A00100E780003C83
:104A500017C501001305C52497A00100E780003B9E
:104A60002244B24092442945410117A30100670046
:104A7000C33E37E404007C44414617F5FF1F13058D
:104A8000257F829717F5FF1F1305857E972000006D
:104A9000E780A0B397200000E780E09D0323840512
:104AA000224497F7FF1F2391977CB240924417F559
:104AB000FF1F034525F11306000A894541010283C2
:104AC000B7E70400FC471171A2DDCAD986DFA6DB77
:104AD000CED72E8432892E86AA8517F5FF1F13059F
:104AE000257B829717F7FF1F1307877A83470700F5
:104AF000930680029387E70793F7F70FE3ECF6102E
:104B0000BA898A0717C701001307070BBA979C4396
:104B1000BA9782878D4797D501009385658117C520
:104B2000010013052500630FF40097A00100E78042
:104B3000E02D17C501001305653C97A00100E78033
:104B4000E02CBDA497A00100E780402C17C5010010
:104B50001305453C97A00100E780402B294597A00D
:104B60000100E780802F930720F8114697F5FF1F7B
:104B7000938505724A8517F7FF1F230BF77097F788
:104B8000FF1FA388077097F0FFFFE78000322A8499
:104B90001DC997C501009385A57917C501001305A7
:104BA00065F897A00100E7806026A28517C501007F
:104BB0001305053A97A00100E7804025294597A0F5
:104BC0000100E780802997C501009385657617C5A8
:104BD0000100130525F597A00100E780202317C5E4
:104BE00001001305253897A00100E7802022294500
:104BF00097A00100E78060264165930730FA0546DB
:104C000097F5FF1F9385C5687D1517F7FF1F2301D3
:104C1000F76897F0FFFFE78040292A841DC997C5F0
:104C200001009385E57017C501001305A5EF97A056
:104C30000100E780A01DA28517C5010013054531BD
:104C400097A00100E780801C294597A00100E7801C
:104C5000C020B7E70400BC4F0566130606C8A1458F
:104C600017F5FF1F034505D68297FE506E54DE549C
:104C70004E59BE591161828091476303F40297C572
:104C800001009385E56A17C501001305A5E997A002
:104C90000100E780A01717C501001305E52F71BDBE
:104CA000B7E70400FC4F914517F5FF1F034585D179
:104CB000829797C501009385A56717C50100130565
:104CC00065E697A00100E780601417C50100130591
:104CD000652E97A00100E7806013294597A0010089
:104CE000E780A01797400000E780E046914535A493
:104CF00085476303F40297C501009385656317C573
:104D00000100130525E297A00100E780201017C5D8
:104D100001001305A52B15B597F7FF1F239C274D01
:104D2000B7E704000566BC4F130606C8C1450DBFB2
:104D30008D476303F40297C501009385655F17C52E
:104D40000100130525DE97A00100E780200C17C5A0
:104D5000010013056529D5B3930740F8114697F56F
:104D6000FF1F9385E5524A8517F7FF1F2302F7526D
:104D700097F7FF1FA38F075097F0FFFFE780E01220
:104D80002A84E30405EE97C501009385655A17C58B
:104D90000100130525D997A00100E7802007A2850F
:104DA00017C501001305C51A97A00100E78000068A
:104DB000294597A00100E780400A45BD9147E31CC3
:104DC000F4F6B7E70400FC4F9305000217F5FF1F48
:104DD000034545BF829797C501009385655517C563
:104DE0000100130525D497A00100E780200217C514
:104DF00001001305E520F1BD894763E3870297C5EC
:104E000001009385E55217C501001305A5D197A0B0
:104E10000100E780A0FF17C501001305A51F31BBE6
:104E200097F4FF1F83C4E44697F7FF1F83C75746D5
:104E300097C501009385C54FA20417C5010013054E
:104E400065CEDD8C97A00100E78040FCA28517C5E8
:104E500001001305651D97A00100E78020FBC20437
:104E6000294597A00100E78040FFC1849305D4FF46
:104E700093960401C1824A8693F5F50F17F5FF1F3B
:104E80001305354197200000E7802073E35F90DC35
:104E9000930750F817F7FF1F230CF73E83C739001D
:104EA000228697F5FF1F9385A53E85074A8517F74C
:104EB000FF1FA300F73E97F0FFFFE78000FF2A8463
:104EC000E30505DA97C501009385854617C50100FE
:104ED000130545C597A00100E78040F3A28517C5DB
:104EE00001001305E566C9B5894763E3870297C5E5
:104EF00001009385E54317C501001305A5C297A0DE
:104F00000100E780A0F017C501001305A51335B116
:104F100097400000E7802024A28517F5FF1F1305A6
:104F2000253797500000E78040CE81B38D4763035B
:104F3000F40297C501009385A53F17C5010013052D
:104F400065BE97A00100E78060EC17C5010013055E
:104F50002511E5B6B76602000146B77502000545A2
:104F600097E0FF1FE7804087930760F817F7FF1F60
:104F70002300F73297F7FF1FA38D07309307000632
:104F800017F7FF1F2308F730894717F7FF1FA30301
:104F9000F73097F7FF1F2380073097F7FF1FA38C89
:104FA000072EC14717F7FF1F2308F72E930720F995
:104FB00017F7FF1FA302F72E314697F7FF1FA38EA7
:104FC000A72C97F5FF1F9385A52C4A8597F7FF1F00
:104FD0002385072C97F0FFFFE78020ED2A84E30666
:104FE00005C897C501009385A53417C501001305B1
:104FF00065B397A00100E78060E1A28517C50100B5
:105000001305850755B3B1476303F40297C5010043
:105010009385053217C501001305C5B097A001009F
:10502000E780C0DE17C501001305C50639B6B7E72E
:105030000400FC4F9305000417F5FF1F03458598F6
:10504000829797400000E7800011B145F9B591477C
:1050500063E3870297C501009385852D17C501007D
:10506000130545AC97A00100E78040DA17C50100A1
:1050700013050504D9B497F4FF1F83C4A42197F73F
:10508000FF1F83C71721A204DD8C8E04B7770200AF
:105090006D14BE942286A68517C5010013058502EE
:1050A00097A00100E78080D6B7E70400FC4722867E
:1050B00097F5FF1F9385151E28008297931604010C
:1050C000C1823000A685094597D0FF1FE780C070D8
:1050D0002A8409C917C501001305850097A001009E
:1050E000E780A0EA930770F8194697F5FF1F9385AC
:1050F000251A4A8517F7FF1F230CF71897F7FF1F8C
:10510000A38A871897F0FFFFE78020DA2A84E30E4E
:1051100005B497C501009385A52117C501001305A6
:1051200065A097A00100E78060CEA28517C50100A9
:10513000130505FC95B99947630BF41297C5010057
:105140009385051F17C501001305C59D97A0010094
:10515000E780C0CB17C50100130505FBF9BA9147DD
:1051600063E3870297C501009385851C17C501007D
:105170001305459B97A00100E78040C917C50100B2
:10518000130505FA5DBA97F4FF1F83C4A41097F7BF
:10519000FF1F83C71710A204DD8C8E04B7770200AF
:1051A0006D14BE942286A68517C50100130585F8E7
:1051B00097A00100E78080C5B7E70400FC4722867E
:1051C00097F5FF1F9385150D28008297931604010C
:1051D000C1823000A6850D4597D0FF1FE780C05FD4
:1051E0002A8409C917C50100130585F697A0010097
:1051F000E780A0D9930780F8194697F5FF1F93859C
:1052000025094A8517F7FF1F2304F70897F7FF1FA3
:10521000A382870897F0FFFFE78020C92A84E3066E
:1052200005A497C501009385A51017C501001305B6
:10523000658F97A00100E78060BDA28517C50100BA
:10524000130545F295B699476303F40297C501002B
:105250009385050E17C501001305C58C97A00100A5
:10526000E780C0BA17C50100130545F1F9B0B7E7EB
:105270000400FC4F9305000417E5FF1F03458574E8
:10528000829797400000E78000ED994579B18D47FE
:105290006303F40297C501009385850917C50100D2
:1052A0001305458897A00100E78040B617C50100A7
:1052B000130545EE59B017C501001305A5EE97A0DB
:1052C0000100E78080CC1305C01297D0FF1FE78054
:1052D0004007014597E0FFFFE78080DB0D45971011
:1052E0000000E780E0A3294597D0FF1FE780600515
:1052F00097D0FF1FE780C0F58DBA99476303F4028A
:1053000097C501009385C50217C501001305858166
:1053100097A00100E78080AF17C50100130545E99C
:1053200029B817F7FF1F0347F7F697F7FF1F83C743
:1053300067F622075D8F9166BA96C2061166C18232
:105340001306F6EF8D476365D60297E7FF1F938735
:10535000E7059C4B17F6FF1F0346B6F39386C7007D
:105360002DC203D6070069CA8907E39CD7FE894787
:105370001307A0F8114697F5FF1F938565F14A853D
:1053800097F6FF1F2386E6F017F7FF1FA303F7F03A
:1053900097F0FFFFE78060B12A84E308058C97C58A
:1053A00001009385E5F817B501001305A57797A0CF
:1053B0000100E780A0A5A28517C50100130585E0BF
:1053C000E5B203D60700630EE60A8907E39BF6FE03
:1053D0008D4779BF91476304F40297C50100938517
:1053E00025F517B501001305E57397A00100E780C7
:1053F000E0A117C50100130565DE6FF00FF4B7E7F4
:105400000400FC4F9305000817E5FF1F0345855B6B
:105410008297C9B897C50100938585F117B501003A
:105420001305457097A00100E780409E17C5010055
:10543000130545DC6FF06FF02390E70017E5FF1FC1
:105440001305C5F697300100E780C0C897C5010075
:10545000938505EE17B501001305C56C97A00100F3
:10546000E780C09A17C501001305C5D997A00100B0
:10547000E780C099294597A00100E780009E8147F9
:10548000C5BD2390070017E5FF1F130525F29730D0
:105490000100E78020C497C50100938565E917B531
:1054A00001001305256897A00100E780209617C525
:1054B00001001305A5D65DBF411122C406C626C250
:1054C0004AC0834705002A84A1C397C5010093857C
:1054D000E5DF17B501001305E56497A00100E7803B
:1054E000E0924C4017C501001305C50C97A00100C0
:1054F000E780C0912244B2409244024929454101CB
:1055000017A30100670063955841B707CF00938741
:10551000777D631CF7080445638504120359C500B1
:10552000630109120354E50097C50100938505DA6C
:1055300017B501001305055F97A00100E780008DF6
:1055400003C60400A286CA8517C501001305050815
:1055500097A00100E780808B294597A00100E78094
:10556000C08F4A86A685228597200000E780E0DF6D
:1055700083C7140003C70400A207D98F13978700BD
:10558000A183D98FC2073167C1831307C755638AC7
:10559000E70A22862244B240CA85268502499244FF
:1055A000410117F3FFFF6700E351B707CC00938772
:1055B000777D6310F70697C50100938525D117B550
:1055C00001001305255697A00100E78020841C44A4
:1055D0008355C4008356E40003C6070017C50100C5
:1055E0001305C5FE97A00100E7804082294597A0DA
:1055F0000100E78080860356C4000C440355E40094
:105600002244B2409244024941011723000067003E
:10561000C3D5B707CE009387777D6304F70297C59C
:1056200001009385A5CA17B501001305A54F9790F2
:105630000100E780A07D4C4017C50100130545EE31
:1056400075B5B24022449244024941018280B7E7D5
:105650000400FC4741112E8606C622C426C24AC059
:105660002E842A89AA8517F5FF1F130565C2829724
:1056700097C50100938585CD17B501001305854AAF
:1056800097900100E780807897F5FF1F83C545C09C
:1056900017B501001305857197900100E780007729
:1056A000294597900100E780407B97F4FF1F938482
:1056B00024BE83C7040041479387070693F7F70F7B
:1056C000636AF75C17B70100130747598A07BA974F
:1056D0009C43BA9782879D476307F40297C50100F0
:1056E0009385C5C617B501001305C5439790010002
:1056F000E780C07117B501001305C56B97900100D5
:10570000E780C070ADAC97F7FF1F83C777B8DDCBDC
:1057100017F7FF1F0347F7B797F7FF1F83C767B751
:1057200022075D8F97F7FF1F83C7C7B6C2075D8F3C
:1057300097F7FF1F83C717B6E207D98F17F7FF1F29
:105740002326F7B283C7640097C50100938505C07F
:1057500017B501001305053D17F7FF1F2307F7B025
:1057600097900100E780806A97F7FF1F938707B043
:105770008C4317F6FF1F034646AF17B5010013050C
:10578000256597900100E7806068294597900100A2
:10579000E780A06C97F7FF1FA38C07AE2244B240AE
:1057A00092440249930700F817F7FF1F2302F7AE50
:1057B0009D4517F5FF1F1305A5AD410117430000D7
:1057C0006700A34497600000E780C01497F7FF1FAD
:1057D0002381A7AC9357850017F7FF1FA30BF7AAE8
:1057E000935705012A8417F7FF1F2305F7AA93573C
:1057F0008501014517F7FF1FA30EF7A8976000006A
:10580000E780001297F7FF1F2387A7A897C501001D
:105810009385C5B317B501001305C53097900100F6
:10582000E780C05E17F6FF1F0346E6A6A28517B500
:1058300001001305655BB1B7CD476303F40297C55B
:1058400001009385A5B017B501001305A52D97900C
:105850000100E780A05B17B501001305655A79BD0B
:1058600037E404007C44414697F5FF1F938555A219
:1058700017F5FF1F1305C59F829717F5FF1F130527
:10588000259F97100000E78040D497100000E78024
:1058900080BE97F7FF1F83C7C7A017F7FF1F0347F7
:1058A00037A0A20703238405D98F17F7FF1F231DF5
:1058B000F79A1306000A89452244B24092440249ED
:1058C00017E5FF1F03450510410102838D47630360
:1058D000F40297C50100938565A717B5010013056C
:1058E000652497900100E780605217B50100130509
:1058F000E56029B517F4FF1F0344A49997F7FF1F2C
:1059000083C7179997C50100938545A4220417B54D
:105910000100130525215D8C97900100E780004F61
:10592000A28517B501001305254F97900100E78068
:10593000E04D294597900100E78020520D4697F5EC
:10594000FF1F9385E594228597E0FFFFE780E055F0
:10595000AA8421C197C501009385459F17B5010011
:105960001305451C97900100E780404AA68517B5AE
:1059700001001305A54B97900100E78020492244C0
:10598000B240924402492945410117930100670042
:10599000C34C97F7FF1F239F8784B7E70400116666
:1059A00003A38705130606E8914539B78D476303BE
:1059B000F40297C501009385659917B50100130599
:1059C000651697900100E780604417B50100130544
:1059D000A5612DB317F4FF1F0344A48B97F7FF1F96
:1059E00083C7178B97C5010093854596220417B589
:1059F0000100130525135D8C97900100E78000419D
:105A0000A28517B501001305A54397900100E78013
:105A1000E03F294597900100E78020440D4697F527
:105A2000FF1F9385E586228597E0FFFFE780E0472B
:105A3000AA841DC197C501009385459117B5010042
:105A40001305450E97900100E780403CA68517B5E9
:105A500001001305254005B797E7FF1F239E8776B2
:105A6000B7E70400116603A38705130606E893054C
:105A7000000299B5894763E3870297C501009385C2
:105A8000E58C17B501001305E50997900100E78043
:105A9000E03717B501001305E5578DB197E4FF1FF7
:105AA00083C4247F97E7FF1F83C7977E97C50100B4
:105AB0009385C589A20417B501001305A506DD8CE1
:105AC00097900100E7808034A68517B50100130583
:105AD000E53997900100E7806033294597900100F0
:105AE000E780A037228697E5FF1F9385657A268594
:105AF00097E0FFFFE780603B2A84630E051A97C595
:105B000001009385A58417B501001305A5019790A1
:105B10000100E780A02FA28517B5010013054536C7
:105B200099BD854763F98718834519002244B2401F
:105B300092440249B335B00097E7FF1F2386B76C44
:105B400017B50100130505354101179301006700E2
:105B5000E32BA2852244B24092444A850249410186
:105B6000170300006700032299476303F40297B507
:105B700001009385A57D17B501001305A5FA97903F
:105B80000100E780A02817B5010013056562BDB6C6
:105B900017E4FF1F0344E46F97E7FF1F83C7576FA6
:105BA00097B501009385857A220417B50100130586
:105BB00065F75D8C97900100E7804025A28517B5B9
:105BC00001001305A52E97900100E78020242945A8
:105BD00097900100E7806028194697E5FF1F93859D
:105BE000256B228597E0FFFFE780202CAA841DC14A
:105BF00097B501009385857517B50100130585F2EA
:105C000097900100E7808020A68517B50100130555
:105C1000E52A95B397E7FF1F23948766B7E704004B
:105C2000116603A38705130606E89305000869B10A
:105C3000854797B501009385657117B50100130578
:105C400065EE630BF40097900100E780201C17B508
:105C500001001305E5275DB497900100E780001B64
:105C600017B501001305452897900100E780001A39
:105C7000294597900100E780401E2244B24092449B
:105C8000024997E7FF1F2391075E41011763000058
:105C90006700C3B897B501009385456B17B5010040
:105CA000130545E897900100E780401617B50100FD
:105CB00013054554A1B4B240224492440249410123
:105CC0008280411106C622C497E0FFFFE780E01DF5
:105CD0009377F50FA1C32A8497B501009385856852
:105CE00017B50100130505E497900100E780001245
:105CF0009375F40F17C50100130585859790010072
:105D0000E780C0102244B2402945410117930100A9
:105D10006700A314B240224441018280411122C491
:105D200091462A8417E6FF1F1306C6649D652D451C
:105D300006C697D0FF1FE78020AAB7F7070003C762
:105D40000701A5476313F70001A093060010014661
:105D50009D65254597D0FF1FE78000A897E7FF1FA7
:105D6000238A87602244B240914617E6FF1F13063C
:105D700066609D652945410117D3FF1F6700C3A5D4
:105D80001171CED7B7E9040083A7C904CAD917E9AE
:105D9000FF1F1309E94FA2DD2E8686DFA6DB2E84C6
:105DA000AA854A85829797E7FF1F83C7674E130727
:105DB000700A6385E710636DF7001307600A638557
:105DC000E704FE506E54DE544E59BE591161828074
:105DD0001307800A6385E7161307900AE393E7FE2B
:105DE0008D476306F41C97C501009385A58917B5F7
:105DF0000100130525D397900100E780200117C506
:105E000001001305658525A08D47630CF40297C535
:105E100001009385258717B501001305A5D097903C
:105E20000100E780A0FE17B501001305257C9790BF
:105E30000100E780A0FD294597900100E780E0017F
:105E400049B7854717B501001305057C17E7FF1F04
:105E5000230CF73A97900100E7802013B7750200F2
:105E6000B76602000146054597D0FF1FE780C09640
:105E7000930760F817E7FF1F230CF74097E7FF1F12
:105E8000A38907409307002617E7FF1F2324F74045
:105E9000E5779387072117E7FF1F231FF73EB145DB
:105EA00097E7FF1F238B073E97E7FF1FA387A73EB8
:105EB0004A8597000000E780401621B7914763E3C9
:105EC000870297B501009385E57B17B5010013059F
:105ED00065C597900100E78060F317B501001305D1
:105EE000A574B1B797E4FF1F83C4C43A97E7FF1FB7
:105EF00083C7373AA204DD8C83A7C9046D142286B8
:105F000097E5FF1F93851539280082978E04931615
:105F10000401B7750200C1823000A695094597D0EB
:105F2000FF1FE780608B930770F817E7FF1F2301BF
:105F3000F736994597E7FF1FA38EA73495BF914782
:105F400063E3870297B501009385C57317B5010018
:105F5000130545BD97900100E78040EB17B50100A0
:105F60001305056EE9B597E4FF1F83C4A43297E7D4
:105F7000FF1F83C71732A204DD8C83A7C9046D14E9
:105F8000228697E5FF1F9385F530280082978E04BF
:105F900093160401B7750200C1823000A6950D4525
:105FA00097D0FF1FE7804083930780F8BDBF17B5E8
:105FB00001001305A56B97900100E78000FD930792
:105FC00090F82304F100834719008D452800A304AD
:105FD000F100834729002305F10097000000E780C6
:105FE000C0031305C01297C0FF1FE780803501452D
:105FF00097D0FFFFE780C0090D4597000000E780BC
:1060000020D2294597C0FF1FE780A03397C0FF1F0C
:10601000E78000247DB397E7FF1F9387A73603A38C
:106020000700630303000283174300006700E3BD1A
:1060300041114AC09706002083D6A685328917D61B
:10604000FF1F0356C63822C426C206C62A84AE8461
:1060500097000000E780A06A35C12DC0994763FF13
:1060600097048347140003470400A207D98F1397AE
:106070008700A183D98FC2073167C1831307C75532
:10608000639EE70297D7FF1F83D76734A301F4000D
:10609000A1832302F40097F7FF1F83D7877F91C75F
:1060A000A302F400A1832303F400A68517B5010021
:1060B0001305456197900100E78040D597F7FF1FD2
:1060C00083C7C76CB9CF97D5FF1F83D5453017B5A8
:1060D00001001305E56097900100E78020D3268634
:1060E000A28517D5FF1F0355852E97000000E78076
:1060F00080BD6301090497E7FF1F83C7E7289DCB95
:1061000095C897E7FF1F83C727108DE72285224494
:10611000B2400249A685924441011743000067003E
:10612000C3AE17B501001305A55C97900100E78089
:10613000C0E5C1B7B2402244924402494101828085
:10614000011126CA06CE22CC0344550083474500E0
:10615000AA8422045D8C2EC617B50100130545558F
:10616000A28597900100E78060CA2285624432468A
:10617000F240A685D2440561170300006700A3B46E
:10618000011122CC2A8417B501001305655106CEF2
:106190002EC697900100E78040DF22856244B24519
:1061A000F2400561171300006700832A8D4763FBE7
:1061B000B70A011126CA06CE22CC0344350097E463
:1061C000FF1F83C4741C97B5010093852553B33713
:1061D000800017E7FF1FA309F71A09C497B501004C
:1061E0009385855217B501001305855297900100DC
:1061F000E780C0C197E7FF1F83C717196386970021
:1062000097000000E780603097E7FF1F83C7D7172C
:106210008DC785472306F100B7E7040083A747171A
:106220007000854513055030829717B5010013059E
:10623000254F97900100E78040D59967938757EEE7
:106240002316F100680085479145A30781002307C5
:10625000F10097000000E78040DCF2406244D24445
:10626000056182808280894763F7B708011122CCDB
:1062700006CE26CA8344250085472A84639DF404FC
:10628000914763F5B7040345450083473400220571
:106290005D8D97D7FF1F239CA71297000000E78012
:1062A000E04E9967938767EE2314F100834734002B
:1062B00023059100A305F10083474400954528007C
:1062C0002306F10097000000E78020D5F2406244E9
:1062D000D24405618280FDF89967938767EE2314A5
:1062E000F10097D7FF1F83D7870EA305F100230581
:1062F0000100A183E1B782800111996722CCD517F3
:1063000017F4FF1F130484482314F100834704008B
:1063100026CA97F4FF1F9384C4572305F10083D73F
:10632000040028009545A305F100A18306CE2306AD
:10633000F10097000000E78040CE03D604008345BB
:10634000040017B501001305253F97900100E78071
:10635000E0ABF2406244D244056182809D6779716E
:10636000D9172316F10097F7FF1F83C7274206D6D8
:106370002307F100A9C3B7E70400FC47414697E5AE
:10638000FF1F9385E5EE1305F10082976800CD4568
:1063900097000000E78060C897F5FF1F83C5053FA1
:1063A00017B501001305453C97900100E78000A652
:1063B000B25045618280B7E70400BC474146814541
:1063C0001305F1008297D9B745C5411106C622C40D
:1063D000930750FA2300F5009307A005A300F500EA
:1063E00089472301F5009147A301F5009307500366
:1063F000A302F50097F7FF1F9387473983C707006C
:10640000230205002A842303F50097E7FF1F9387E3
:10641000B7F783C70700414697E5FF1F938545E51A
:10642000A303F50097F7FF1F83D7A7462304F500C2
:10643000A183A304F50097D7FF1F83D747F923054E
:10644000F500A183A305F500B7E70400FC4731057B
:1064500082972285F14597000000E7804026230EB1
:10646000A4002181A30EA400B240224441018280F5
:1064700082805D710A8586C6A2C497000000E7800D
:10648000E0F437E404007C448A850810794682975A
:106490003C441305E103094681458297101093059A
:1064A0000002014597D0FFFFE7802023B640264435
:1064B00061618280011122CC2A84680006CE26CA3E
:1064C0004AC8AE84328902C697D0FFFFE78040BC3D
:1064D000A28585660146254597C0FF1FE780C02F2E
:1064E000CA862686A285294597C0FF1FE780C02E51
:1064F000324597D0FFFFE78060BBF2406244D24450
:106500004249056182800111B7C7A55A22CC938701
:10651000C73317E4FF1F130434E73EC48347040066
:106520002C002146196506CE3EC697000000E78084
:10653000A0F88345040017B501001305A533979013
:106540000100E780A08CF240624405618280011165
:10655000A146300099652D4522CC06CE97C0FF1F7D
:10656000E7808027A24737C4A55A1304C433639534
:106570008702B24517B5010013050523B335B000F6
:1065800097E7FF1FA382B7E097900100E78000889C
:10659000F2406244056182809165A1463000938596
:1065A00005F02D4597C0FF1FE7800023A247E38237
:1065B00087FC97E7FF1FA38907DC814517B501001A
:1065C0001305C520D1B7B7C7A55A79719387F73599
:1065D0003EC6B7E70400FC4706D6AA854146080830
:1065E00082976C005146116597000000E780C0EC6F
:1065F00017B501001305C52B97900100E780E098BF
:10660000B250456182807971D146700091652D4507
:1066100022D406D697C0FF1FE780001CB24737C4BC
:10662000A55A1304F43563988702B7E70400FC47C2
:1066300017E5FF1F1305C5C341460C08829717B520
:1066400001001305A51E97900100E7800094B25049
:106650002254456182809165D1467000938505E89A
:106660002D4597C0FF1FE7802017B247E38F87FAB9
:1066700017B501001305851DF9B70111680006CE95
:1066800002C697D0FFFFE780A0A08566014691650E
:10669000254597C0FF1FE7802014324597D0FFFFA4
:1066A000E780C0A017B501001305450E97900100C3
:1066B000E780A08DF24005618280C16769768146DE
:1066C000FD1705061397060141836364B7003E85F5
:1066D00082803307D50003470700B98F214713F89D
:1066E0001700858363050800B18FC207C1837D173A
:1066F0001377F70F6DF78506F1B741C5A547054735
:1067000063F2B70883471500034705003168A20705
:10671000D98F13978700A183D98FC207C18313082C
:10672000C855054763900707411106C622C426C213
:1067300003442500914763F087049307540063ECFA
:10674000F502A301C50021822302C5009304340091
:1067500091C6A302D500A1822303D5002A84A68571
:1067600097000000E780A0F526942300A400218173
:10677000A300A4000147B240224492443A8541015B
:10678000828005473A8582800111B7C7A55A22CC7D
:106790009387E7342A842AC621462C00156506CE45
:1067A0003EC497000000E78020D1A28517B5010004
:1067B0001305450E97800100E780406597000000B3
:1067C000E78060CBF2406244056182800111A146FE
:1067D000300095652D4522CC06CE97C0FF1FE7807F
:1067E000A0FFA24737C4A55A1304E4346395870277
:1067F000B24517B50100130565FF97D7FF1F239812
:10680000B7BCC205C18197800100E7802060F240DB
:106810006244056182809165A1463000938505EE52
:106820002D4597C0FF1FE78020FBA247E38287FC2E
:10683000D14717D7FF1F231CF7B8D14517B5010063
:106840001305C5FCC9B7411122C406C693F715004C
:106850002E8485CBAD67371700409387A7AA1CC34A
:10686000B7E70400BC4F13060019854517D5FF1F75
:106870000345C5B5829713451400B2402244410137
:10688000828093F7250081CB97F7FF1F23920700A3
:1068900013C52500DDB793F745000145F9DF17B5AE
:1068A00001001305E50297800100E780006E973034
:1068B0000000E780206413454400C1B7411122C4A1
:1068C00037E404005C5C06C6354697B50100938545
:1068D00065B217C5010013056599829711E917B5CF
:1068E00001001305A5FF97800100E780006A01A061
:1068F0008327041C82972A84054597C00000E780FF
:10690000401D97700100E78060A297600100E7805A
:10691000607797B00000E780C02E2285B240224405
:10692000410182801567B71700401307575598C378
:10693000D8439D66558FD8C3D843FD76758FD8C38D
:10694000D8431367F70FD8C335671307C7CC98C36D
:1069500082804111054506C622C426C297C0FFFFAA
:10696000E780E05C1305A00497B0FF1FE780207468
:10697000757585457D1597C0FFFFE78080467D755D
:1069800085451305F53697C0FFFFE780E04F3714C4
:1069900000408327840A8D451305002093E70720D4
:1069A0002324F40A97C0FFFFE780A043B7E4040064
:1069B00097D0FFFFE7802087C85897800100E780C5
:1069C000C05C17C501001305658A97800100E78048
:1069D000C05B8327840C8545414593E70708232442
:1069E000F40C97C0FFFFE780204A8D45130500088F
:1069F00097C0FFFFE780404997C0FFFFE780207600
:106A000037A507001305051297C0FFFFE780C07187
:106A10009D45014597C0FFFFE780C077B7E700E0DD
:106A20003707000423A0E7180100010097D0FFFFFB
:106A3000E780000997D0FFFFE780C01C97000000A7
:106A4000E78000E897000000E780A0B09700000012
:106A5000E78000D897E0FFFFE780A0F897000000EC
:106A6000E780003597100000E780E0AE9710000047
:106A7000E780E0A983A70408170500001305E5DCFB
:106A8000829797D7FF1F2383A794BC4C13060064FB
:106A90008545829797000000E78000E997C0FF1FB7
:106AA000E780009501458280B7F7070003C707011B
:106AB000A547AE866316F7009397450191C301A0E1
:106AC000AA850146254517C3FF1F6700E3D0411182
:106AD000B2862E86AA852D4506C697C0FF1FE78081
:106AE000A0CFB2400145410182809307000463E8D2
:106AF000C7021D71A2CC2A84080886CE32C69780B0
:106B00000100E7804025B2461008A285294597C0BC
:106B1000FF1FE78060CCF6406644256182803955CE
:106B2000828097F7FF1FA38507E697F7FF1F238152
:106B300007FC97F7FF1F238D07E4B7E70400FC5F0E
:106B4000411106C682978967938707F4B2403E9544
:106B500097F7FF1F23AAA7D841018280930600025E
:106B60002547830705006385D7006383E70082809C
:106B70000505C5BF17F5FF1F0345E5D60DE5411116
:106B800022C417F4FF1F130424D61C4006C681CB71
:106B9000B7E70400FC5F82971C401D8D7D81B240E9
:106BA00022444101828005458280411106C622C4EB
:106BB00081473307F500030707002DEF97F6FF1F06
:106BC00083D6E6DC17F7FF1F035747DC63EAE600CE
:106BD00017F7FF1F231C07DA17F7FF1F231907DA20
:106BE00097F6FF1F83D686DA1307000A158F3A84BB
:106BF0004207418363F3E7003E84420441801DC4A1
:106C0000B7E70400FC47AA8517F5FF1F130505CE5B
:106C100022863695829797F7FF1F938727D783D7CA
:106C200007003E9497F7FF1F239287D6B240224475
:106C3000410182808507C207C183A5BFAA8713755A
:106C4000F50F130705FD1377F70FA54663E5E6007B
:106C5000138507FD82801307F5F91377F70FE546D3
:106C600063E6E600011593178501E1871387F7FBBB
:106C70001377F70F95467D5563E4E600138597FC7F
:106C8000828035C5011126CA4AC84EC652C406CEF6
:106C900022CCAE8997000000E78080EC2A898144ED
:106CA000414A0305090097000000E78060F92A8443
:106CB0000305190097000000E78080F8634704028D
:106CC000634505021204B3879900498C238087002D
:106CD00085040909E39744FD0545F2406244D24426
:106CE0004249B249224A056182800145FDB701450A
:106CF00082808147E5483387F5000307070019E3E1
:106D000005458280B306F500038606009376F60FEC
:106D10001388F6F91378F80F63E6080181161396C5
:106D2000860161869376F70F1388F6F91378F80FCA
:106D300063E60801138706FE620761876316C700D2
:106D40008507C207C18345BF01458280011122CC5E
:106D50002A842E8526CA4AC84EC606CE2E8997801A
:106D60000100E780E03293140501C1809309D0034C
:106D70008307040099E301450DA0CA852285970089
:106D80000000E78040F70DC1B30794008387070038
:106D9000639C3701138514002295F2406244D2446B
:106DA0004249B249056182800504D9B797F7FF1FB0
:106DB000A38007BE97F7FF1F238C07D297F7FF1F0B
:106DC000238807BC97F7FF1F239E07B097F7FF1F85
:106DD000238B07B097F7FF1F23A807B097F7FF1F74
:106DE000239607BA97F7FF1F239307BA82800111F2
:106DF00006CE22CC26CA4AC84EC697200000E7809D
:106E000060DD3DCD17F4FF1F130464B897F4FF1F36
:106E10009384C4AD17F5FF1F035565B797F5FF1FA2
:106E200083D5C5B66365B50897000000E780C0D478
:106E300025E997F4FF1F9384E4B5130940078D49B2
:106E400097F6FF1F83C6C6B4A1CE17F7FF1F0347EF
:106E500037B4B30727033384F40003552400835564
:106E600004006367B506050733773703FD1697F708
:106E7000FF1F238FD7B097F7FF1FA38BE7B0C9B7CA
:106E800097F7FF1F238107A697F7FF1F23AE07A4DD
:106E900097F7FF1F239C07AE97F7FF1F239907AEB5
:106EA000F2406244D2444249B24905618280898DF0
:106EB000C205C181269597200000E78080D26DD160
:106EC000835704003E9597F7FF1F2392A7AC99B70D
:106ED000898D91073E95C205C181269597200000B6
:106EE000E78020D055DD835724003E952311A40070
:106EF00081BF6309054663870546717156CBC16A38
:106F000026D34AD14ECF52CD5AC95EC762C506D7E5
:106F100022D566C36AC12E8AAA890149B54B17FBDF
:106F2000FF1F130B2B97F91A97D4FF1F9384443438
:106F300017BC0100130C8CAF93170901C18363E0E8
:106F40004703BA502A549A540A59FA496A4ADA4A03
:106F50004A4BBA4B2A4C9A4C0A4D4D618280B387FA
:106F600029010387070097F7FF1F83D7A7976305BA
:106F70007701A9466315D738D5CFDA9717F5FF1FE4
:106F8000130545912380070097000000E78040BD6E
:106F900097B501009385459B2A8497000000E78000
:106FA00080D549C51305640097000000E78040BB09
:106FB0002A8497000000E78000B797B50100938509
:106FC0002599228597000000E780E0D215CD830740
:106FD000240013F7F7FD01C725476397E70213085D
:106FE00050038147114797B601009386A69617B6BE
:106FF00001001306E696930500080A8597800100B4
:10700000E780E0F90A8539A897B501009385C5970F
:10701000228597000000E78000CE19CD17B501004A
:107020001305059797000000E78060B897F7FF1FEA
:10703000239A078A050909B797B501009385059A30
:10704000228597000000E78000CB79C583073400D4
:10705000130700026385E7002547639FE70A1305CE
:10706000340097000000E780A0AF97B5010093853A
:1070700025972A8497000000E780E0C70DC1930799
:1070800050030147914617B601001306A6959305D4
:1070900000080A8597800100E78060F0A5B797B5E2
:1070A00001009385A595228597000000E780A0C484
:1070B0000DC517E7FF1F0347676D97E6FF1F83D6D0
:1070C000467D17B601001306E693930500080A856E
:1070D00097800100E780A0EC35B797B50100938554
:1070E000A594228597000000E780E0C00DC181478C
:1070F0004147B386970083C6060063900622850742
:10710000E399E7FE17B50100130585A721BF17B561
:1071100001001305259239B797B501009385859332
:10712000228597000000E78000BD6305051C8307EA
:107130003400130700026385E7002547639CE71AC4
:107140001305340097000000E78080A197B5010087
:10715000938585902A8497000000E780C0B92DC1EF
:107160009305D003228597800100E780A0EF11C925
:10717000830615000547938706FD93F7F70F63779E
:10718000F70017B501001305A58D69BD930710031E
:10719000639FF60097E7FF1F2387E77497000000BF
:1071A000E780609817B501001305058EA5BD97E728
:1071B000FF1F238A077297E7FF1F23A70772DDB718
:1071C00097B5010093854586228597000000E780EA
:1071D00080B229C19305D003228597800100E78002
:1071E00060E811E517B501001305858B25BD8A857B
:1071F000050597000000E78000A96DD5B7E70400FA
:10720000FC47268541468A85829717B501001305FC
:10721000658B09BD97A501009385457E2285970062
:107220000000E78040AD71C197B501009385C58A24
:10723000228597000000E780A0B12A8D97A5010064
:107240009385857E228597000000E78060B0AA8C38
:1072500063080D046A8502C097000000E780409033
:1072600001468A852A8D97800100E78020FA8247AF
:107270002A846307FD029307F5FF63E3FA0263962E
:107280000C0281474147B386970083C60600A9E2F6
:107290008507E39AE7FE17B501001305259059B35A
:1072A00017B501001305C583B5BB8A8566859700B0
:1072B0000000E780409D11E517B5010013058584A6
:1072C00095B3B7E70400FC4741468A852685829737
:1072D000131504014181A68597D0FFFFE780207533
:1072E00017B501001305458435BB17B5010013051B
:1072F00025850DBB17B501001305858625B393863B
:1073000017001306F004E363D6D2DA9717E6FF1FDF
:10731000231AD65C2380E70031BB97B50100938523
:1073200025870A8597800100E78060D5814C13048A
:10733000B100414DB387940103C607002285E28561
:10734000850C97800100E78000CD0904E394ACFF31
:1073500097A50100938585DF228597800100E7804E
:1073600000D24DB18280F5C1854763F0C70E83C757
:10737000150003C70500A207D98F13978700A183C3
:10738000D98FC2073167C1831307C755639FE70AC7
:1073900097E7FF1F83D7E74F6389A70A011122CC24
:1073A00006CE32C62E842AC497F0FFFFE780C07C49
:1073B00035ED324693070007A24563EDC70617E790
:1073C000FF1F0347E75C894763E6E70697E7FF1F70
:1073D00083C7077213074007B387E70217E5FF1F4C
:1073E0001305455BA2853307F5002310C700231161
:1073F000070037E70400784791073E95029797E723
:10740000FF1F83C7E76E0D478507B3F7E70217E74E
:10741000FF1F230FF76C97E7FF1F9387675783C7FB
:107420000700850717E7FF1F2304F756F240624461
:10743000056182806244F24017A50100130545787A
:107440000561178301006700639C8280011106CEED
:1074500022CC26CA01C5D54763EFB70017A50100A6
:107460001305057897800100E78020B2F24062445E
:10747000D24405618280034705009307500A2A849D
:107480006318F700034715009307A0056307F7008B
:1074900017A5010013054576F1B70347350093079B
:1074A000100A630EF70059476386E500034745005D
:1074B0006305F70217A501001305457565B7D144AB
:1074C0009147D1465D476393D400594763FAE5007D
:1074D00017A501001305057571B7D5449547D5B7B4
:1074E00037E704007847B305F4000A854146029760
:1074F000269483471400034504008A85A2075D8D06
:1075000097D0FFFFE780A05295B741110D658D45DB
:1075100006C697C0FFFFE780C08CB71700408D6696
:1075200023A6D70A17E5FF1F1305C55C1387C70AF3
:107530009387870A1CC15CC5856689675CC958C189
:1075400014C518C9B7E70400B24003A3871E410160
:10755000028397E7FF1F83C7675B99EF411106C658
:1075600097100000E780E05EB240854717E7FF1FF5
:10757000230EF758410182808280411126C2AE84D9
:107580008D4522C406C62A8497C0FFFFE780C08FBE
:10759000B717004099C803A5C70C418D23A6A70CB7
:1075A000B240224492444101828003A5870C418D60
:1075B00023A4A70CF5B78347050003471500A207CE
:1075C000D98FC2076177C18713072720639AE70025
:1075D000834525003705040017030000670023FAE0
:1075E000828017E6FF1F1306A6528147B286130357
:1075F000F00FA9483308F6000348080013F7F70F07
:107600006307A80C630668008507E39517FF294701
:10761000B387E6002380A70097E7FF1F93870750F3
:107620005DA8411113D765001347170006C693F6EE
:107630003500058B954791CA054699476387C60073
:1076400009469D476383C600A14713F645003336BC
:10765000C00093F68503050685C2A145638BB60479
:10766000E145638AB604930580026388B6049305F6
:1076700080036393B600914697E5FF1F2385F5705D
:1076800097E5FF1F2380C57097E5FF1FA38CD56E7C
:10769000BE8517A501001305E55C97700100E78022
:1076A000E076B240854717E7FF1FA30EF76C410154
:1076B00082808546D1B78946C1B78D4675BF17A56B
:1076C00001001305A55C177301006700237417E719
:1076D000FF1F1307A744BA972380B700E147E302CF
:1076E000F5F493077002E30CF5FC82802A8723806F
:1076F0000500814717E5FF1F130585411308F00FAB
:107700002946B306F50083C606006396E60297E6AF
:10771000FF1F9386A640B69783C7070005452380C1
:10772000F5009947636EF7029D4763FDE700E14767
:10773000630DF7008280638506018507E393C7FC2C
:107740000145C5B7238005008280B737004003C7D5
:10775000370083C7050093F70704D98F2380F5000E
:1077600082805D7152DC56DA5ED6716A97EBFF1F3C
:10777000938B8B728D6AA6C24EDE62D486C6A2C47B
:10778000CAC05AD866D26AD06ECEC1495E8C97E420
:10779000FF1F93846439130A0A20938A7ADC17E95D
:1077A000FF1F03496972B3872B0183C7070093F753
:1077B000F70FC9EFB787004003C76700058BE310D9
:1077C000077C03C76700118BE30D077E83C7570053
:1077D000918B99E36F10200317E7FF1F0347E76EB4
:1077E00085476304F7006F10400197E7FF1FA38CE4
:1077F000E75897E7FF1F2389073E97E7FF1F238777
:10780000074A97E7FF1F2385075697E7FF1F238245
:10781000075697E7FF1FA389073C97E7FF1FA3873A
:10782000074897E7FF1FA385075497E7FF1FA38229
:10783000075497E7FF1FA389075497E7FF1FA38605
:107840000768B787004011476F00707793071900EA
:1078500093F7F70F3D476364F70617E7FF1F23050C
:10786000F76697E7FF1F93872765CA9783C70700C7
:107870001307100293F7F703638EE71E6366F7049E
:1078800005446385871CE38C07620947638EE71014
:1078900013070002E384E74EB7E700E03707400034
:1078A00023A0E71801000100629923000900FD19D7
:1078B00023A0E71093F9F90FE39309EEE5BD97E7ED
:1078C000FF1F2383076071BF130730026388E70C33
:1078D00063E8E71613074002638CE70A1307000307
:1078E000E39CE7FA97E7FF1F9387075CCA9703C7F4
:1078F0000700A1471377F70FE31BF71483C7640052
:1079000097E6FF1F2388F64697E7FF1F83C73722B6
:1079100091C7FD5797E6FF1F238EF64497E5FF1F9B
:1079200083C5952097E7FF1FA386B74497E7FF1FFE
:1079300083C7871F13FB07089306000493F7070606
:10794000639FD74C9307A009638DF51663EAB712BE
:107950009307F0056386F54A930750096384F52A77
:10796000014497E7FF1F83C7F7401547E392E736C7
:10797000B7E700E03707400023A0E7180100010047
:10798000B786004023808602130680FC6F00500EED
:10799000FD5717E7FF1F230EF73CFDBDFD5717E707
:1079A000FF1F2307F73CCDBD17A501001305853F39
:1079B00097700100E780605D97E7FF1F9387C74ED0
:1079C000CA9703C40700014B97ECFF1F938C4C2E02
:1079D0001374F40F17AD0100130D4D3D63478B0475
:1079E000294597700100E7804047854717E7FF1F4B
:1079F000A30EF72A17E7FF1F230B872A17E7FF1F9E
:107A00002304F73837E700E0B70640002320D718F3
:107A100001000100378600408347A60293F7370F25
:107A20002305F6022320D71085BDB3876C0183C5DB
:107A300007006A85050B97700100E780203D79BF3C
:107A4000854717E7FF1F2303F726B9B517E7FF1F81
:107A5000130787454A970347070097E6FF1FA3854B
:107A6000F61897E6FF1F2382E61817E7FF1F230D7E
:107A7000F7301DB5854717E7FF1F2307F71629BD08
:107A80009307400A6389F5349307200B6384F53626
:107A90009307100AE396F5EC838724000144E3D2B0
:107AA00007EC97E7FF1F83C7570893F63700638AF1
:107AB000061A0546638AC62209466395C61A1D47FB
:107AC00055A217E5FF1F03454506C94797ECFF1F61
:107AD00083CCBC0597E5FF1F83C5450517E4FF1F51
:107AE0000344D4046315F510CD476392FC1093074B
:107AF0007008639CF5021307300FB7170E00630878
:107B0000E4001307900DB7B704006314E40817E707
:107B1000FF1F2327F726BE8517A50100130585291A
:107B200097700100E780802E25BD93078008639D34
:107B3000F500B307804013F4F70FB777460093873B
:107B400087CDB3D78702E1B793079008639AF50012
:107B5000B307804013F4F70F91679387C766D5B7D3
:107B60009307A008639BF500B307804013F4F70F59
:107B7000B7173D0093870790E9B79307B008639A5A
:107B8000F500B307804013F4F70F9167938797D000
:107B90004DBF93F5F5078D47639BF500B307804014
:107BA00013F4F70FB7975B00938707D859BF89473E
:107BB000639BF500B307804013F4F70FB7770B0012
:107BC0009387071BBDBF8547639AF500B3078040C5
:107BD00013F4F70FDD67938767E3A5B7D28785F9BD
:107BE000B307804093F7F70FB3D7FA020DB79700AA
:107BF0000000E780409FA285668597000000E7802F
:107C0000809EB9BB9305610017E5FF1F0345E5F1B1
:107C100017E4FF1F034474F197000000E78040ADB4
:107C200093057100228597000000E78060AC3C005E
:107C300017E7FF1F2320F726834761002304F10085
:107C400083477100A304F100894717E7FF1F23034F
:107C5000F7128357810017E7FF1F2317F7EC09443A
:107C600009B3154793F64700B336D00093F787035F
:107C7000850685C32146638BC7066146638AC706AE
:107C8000130680026388C706130680036393C70048
:107C9000914717E6FF1F2307D60E97E6FF1FA38322
:107CA000F60E97E7FF1F2380E70E17E7FF1F034736
:107CB000E7E79376070497E7FF1F83C737E78DEE63
:107CC0001377770C93067008630CD7021377F707C6
:107CD0008D466312D70CB307F040B7955B0093F75E
:107CE000F70F938505D849A81947ADBF854755B704
:107CF000894745B78D4771BF930670086311D70256
:107D00001307300FB7150E006389E7021307900DB4
:107D1000B7B504006383E7021307700845BF9306F5
:107D2000800C6311D702B307F040B775460013F714
:107D3000F70F938785CDB3D5E70297E7FF1F23A100
:107D4000B704D9BB9306900C631CD700B307F0406F
:107D500093F5F70F91679387C766B3D5B702F1BF65
:107D60009306A00C631DD700B307F040B7153D0084
:107D700093F7F70F93850590B3D5F5027DBF930672
:107D8000B00CE315D7F4B307F04093F5F70F916704
:107D9000938797D0D9B78946631BD700B307F040C4
:107DA000B7750B0093F7F70F9385051BF1B7854661
:107DB000631AD700B307F040DD6593F7F70F93859B
:107DC00065E35DBFD28535FBB305F04093F5F50F54
:107DD000B3D5BA029DB783C72400C18B99C7854725
:107DE00017E7FF1F230BF7F8A5BE97E7FF1F2386B2
:107DF00007F8BDB6854717E7FF1FA306F7F88DB64E
:107E00003C0017E7FF1F2327F708094793070003E4
:107E10002314F10097E6FF1F238EE6F42DBD639433
:107E20000756A94763E5B74217A701001307C7E044
:107E30008A05BA959C41BA97828717E4FF1F0344CD
:107E4000D4CE894C6306940D63E68C0685476303A4
:107E5000F4089307F00F17E7FF1F0347A7F163F636
:107E6000E70017E7FF1F2307F7F097ECFF1F83CC0E
:107E70006CF09307000413F4FC0F63F497011304F0
:107E8000000497E7FF1F9387E70003AD07002286F2
:107E90002685EA85B38C8C40229D97700100E7808F
:107EA00080EB97E7FF1F238797ED97E7FF1F23A33B
:107EB000A7FF45BC8D47630CF40A9947E31BF4F810
:107EC00097A701009387C7DD17E7FF1F2324F7FC5F
:107ED000A94751B717E7FF1F034727FF97E7FF1F82
:107EE000938747EB494697A50100938565E46306B0
:107EF000870097A501009385A5DF3E859770010057
:107F0000E78060E517E7FF1F2326A7F8C947A1B759
:107F100097E6FF1F83C666FB054797E7FF1F93871A
:107F200067E76394E6023E851306700297A5010099
:107F3000938585DD97700100E780E0E117E7FF1F7B
:107F4000232AA7F49307700239B73E85130630043D
:107F500097A50100938585D597700100E780A0DF84
:107F600017E7FF1F2328A7F293073004EDB597E525
:107F7000FF1F83C585BB17A501001305E5E49770B6
:107F80000100E780A0E8054D97EDFF1F83CDEDF3DD
:107F900097E5FF1F83C565B917A501001305C5E265
:107FA0006398AD0B97700100E78040E697E7FF1FED
:107FB00083C7A7B7B5CBE36EF4E817A40100130499
:107FC00064DB638CB70117A40100130424DB638610
:107FD000970117A401001304E4DB228597700100C8
:107FE000E780000B1375F50F93071500860717E759
:107FF000FF1F2301F7DA8D4717E7FF1FA30CF7D800
:1080000097E7FF1F938707D90147BE861376F70FBF
:1080100089076365A60297E7FF1F23ADD7E697E7B9
:10802000FF1F83C727D705BD97A70100938787CD7B
:1080300017E7FF1F2320F7E6914731BD3306E40021
:1080400003460600A380070005072380C7007DBF05
:1080500097700100E78080DB97E7FF1F83C7E7ACDD
:10806000E1D7E368F4DE17A401001304A4CD638C08
:10807000A70117A40100130464CD6386970117A418
:108080000100130424CE228597700100E780400090
:108090001375F50F93071500860717E7FF1F230BCE
:1080A000F7CE8D4717E7FF1FA306F7CE97E7FF1F11
:1080B000938747CE0147BE861376F70F8907E37C87
:1080C000A6F43306E40003460600A3800700050774
:1080D0002380C700D5B797E5FF1F83C505A517A562
:1080E0000100130525CF97700100E78020D297E7A4
:1080F000FF1F83C7F7C993E7470017E7FF1FA309CF
:10810000F7C883C7240017E7FF1FA301F7C889B882
:1081100017A50100130545CD97700100E780E0E643
:1081200097E7FF1F938787C683C7070017E7FF1FDF
:10813000230CF79E17E4FF1F0344C4C333348000AD
:108140000DB017A50100130565CB97700100E780FE
:10815000C0E397E7FF1F83C7B7C393E7070117E79C
:10816000FF1FA307F7C283C7240017E7FF1F230FD2
:10817000F7C06FF0EFFE17A50100130565C99770F2
:108180000100E78080E003C704007D8B51EFB787D3
:10819000004003C767021377C70B136727002383C9
:1081A000E70203C7A7021377C70B136727002385CE
:1081B000E70203C7E7021377C70B1367270023877C
:1081C000E70203C727031377C70B13672700238929
:1081D000E702854717E7FF1F2308F7A017E7FF1FF0
:1081E0002306F7AC17E7FF1F2304F7B817E7FF1FB5
:1081F0002301F7B897E7FF1FA388079E97E7FF1FA4
:10820000A38607AA97E7FF1FA38407B697E7FF1F78
:10821000A38107B697E7FF1FA38807B697E7FF1F5D
:10822000A38507CA6FF0CFF389476312F70297E778
:10823000FF1F83C7A78F9146638CD70863E0F604BE
:10824000638EE70C6369F70A05476380E70EFD5705
:1082500017E7FF1FA300F7B237074000B7E700E0BA
:1082600023A0E71801000100B78600401306F0FCC8
:108270002381C60223A0E7106FF00FE21307200846
:108280006382E7086362F70213071008E391E7FCD3
:10829000378700408347670293F7C70B93E72700B0
:1082A0002303F7026FF0CFEB130730086389E7026F
:1082B00013074008E39DE7F837870040834727030B
:1082C00093F7C70B93E727002309F7026FF04FE9F5
:1082D000378700408347270393F73707F5B737877A
:1082E00000408347E70293F7C70B93E72700230774
:1082F000F7026FF0EFE6378700408347E70293F716
:108300003707F5B7378700408347A70293F7C70BB6
:1083100093E727002305F7026FF08FE437870040CB
:108320008347A70293F73707F5B73787004083479E
:10833000670293F73707ADB717A50100130545AEE0
:1083400097700100E78060C497D7FF1F238E077CDA
:10835000D5B317A501001305A5AD97700100E780FF
:10836000C0C297D7FF1F2391077C97E7FF1F938712
:1083700067A003C40700894763F3870009441374A7
:10838000F40F6FF00FDE13070002E392E7EC631BBC
:108390000B0A638FF500930720026383F50817A586
:1083A0000100130565AC97700100E78020A645B574
:1083B00017A50100130585A897700100E780E0BCB0
:1083C000014417AD0100130DADA8A14CB387840083
:1083D00083C507006A85050497700100E78000A344
:1083E000E31694FF17950100130545DC9770010013
:1083F000E780A0B917D4FF1F0344447301E897D75F
:10840000FF1F23860770014B6FF0AFD58947E3103C
:10841000F4E4854717D7FF1F230BF76E6FF04FD497
:1084200017D6FF1F0346767097D5FF1F83C5E56FEC
:1084300017A50100130545A297700100E780009D74
:108440006FF00FD26380F50693071002E399F5F4FD
:1084500097D5FF1F83C5856D17A501001305C5A11D
:1084600097700100E780809A97E7FF1F23A497A2E7
:1084700097E7FF1F9387C790944383D7470017E779
:10848000FF1F0347479017D6FF1F232FD6681D44B1
:1084900097D6FF1F239CF66897D7FF1F2389E768AD
:1084A0006FF02FCC97D5FF1F83C5456817A5010036
:1084B0001305059E97700100E780409597D7FF1F31
:1084C0002387076497D7FF1F239007666FF02FF964
:1084D0002547638FE7C89946378700406394D702E2
:1084E00023008702B7E700E0B706400023A0D718B3
:1084F00001000100130600FC2301C70223A0D710CE
:108500006FF08FB99306100A639FD700230087028C
:10851000B7E700E0B706400023A0D718010001002C
:10852000130680FCD1BF9306A009E381D7FE930612
:10853000400AE38DD7FC93062002639DD700B7E77E
:1085400000E0B706400023A0D71801000100230077
:108550008702F9B78546E384D7FE93070008E30056
:10856000FBFEB7E700E0B706400023A0D7180100E4
:108570000100130620FC23008702BDBF17D7FF1F91
:108580000347577F6302F71E63E7E70295476300DF
:10859000F7109947630AF704B78600402380060264
:1085A000B7E700E03707400023A0E718010001000B
:1085B0001306A0FC75B99307F005630AF70093074B
:1085C00050096306F70093071002E317F7FCB7E7BB
:1085D00000E03707400023A0E71801000100B7863C
:1085E0000040130620FC69B117DBFF1F034B8B789B
:1085F000930700045A8D63F46701130D000497E795
:10860000FF1F9387278983AC07001374FD0F228611
:10861000E685268597600100E780E073B3078B400D
:10862000669417D7FF1F2307F77497E7FF1F23A34D
:108630008786B7870040630C0B022380A703B7E649
:1086400000E03706400023A0C6180100010003C760
:108650002702134707042381E70203C72702137782
:10866000C70F2381E70223A0C6106FF0EFA223807B
:10867000070237E700E0B70640002320D7180100C3
:108680000100130620FC2381C7026FF0AFB93787C2
:1086900000408347370097D6FF1F83C6366F93F796
:1086A0000708D58FA301F700B7064000B7E700E041
:1086B00023A0D718010001001306A0FC35BD97D7F1
:1086C000FF1F9387677ECA9783C7070093F7F70F4B
:1086D000C1CF97D7FF1F83C7477FD9E717D7FF1FA2
:1086E00003475769930700026310F70883AD04003E
:1086F00017DDFF1F034D8D4397DCFF1F83CC1C4309
:1087000017DBFF1F034BAB42E6876A87DA866E866C
:1087100097D5FF1F83C5A53F179501001305C578A1
:1087200097600100E780806E97D7FF1F23AAB76587
:1087300097D7FF1F2388A76597D7FF1FA384976547
:1087400097D7FF1F2381676597D7FF1FA380873CBB
:10875000B7E700E03707400023A0E7180100010059
:10876000B78600406FF04FA2B7E700E03707400040
:1087700023A0E71801000100B786004015BD97D679
:10878000FF1F83C686740547639CE604294723813F
:10879000E70209472383E7022385E70297D7FF1FF4
:1087A000A384075E97D7FF1FA3810772B787004096
:1087B000A381070017D7FF1FA30A075C0547238380
:1087C000E700B640264496440649F259625AD25A06
:1087D000425BB25B225C925C025DF24D6161828021
:1087E00029472381E70209472383E7022385E7021C
:1087F0002387E7022389E70255B717D7FF1FA3078F
:10880000F7306FE01FFF854717D7FF1F230EF73C98
:1088100017D7FF1F230CF74817D7FF1F230AF7545A
:1088200017D7FF1F2307F7546FE0BFFE854717D701
:10883000FF1F230BF73A17D7FF1F2309F74617D758
:10884000FF1F2307F75217D7FF1F2304F75217D72D
:10885000FF1FA30B073817D7FF1FA309074417D71C
:10886000FF1FA307075097D7FF1FA38407508280DD
:10887000411106C697000000E78080FBB7870040E3
:1088800023800700130740FC2386E7001307C0047A
:10889000A386E70017D7FF1F130707292398E700D0
:1088A00017D7FF1F1307472C239AE70017D7FF1F7F
:1088B0001307C737239CE70017D7FF1F130747434A
:1088C000239EE70029472381E70209472383E70224
:1088D0002385E7022387E7022389E702A3810700B4
:1088E000930600F8A380D700930690022380D70058
:1088F000FD562383D7002381E7009306000537E761
:1089000000E0230BD740B70640002320D71003C751
:10891000170013671700A380E700B24097D7FF1F27
:108920002396074641018280411106C69700000048
:10893000E78000F0B787004023800700130700FCA2
:108940002386E7003147A386E70017D7FF1F1307E9
:10895000A71D2398E70017D7FF1F1307E720239AC7
:10896000E70017D7FF1F1307672C239CE700294751
:108970002381E70209472383E7022385E702A381D6
:108980000700930600F8A380D70093069002238087
:10899000D700FD562383D7002381E7009306000507
:1089A00037E700E0230BD740B70640002320D7105D
:1089B00003C7170013671700A380E700B24097D7DB
:1089C000FF1F2395073C41018280F16793870720B1
:1089D00017D7FF1F2326F73A854717D7FF1F231303
:1089E000F73AA14717D7FF1F230FF73897D7FF1F75
:1089F000A38B073897D7FF1F2388073897D7FF1F08
:108A00002387071097D7FF1FA3820710814717D529
:108A1000FF1F1305E50FFD5517D6FF1F13060610A0
:108A20002947B306F5002380B600B306F60023807D
:108A300006008507E397E7FE97D7FF1FA38D073250
:108A400097D7FF1FA38B073297D7FF1F23860732C5
:108A500097D7FF1F2381073297D7FF1F2380073245
:108A600097D7FF1FA38A073097D7FF1F23870730A9
:108A7000814717D6FF1F130626424147B306F6006B
:108A8000238006008507E39BE7FE828017D7FF1F40
:108A90000347A74385476316F700170300006700E5
:108AA000E3E8170300006700E3DC411122C406C6B7
:108AB00017D7FF1F0347674185472E8613F4F50F2D
:108AC000AA856317F70417D5FF1F1305251A9760AA
:108AD0000100E780402897D7FF1F2389071CB7872D
:108AE000004023848702B7E600E03706400023A059
:108AF000C6180100010003C7A7021377C70F23851B
:108B0000E702B240224423A0C61001454101828001
:108B100017D5FF1F1305450997600100E780A023C3
:108B200097D7FF1F2382070CB78700402382870255
:108B3000B7E600E03706400023A0C6180100010098
:108B400003C767021377C70F2383E7025DBF411195
:108B500006C697000000E78080E7B2404101170396
:108B600000006700E3F2411106C697F0FFFFE780BF
:108B700080BF97D7FF1F83C73707A1CB97D5FF1FAC
:108B800083C5A50689C917D5FF1F1305250697E0DC
:108B9000FFFFE780403697D7FF1FA387070497D7CB
:108BA000FF1F2383071E37E700E0B706400023209E
:108BB000D71801000100378600408347660293F70B
:108BC000370F2303F6022320D710B24041018280E1
:108BD00017D5FF1F0345851B3335A0008280411147
:108BE00006C622C429C12E8495C997D7FF1F83C703
:108BF000E71995CB97D7FF1F83C707FF8DC71307CB
:108C00000004AE876374B700930700041394070150
:108C10004180A28597000000E78060E92285B2408C
:108C20002244410182800144D5BF97D7FF1F93871B
:108C3000672D18429C4383D645000345070083C532
:108C4000C700035646006396A50083D5E700638DF1
:108C5000D502011106CE2386A7002397D700B705BA
:108C6000CF00DC4B9385757D05077D162EC2230052
:108C700001003AC42316C1002317D10099C30A8505
:108C80008297F240056182808280DC4DDC4B81CF8F
:108C9000B7E70400904503A38705914517D5FF1F4B
:108CA00003458526028382806D713C083EC6B70766
:108CB000E500232291103EC8AA843C083285232671
:108CC00011103ECA23248110232021112E899730B0
:108CD0000000E780005E2A84979501009385452077
:108CE00017850100130505E497600100E780001275
:108CF000A285179501001305252F97600100E780D5
:108D0000E010294597600100E7802015B705CB00EA
:108D10009385757D680097100000E7802067A28525
:108D2000680097300000E780204B014781467000C3
:108D3000CA85268597200000E780A08A05CD2A8471
:108D4000979501009385C51917850100130585DDE9
:108D500097600100E780800BA2851795010013053D
:108D6000652997600100E780600A29459760010046
:108D7000E780A00E8320C1100324811083244110BA
:108D8000032901105161828097D7FF1F93878717AE
:108D900018429C43797122D406D60348070083C841
:108DA00007012A8483D645000355460063960801CF
:108DB00083D82701638DD8022388070105072399EB
:108DC000D7003708CC00DC4B1308787D3ACC13076A
:108DD000F5FF42CA23080100231EE100231FD10032
:108DE00099C7080832C62EC482973246A24522850A
:108DF00097000000E78080EBB250225445618280EA
:108E00006D713C083EC0B707E5003EC23C083EC459
:108E100023261110232481102322911023170100EF
:108E20002318010023190100231A0100231B01004C
:108E300097A7FF1F83D7075C99E3C167FD17231628
:108E4000F10097A7FF1F83D7075B91EB97D7FF1F11
:108E50009387470B9C439C43DC4783D7070017A4A9
:108E6000FF1F13042459584C2317F1008357440063
:108E7000484B2318F10031E1979501009385450D8A
:108E800017850100130505CA97600100E78000F807
:108E9000179501001305050D97600100E78000F7A5
:108EA000294597600100E78040FB8320C11003241F
:108EB0008110832441105161828097A7FF1F83C7CF
:108EC000D75389EBB7E70400BC5782975C4C23AAC1
:108ED0000700E1BFFD1797A6FF1FA380F6520356B8
:108EE0000701834704014C470A85230BF1009730A3
:108EF0000000E780802B97D7FF1F9387A7009C4334
:108F00000147814688430A866C0097100000E7807D
:108F1000406DAA8429C19795010093856503178543
:108F20000100130525C097600100E78020EEA685AB
:108F3000179501001305C50397600100E78000ED58
:108F4000294597600100E78040F1584CB7E70400DD
:108F5000BC57484B9DBF97A7FF1F83C7174AF5D73C
:108F6000B7E70400BC4F1044854517D5FF1F0345E4
:108F7000A5F982971DBF5C4EDC4BB9CFB1CD411135
:108F800022C4178501001305E5B92E8497950100C9
:108F9000938545FA06C697600100E78020E7A28521
:108FA00017950100130585FF97600100E78000E633
:108FB000294597600100E78040EAB7E704002244B2
:108FC000B24003A3870517D5FF1F0345E5F313063A
:108FD00040069145410102838280411122C417A4B9
:108FE000FF1F1304E43E1C4C06C689C7DC4399C32B
:108FF0004C488297584CB7E70400BC57484B8297BF
:109000005C4CB240224423AA07004101828017A78A
:10901000FF1F1307E73D834707009306F00B850703
:1090200093F7F70F63E9F60097A6FF1F2382F63C3C
:10903000034507008280930700F8FDB7835745007A
:109040006386071001114AC817A9FF1F1309893A3F
:1090500052C4032AC90106CE22CC03274A0126CADC
:109060004EC656C2F15735E31307D00DFD57636E58
:10907000C704B7E9040083A709072A8413058600FB
:1090800042054181B284AE8A8297232AAA00032531
:10909000C9015C49A9E7979501009385A5E7178564
:1090A0000100130525A897600100E78020D61795D9
:1090B00001001305E5F697600100E78020D52945FA
:1090C00097600100E78060D9DD57F2406244D244E6
:1090D0004249B249224A924A3E850561828093877D
:1090E0004400B705CF002319F5009385757D310540
:1090F00097100000E78080290325C901834564009B
:10910000310597300000E780200D0325C901268630
:10911000D685310597300000E78020097146A28589
:109120004A8597600100E78000C3504419CA83A7AD
:109130008905854517D5FF1F034505DD82978147C2
:1091400069B797000000E780E0CBD5BFFD573E85AB
:109150008280411126C297A4FF1F9384A429D84C72
:1091600022C437E404003C54484B06C68297DC4CCA
:109170000323C4052244B240924423AA070017D512
:10918000FF1F034565D8854541010283411126C271
:1091900097D4FF1F938404D79C4006C622C44AC0BC
:1091A000D5C3DC43C5C35CC12300B5002A849795B1
:1091B0000100938565D1178501001305A596976079
:1091C0000100E780A0C4294597600100E780E0C85E
:1091D0009C4023A4070023A2070097A7FF1F9387A3
:1091E000271FDC4FDC4B91C7295597000000E78013
:1091F00000DF97A7FF1F9387E71FDC4FDC4B89C772
:1092000097000000E78020F537E904008327C905AF
:10921000894517D5FF1F034525CF82978327C905A9
:10922000914517D5FF1F034525CE82979C4003A388
:1092300047016309030022852244B2409244024957
:1092400041010283B240224492440249410182809A
:109250000111328506CE22CC26CA2E84973000001A
:10926000E7802005AA8497950100938525C9178575
:1092700001001305258B97600100E78020B90307E3
:1092800084000356640083554400A68617950100A8
:109290001305C5D297600100E78040B72945976064
:1092A0000100E78080BB97A7FF1F83C7C712639D9C
:1092B0009700014597000000E78060D281450A854C
:1092C00097000000E780C0ECF2406244D2440561A0
:1092D00082806D7123248110232611102322911086
:1092E00093F745002E84638707143C083EC0B707F8
:1092F000E5003EC23C083EC42317010023180100CC
:1093000023190100231A0100231B010097A7FF1F47
:1093100083D7070C99E3C167FD172316F10097A7C0
:10932000FF1F83D7070B91EB97D7FF1F938787BD4D
:109330009C439C43DC4783D7070017A7FF1F1307F5
:1093400027092317F100544F835747002318F100D2
:10935000DC4AA1E797950100938585BE177501004A
:109360001305457C97600100E78040AA179501002E
:10937000130545BF97600100E78040A92945976024
:109380000100E78080AD134544008320C110032411
:109390008110832441105161828097A7FF1F83C7EA
:1093A00097032555D9C3FD1717A6FF1FA305F6027E
:1093B00003D6060183470701CC460A85230BF1003B
:1093C00097300000E78060DE97D7FF1F938787B351
:1093D0009C4317A7FF1F1307A7FF979601009386CB
:1093E00066BB88430A866C0097100000E780601F08
:1093F000AA8451D997950100938585B4177501000A
:109400001305457297600100E78040A0A685179577
:1094100001001305E5B597600100E780209F29450D
:1094200097600100E78060A3268597000000E78031
:1094300000BB91BF93F725009DC7B7E70400BC4769
:109440004146814528088297255597000000E7800E
:1094500000B928089305F00F97000000E78040D37B
:10946000134524001DB793F71500014599DF9700B8
:109470000000E78020991345140001BF5C4D4111A5
:1094800006C688C317D7FF1F232EF7A6B7E7040029
:1094900083A70708170500001305E5E38297B2408C
:1094A00097D7FF1F2382A7A60145410182800111A2
:1094B0003335A000A307A100B7E7040083A747172F
:1094C00006CE1306F1008545130550308297F24011
:1094D000056182808280411122C406C697D7FF1F92
:1094E00083C707A4014489EF97B7FF1F83C7D7E954
:1094F000054499E717C4FF1F03444429134414008B
:10950000228597000000E780C0FA17950100130537
:10951000E5BC09E417950100130545BD2244B2409E
:109520004101176301006700638E797122D4A30F94
:10953000010037E404008327841726D24AD006D6D8
:10954000AA842E89130550309305F10132C6829703
:1095500032468347F10193150601C18185CB014550
:109560002EC697000000E780C0F483274417B24559
:109570004A8626858297054597000000E78060F3BC
:10958000B250225492540259456182808327441775
:109590004A8626858297EDB741119397050122C42B
:1095A00006C626C2C1872E8463D40702B7E404002E
:1095B000FC5417A5FF1F0345E5E6829719C1BC546B
:1095C00082972165218DB2402244924441018280DC
:1095D00093F715008DC7B7E7040083A7471A17A6AE
:1095E000FF1F130626E397D5FF1F9385A59217A5A6
:1095F000FF1F034525E3829713451400E9B793F74E
:10960000250099CFB7E70400BC4F130600648945D5
:1096100017A5FF1F034505E182971345240065B791
:1096200093F7850085CF97D7FF1F83C7279085E7DE
:10963000B7E7040003A8871A1307401F97A7FF1F67
:1096400083C747DE814613064006994517D5FF1F9D
:109650000355458D029813458400B5B793F745002F
:109660000145B5D3B7E4040083A7041817D5FF1F3D
:109670000355458B8297BC4C13060064914517A592
:10968000FF1F034525DA8297134544002DBF97D766
:10969000FF1F83D727896398A70217D7FF1F2314BB
:1096A000B78817D7FF1F2311C78817D7FF1F231E9F
:1096B000D7862E8617950100130585A8BE851753FA
:1096C00001006700A374179501001305E5A817634F
:1096D00001006700838B0357450097D7FF1F83D78F
:1096E0006784631EF704C1674111F91722C417D7B5
:1096F000FF1F2329F78237E4040097D7FF1F23A514
:10970000078297D7FF1FA38D078097D7FF1F238F4F
:1097100007807C4C06C6894517A5FF1F034585D0E9
:1097200082977C4C914517A5FF1F0345A5CF8297D3
:109730002244B240410117030000670003DA179585
:109740000100130565A117630100670003847D15FF
:10975000954763E2A71C179701001307E7950A05D1
:109760003A951C41011122CC06CEBA972E848287ED
:10977000179501001305C59E97600100E780E08002
:10978000A1A203C7250099476311F7022E85970010
:109790000000E78080F483456400179501001305FD
:1097A000259D97500100E780606697B7FF1F238DC6
:1097B00007BC179501001305659D7DBF03C72500F4
:1097C00095476319F702C16717C7FF1F03578775CE
:1097D000F91703D5A5006309F702B7E7040083A7CB
:1097E000C7178297179501001305459B97500100F5
:1097F000E780A079854717B7FF1F2307F7B81795AC
:1098000001001305259C8DBF97C7FF1F239CA770E0
:1098100083D7E50097C6FF1F2397F67083D705010E
:1098200097C6FF1F2392F67083D7250197C6FF1FA7
:10983000239DF66E97C7FF1FA384076E631BE50287
:10984000B7E70400BC4F096613060690A14517A5AB
:10985000FF1F034525BD82970356E4008355A400EE
:10986000179501001305C59497500100E780005A31
:1098700051B79307700F2316F100B7E7040083A7D1
:10988000870D17A6FF1F0346E6B96C0082974DF9B6
:10989000854717C7FF1FA305F7685DB71795010038
:1098A00013050593D1BD83C5250091476392F50249
:1098B000179501001305459397500100E780E06C70
:1098C00097000000E78060C1F24062440561828039
:1098D00099476392F502228597000000E780E0DF58
:1098E0008345640017950100130585889750010092
:1098F000E780C051D1BF9547639AF50083471400B4
:10990000E1F31795010013056590BDB517950100AA
:1099100013054590E1BF8280411122C417A4FF1FA7
:10992000130484B1AA86178601001306667A22857D
:10993000C14506C697500100E780606603574400A2
:1099400097A7FF1F938747B02393E700035764004F
:109950002394E700B240224441018280411106C6AF
:1099600097000000E78080FBB7E7040083A7871417
:1099700017A6FF1F130646ACD54501458297B24096
:109980004D4697A5FF1F938525AC13057030410107
:10999000170300006700A3B961712324811A37E41B
:1099A0000400832704082326111A2322911A232056
:1099B000211B232E311917050000130525BE8297A0
:1099C00017A9FF1F130909A6994785442300A90079
:1099D000231CF1009785010093858573930740064A
:1099E0001775010013050514231CF10823089100C5
:1099F00097C9FF1F9389E9E997500100E78000416B
:109A000083D50900178501001305856F9750010064
:109A1000E780C03F294597500100E780004403D507
:109A20000900896997000000E78040EF8327441709
:109A3000100885451305503082978327441717A6D1
:109A4000FF1F130666A0CD4513057030829783274C
:109A5000441717A6FF1F1306269DB5451305603052
:109A60008297832744173008894513051031829760
:109A700083274417300989451305203182978327AE
:109A80004415938509900D45829783274415938546
:109A9000099011458297A3059100230691002308A0
:109AA000910002CD230C01008327841630099145D3
:109AB000130570408297832784161306B1008545ED
:109AC000130500408297832784167000854513058F
:109AD000104082978327841630088545130520405F
:109AE0008297832784161008854513055040829776
:109AF000832704157D558297832744137D558297CC
:109B00007D5597A0FFFFE78020B68327440C8297FE
:109B100097A0FFFFE78080918327841417A6FF1F7B
:109B200013068691D5450145829789471306700F24
:109B3000814528092306F1009780FFFFE780A05C9C
:109B40008D471306000881452808230CF1089780EB
:109B5000FFFFE780405B9147230CF10097770100FE
:109B60009387C7ED984383C747003AC8230AF1009B
:109B700097D0FFFFE780209070008545054597A0AE
:109B8000FFFFE78080B530099305700F094597A066
:109B9000FFFFE78080B43008930500080D4597A0CB
:109BA000FFFFE78080B310089545114597A0FFFFA0
:109BB000E780A0B2C16717C7FF1F1307A736F917C1
:109BC0001CC32322070017A5FF1F1305658597A057
:109BD000FFFFE78060AF8327C41D17C5FF1F130574
:109BE000E53282973C4803450900854582978320EA
:109BF000C11A0324811A8324411A0329011A8329D3
:109C0000C1195D618280C16717C8FF1F0358883181
:109C1000F9176301F8083DCDB5CD011126CAB7E4A7
:109C2000040083A7841222CC2E862315B10006CE11
:109C30002A8401478146ED45428582972AC611ED67
:109C4000178501001305C54D97500100E780E033EB
:109C5000F2406244D24405618280FC440356A10074
:109C6000A28582972C0017C5FF1F0355A52B97A02F
:109C7000FFFFE78020B269DD178501001305854BE2
:109C800097500100E780603083A7C412ED4528009B
:109C900082977DBF8280411106C61DC985471797EF
:109CA000FF1FA308F77835469795FF1F9385C57763
:109CB000130560309797FF1F238E077697000000EB
:109CC000E780E086B2404101170300006700E380AF
:109CD0009797FF1FA38F0774F9B797C7FF1F83C715
:109CE000E724A9EFC16717C7FF1F0357A723F91779
:109CF0006306F7044111854722C417C7FF1F2307D6
:109D0000F72237E404007C4C06C6A1451795FF1FD7
:109D10000345457182970323841A2244B2409797E2
:109D2000FF1F83C7277017C5FF1F0355A51F130704
:109D3000401F8146314699454101028382806D7101
:109D4000232481102326111023229110328401CD67
:109D50008947630AF5028320C110032481108324FC
:109D6000411051618280178501001305654BAE8457
:109D700097500100E7806021A285268597C0FFFFEC
:109D8000E780208DC9BFB7E70400FC472800829711
:109D9000178501001305854997500100E780E01EF3
:109DA0008347810039C41307000B6380E7021387E0
:109DB000A7051377F70F8D4663EDE602A28528000D
:109DC00097C0FFFFE78000FC79B78547E3F587F888
:109DD00083459100177501001305C50BB335B0001D
:109DE00097A7FF1F2382B74297500100E780000228
:109DF0009DB703479100A207D98F35671307D75541
:109E00006385E7086368F7022D671307B755638713
:109E1000E70631671307C755638AE7042967130705
:109E2000A7556394E702A285280097C0FFFFE7804B
:109E3000603515B739679306E7656381D70863E92D
:109E4000F6001307E7556384E706A28528003DB7AF
:109E50003D679306F755638AD7061307F766E396BF
:109E6000E7FE97C0FFFFE780A04FF5B50146A2854A
:109E7000280097C0FFFFE780E01BF1BDA285280006
:109E800097C0FFFFE780002CF9B58947E3F587EC21
:109E900097000000E780A0E49305E4FFC205C181BC
:109EA0001305A1009790FFFFE78060316DB5A28593
:109EB000280097C0FFFFE780A02F71BDA285280072
:109EC00097C0FFFFE780603A79B597C0FFFFE78052
:109ED000E04251B5C16717C5FF1F0355A504F91727
:109EE0006307F500B7E7040003A3C7170283828066
:109EF000854717C7FF1F2305F702014517F3FFFF2B
:109F00006700235B1783FFFFE702431B2A84084592
:109F10002E89B28919C900C1971500009385A586BD
:109F2000610597300100E780800181447D5A9710D8
:109F30000000E780E03963C7A40481449710000063
:109F4000E780003A63C8A40497C7FF1F938747FEC2
:109F50009C43DC47B307F94091872302F4006383F5
:109F600009048327C900B307F4409587A302F400CE
:109F70001C4C89C79C4799C3228582971783FFFF92
:109F8000670003175C44139714008504BA97239065
:109F9000470171BF1C48139714008504BA9723909A
:109FA000070069BF832789000547B307F4409587F9
:109FB000A302F40083570400638EE7028DC30947B0
:109FC0006384E7040D47E395E7FA978701009387D9
:109FD000A7781CCC978701009387077911A89787EA
:109FE00001009387E73E1CCC978701009387473F8A
:109FF0005CC8BDBF978701009387872A1CCC9787D1
:10A0000001009387E72AEDB7978701009387877947
:10A010001CCC978701009387E779D9BF95E5178313
:10A02000FFFFE702430B0046184483479400758303
:10A030009D8B6317F70097100000E78060B448C459
:10A040001783FFFF6700630B82801783FFFFE70220
:10A05000E30613893500C16442094111AA8901440C
:10A06000F11413590901054A2EC697100000E78024
:10A070002026B2456348A400014541011783FFFF34
:10A080006700030783A7090013171400BA9783D743
:10A0900007006388B7006394970063742A0105047E
:10A0A000E1B70545D9BF1783FFFFE7024300AA893F
:10A0B0002E89328BB6843A8ABE8A97A00000E78048
:10A0C00020FB71C9268597200000E78020098D4775
:10A0D00063E7A7007D551783FFFF6700C30083DB9D
:10A0E000440097100000E780A0242A849710000005
:10A0F000E78040259307740031443305850263CD22
:10A10000A70297100000E780A02297100000E780C8
:10A1100020222A8497100000E780C0229307740051
:10A1200031443305850263C3A70497100000E7801C
:10A1300020209307450029A897100000E780802081
:10A14000330585021307F0179307C017E35FA7FADB
:10A150002D55E3C277F963040B02D6865286A68595
:10A160004A8597200100E78020BAB5B79710000014
:10A17000E780401D330585029307C5FFD1BF8327C4
:10A1800049001385C90083D5270097000000E780A8
:10A1900000EC61F581B769553DBF97C7FF1F239B51
:10A1A000A7D897C7FF1F9387A7D8904381470C462E
:10A1B0003307F500420741836393B700828054461A
:10A1C000139847008507C2962390E600D5B797C736
:10A1D000FF1F9387E7D59C4303C58700828017C57F
:10A1E000FF1F035525D582801783FFFFE702A3EEEB
:10A1F000C1671387D7FF630BE502636AA700F117F6
:10A200006300F50201451783FFFF670003EF138723
:10A21000E7FF6302E502FD171D8D13351500E5B755
:10A2200097500000E780C0267D15C5BF97500000FD
:10A23000E78040FBD5BF97500000E78060F9EDB79D
:10A240001783FFFFE70223E94111AA8401442EC6C8
:10A2500097100000E780C008B2456348A40001459C
:10A2600041011783FFFF670043E99C481315140061
:10A270003E9583570500E385B7FE0504C9BF034833
:10A280005500814693F7F60F63E5070181473E8548
:10A290008280584593975600BA9703D727006316D4
:10A2A000B70003D70700E304C7FE8506E1BF834676
:10A2B000450001479377F70F63E4D700814711A862
:10A2C0001C45131657000507B29703D60700E31382
:10A2D000B6FE3E8582801783FFFFE70223DE9317D9
:10A2E0000501C18797CAFF1F938A8AC4635BF00880
:10A2F00083A70A00C0479C4703570400198D4205F5
:10A3000041816368F500014422851783FFFF6700E0
:10A3100023DE12052A94CDBFDC4713944900014A7D
:10A320003E94834744006341FA02014A8347540044
:10A330006349FA028509C20993D9090183A70A0072
:10A340009847E3EBE9FCC1B71C4413195A00A685F2
:10A350003E994A8597000000E780C0EE05E1050AB6
:10A36000C9B75C4413195A00A6853E994A859700DF
:10A370000000E78020ED19E1050A4DBFE30C09FA62
:10A3800061B7AA8481495DBF1783FFFFE702A3D4A9
:10A390001C452A8481E79307C5001CC51C44231271
:10A3A00004001CC09307F00F63EDB70093F5F50FA1
:10A3B000228597200000E78020E21783FFFF6700D7
:10A3C000C3D393940501C167C18063F9F500A685E5
:10A3D000228597200000E78040E5C5B7C18193F54D
:10A3E000F50F228597200000E78000DFA6852285F3
:10A3F00097200000E78040E0C9B797C7FF1F938709
:10A4000027B3884382801C4599C797C7FF1F23A1A4
:10A41000A7B2014582807D55828097C7FF1F938731
:10A4200027B1984383474500484792073E9582806D
:10A430001783FFFFE70223CA617100451C183EC65F
:10A44000B70780013EC81C183ECA8357440002CE9D
:10A4500002D002CC231EF100834784002A8902D255
:10A460002301F1023C083ED402D697000000E780A9
:10A4700000FB835705002316F10297500000E78088
:10A4800060C42307A1025C4003556400F18313F705
:10A4900017008347F10252055181F99BD98FA30719
:10A4A000F10297100100E780807539CDAA84035529
:10A4B000050097A00000E78080BC83D704002AD263
:10A4C0006800231CF10083D72400231DF1001C48E1
:10A4D00003D647008C4397200000E78000CD8347D8
:10A4E000B400CA8617860100130606D58117A30596
:10A4F000F4006C00481097200100E780E0805D6167
:10A500001783FFFF670063BF2155D5BF1C45B1CF3F
:10A5100003C5A700894613576500630BD7028D4614
:10A52000630ED70285466300D70213074006330542
:10A53000E50203C7B700418B15CB83C7B700BD8BBE
:10A540003355F54082801375F5031307803EC5B778
:10A5500009671375F50313070771D1BF3727090082
:10A560001375F5031307077CD9B70145828017835C
:10A57000FFFFE70243B603A98500630C0904834784
:10A58000B900AE8493F7070E85C303459900930580
:10A5900020030D810505B305B50288446105973098
:10A5A0000100E780E0A935A02E8597000000E78034
:10A5B00020F62A8419CD97000000E780605C83258F
:10A5C000C900B307B54063FA87002E94B305A440D1
:10A5D000E9F51783FFFF670043B285457DBF178309
:10A5E000FFFFE70243AF2A8403D50500011132C6FD
:10A5F00036C43AC22EC002CA02CC02CE97A00000D6
:10A60000E780E0A782452ACA22852ECC9700000069
:10A61000E780E0E003570500231EE10097500000AB
:10A62000E78040AAA24632469247230FA100368710
:10A630004C08B2862285014697000000E780E0A61C
:10A6400005611783FFFF670043AB1783FFFFE70236
:10A6500083A861711C183EC6B70780013EC81C184C
:10A660003ECA3C0800453ED4AA8402CC02CE02D0A9
:10A6700002D202D697000000E78060DA8357050017
:10A6800035592316F10297500000E780A0A3230755
:10A69000A10209C48357440081EB21594A855D61B9
:10A6A0001783FFFF670063A50355640052055181BE
:10A6B00097100100E780A0542A8965D18347B40030
:10A6C00093F7070E99C71305840197300100E780BF
:10A6D000609983574400231EF100834784002301BF
:10A6E000F1025C4003550900D98313F7070883473B
:10A6F0001102231CA10093F7F707D98FA300F102E1
:10A7000083572900231DF1005C40F18313F71700E4
:10A710008347F102F99BD98FA307F10297A00000AC
:10A72000E780E0952AD235D98347940068001397D3
:10A7300057008347B400FD8BD98FA305F4001C4854
:10A7400003D647008C4397200000E78000A6A68729
:10A7500017870100130747AE740005464C10268585
:10A7600097000000E78060942A890DD98347B400E0
:10A77000A685FD8BA305F40097000000E78060DF4D
:10A7800031BF1783FFFFE7020395832485FE2A84E8
:10A790004111268597000000E78080D7834734FF6A
:10A7A00093F7070E8DCB2AC6268597000000E78019
:10A7B00060C809CD834734FFB245FD8BA309F4FE81
:10A7C00091C5228597300100E7808087410117837A
:10A7D000FFFF670083927DD98327C4FF2685829778
:10A7E00075F5834734FF93F7070E91C7228597309D
:10A7F0000100E7802087032584FE97000000E780A2
:10A8000000E5E9B71783FFFFE702E3899C414111A7
:10A810002A8903C7070089472E84935667006380FF
:10A82000F6040D466388C6049307F0076304F70235
:10A830002E8597200000E780C0A7AA848149C16BBC
:10A84000130C490097B7FF1F9387876E9C43984767
:10A8500063E4E90441011783FFFF6700838803D79E
:10A8600045008547E3F8E7FE2E8597200000E78046
:10A87000A0A9E1B703D74500E3FEE7FC2E859720AA
:10A880000000E78000A3AA84228597200000E780CB
:10A8900060A4C204C98C5DB7DC470355A900139AB4
:10A8A00049003E9A93170501C187635DF000835705
:10A8B0000A006397A70263E774038327CA00034D66
:10A8C0005A002DA0A1672167A98F1307F7EFE37442
:10A8D000F7FE6397090097000000E780209161FD73
:10A8E00085098DB783278A00034D4A00835DA9003F
:10A8F00003576900216A138BC7003AC6814A33CADD
:10A900004D01631E5D0197B7FF1F9387E7629C436C
:10A91000E1DBA2866286814526858297D1B7A16751
:10A920009387F7EF930C4BFF63F24703B2455A85C9
:10A9300097F0FFFFE780A0710DC103278B00104740
:10A9400009CE10436382C4023107D5BFEE85668508
:10A9500097000000E780008F71F993861A0093FA40
:10A96000F60F130B0B0271BF835644005C43E3E9FF
:10A97000F6F622853AC697100000E780807DA16731
:10A980009387D7042A8A035D4400324763E897001F
:10A990008347D90093E707F8A306F9001C476685AB
:10A9A0002286E2858297C1670844FD17337AFA0050
:10A9B000529508C02312A40125B797B7FF1F9387AC
:10A9C00027579843814715C31447814763FFD50034
:10A9D000939745004C47BE9519C903C75500814759
:10A9E0006375E600DC451606B2973E85828003C794
:10A9F00045008147E37BE6FE16069C45F5B71773D5
:10AA0000FFFFE702A36BAA892E8A814497BAFF1F32
:10AA1000938A0A5283A70A00984763E6E4001773F3
:10AA2000FFFF6700E36CDC471394440001493E9448
:10AA300013BB140083474400634BF900014913BB67
:10AA4000140083475400634FF9008504E1B70844BC
:10AA5000931759005287DA860146A2853E9582995E
:10AA60000509C9BF4844931759005287DA8605463D
:10AA7000A2853E9582990509E9B71773FFFFE702A2
:10AA80008365814517F5FFFF1305054897B7FF1F3D
:10AA90002392074A97000000E780A0F61773FFFF94
:10AAA0006700A36597B7FF1F938787489C4395C3AB
:10AAB0001773FFFFE7022362814517F5FFFF1305B8
:10AAC000A54497000000E780C0F31773FFFF6700FD
:10AAD000C36282801773FFFFE702435E37E404001E
:10AAE0008327841241112315E100AE893289368A09
:10AAF0003A8681460147ED45AA8482972AC621C934
:10AB00000356A100D28597400100E780C024832727
:10AB1000C413CE8526858297058905C98327440DF0
:10AB20002314210101462C00268582972A8401C91D
:10AB3000B7E7040083A7C712ED4528008297228556
:10AB400041011773FFFF6700A35A4944D5B7655405
:10AB5000FDB75C41FD175CC182801773FFFFE70200
:10AB60008357B7E70400FC5F829795473305F502EA
:10AB700081450D811773FFFF670023581773FFFF8F
:10AB8000E7026355B7E70400FC5F829795473305FA
:10AB9000F5020D811773FFFF670023561773FFFF40
:10ABA000E7026353B7E7040083A7870B035505004B
:10ABB00082971773FFFF670043541773FFFFE70285
:10ABC0008351035505003287AE861796FF1F035643
:10ABD000C68D97B5FF1F9385653697000000E78007
:10ABE000A0EF1773FFFF670043511773FFFFE702E2
:10ABF000834EB7E7040083A7C71782971773FFFF39
:10AC00006700A34F1773FFFFE702E34CB7E70400A9
:10AC100083A7871397B5FF1F938545328297014518
:10AC20001773FFFF6700634D1773FFFFE702A34A27
:10AC3000B7E7040083A7C71F81451795FF1F03557A
:10AC4000C58282971773FFFF6700234B1773FFFFBF
:10AC5000E7026348B7E7040083A7871397B5FF1F90
:10AC60009385C52E829701451773FFFF6700E34860
:10AC70001773FFFFE7022346B7E7040083A7C71F48
:10AC800081451795FF1F0355458482971773FFFF72
:10AC90006700A3461773FFFFE702E3432E85978003
:10ACA0000000E780E0AF97800000E780E0EC1773DA
:10ACB000FFFF670083441773FFFFE702C3419780DC
:10ACC0000000E780E0F61773FFFF670003435C496D
:10ACD000E1175CC95CC583572501A1072319F5005D
:10ACE00083570501A1072318F5008280F14733053A
:10ACF000F50297B7FF1F938767279C433E95828095
:10AD00008D476315F60803D74600854763F0E708CB
:10AD10001773FFFFE702233C368536842E89971090
:10AD20000000E780005929C98357440093140501A6
:10AD3000C18063E39704228597100000E780605785
:10AD4000FD14231294009307A0026300F5029307F9
:10AD5000B0026307F50293079002631FF500228596
:10AD600097000100E780C08501A80146CA852285B9
:10AD700097A00000E78060B01773FFFF6700E3371C
:10AD8000228597100000E780C003FDB7828097B648
:10AD9000FF1F9386E61D9C42014599CF9843D442FC
:10ADA00017B6FF1F2326E61C6396D70097B6FF1F32
:10ADB00023A2E61C1385C7FE82801773FFFFE702FC
:10ADC000833197000000E780A04B71443305850272
:10ADD000914597900000E78020E911E565551773CC
:10ADE000FFFF6700833197B7FF1F23AFA7169700B8
:10ADF0000000E780E0483305850291459790000008
:10AE0000E78080E661DD97B7FF1F23A1A7169700B3
:10AE10000000E780E04697B7FF1F2391A714970033
:10AE20000000E780E04597B7FF1F239AA7129777A6
:10AE300001009387A74517B7FF1F2325F712970730
:10AE40000000938707E917B7FF1F232BF710014571
:10AE500079B71773FFFFE7020328AA8517B5FF1F0D
:10AE60001305C50F97100000E780C05B1773FFFF45
:10AE70006700A3281773FFFFE702E3259700000090
:10AE8000E78060FD97100000E780405B97B7FF1FE9
:10AE90009387070E9C4391CF1387C7FE19CB83D5A9
:10AEA000C7FF17B5FF1F1305250D97200100E78089
:10AEB00020191773FFFF670043241773FFFFE70292
:10AEC000832197000000E780C0EC09CD834785000F
:10AED0002A8493F7070499EB0355E50097000000D7
:10AEE000E78080F91773FFFF670023218347C500C0
:10AEF0009304450117B9FF1F1309890785E38327C9
:10AF000009005CC997B7FF1F23A497068327490050
:10AF1000F1FB97B7FF1F23AF9704E9B7FD1723068F
:10AF2000F500610597800000E780C0D683078400A4
:10AF300063CB07048347840093E707F82304F400F6
:10AF4000B7E704009C5F82974205A94741813375AA
:10AF5000F5028347840093F707FCC98F2304F400AC
:10AF60008347D4003E951C402318A40089CF984302
:10AF700019CB8347C4005040814585073305F5024E
:10AF8000420541810297832709005CC897B7FF1FDC
:10AF900023A097FE8327490089E797B7FF1F23ABBC
:10AFA00097FC8347C4009DDF8355040117B5FF1F3D
:10AFB000130585FC97200100E780800825B71773EB
:10AFC000FFFFE702431197B7FF1F938727209C4796
:10AFD00001448583858B85E3AE84B2853A869710DC
:10AFE0000000E780804B2A8419C597100000E78095
:10AFF000C041829408CC22851773FFFF6700E30FDE
:10B000001773FFFFE702830B41112E8932C6AA890D
:10B0100097000000E780C031324713060502CA8658
:10B02000970500009385C5CC17B5FF1F130505F3E1
:10B0300097000000E780E0F82A8425C99304C50042
:10B0400097000000E780E0411946AA852685971001
:10B050000000E78080158545268597100000E78071
:10B06000601117750100130525204E9583450500D5
:10B07000268597100000E78020165C483146814500
:10B08000A1075CC85CC483572401E1172319F400AD
:10B0900083570401E1172318F4001C4C3E85977078
:10B0A000FFFFE7804006A3042501228541011773B5
:10B0B000FFFF6700E3031773FFFFE702C3014111BE
:10B0C000AA842EC632C497100000E7806036004D77
:10B0D000B2452246834784000CC050C093F7F70363
:10B0E00093E707042304F40023180400268597102F
:10B0F0000000E780803183479400A9462317A4000D
:10B1000013D7370005073307D7029D8B8507230622
:10B11000F400A306E40083C70401D8488507230F81
:10B12000F7FE17B7FF1F1307A7E45843232A0400AD
:10B130009307440129E317B7FF1F232DF7E217B741
:10B14000FF1F2327F7E217B4FF1F1304E4E2228551
:10B1500097200100E78000E11C44858B5D8D19E597
:10B160008145228597200100E78080ED410117731A
:10B17000FFFF670083F81CC317B7FF1F232CF7DE00
:10B18000D9B71773FFFFE70203F597050000938512
:10B1900065B7014597000000E78000B001451773CF
:10B1A000FFFF670083F51773FFFFE702C3F2970005
:10B1B0000000E78080B01773FFFF670003F4834748
:10B1C000C500A5E31773FFFFE702E3F02A840355E8
:10B1D000E50097000000E78000C821C18347840094
:10B1E00093F7F7FB2304F4001C4091C7DC4381C7AD
:10B1F0004C400145829797000000E78080B917B561
:10B20000FF1F130565D797200100E780A0E50355D0
:10B21000E40097000000E78020C61773FFFF670077
:10B22000C3ED82801773FFFFE702E3EA97B7FF1FC2
:10B23000938707D497050000938565C817B5FF1F4E
:10B24000130585D323A0070023A207009720010040
:10B25000E780E0CE1773FFFF670023EA1C4D91CF14
:10B26000DC4381CF1773FFFFE702E3E68345070066
:10B2700082971773FFFF670043E8828097B7FF1F2D
:10B280009387C7D19C4303C50700828097B7FF1FF0
:10B290009387C7D09C4303C51700828097B7FF1FD1
:10B2A0009387C7CF9C4303C52700828097B7FF1FB2
:10B2B0009387C7CE9C4303C54700828097B7FF1F83
:10B2C0009387C7CD9C4303C53700828097B7FF1F84
:10B2D0009387C7CC9C4303C55700828097B7FF1F55
:10B2E0009387C7CB9C4303C56700828097B7FF1F36
:10B2F0009387C7CA9C4303C57700828097B7FF1F17
:10B300009387C7C99C4303C58700828097B7FF1FF7
:10B310009387C7C89C4303C59700828097B7FF1FD8
:10B320009387C7C79C4303C5A700828097B7FF1FB9
:10B330009387C7C69C4303C5B70011E11D458280B2
:10B3400097B7FF1F938787C59C4303C5C7008280BB
:10B3500097B7FF1F938787C49C4303C5D70082809C
:10B3600097B7FF1F938787C39C4303C5E70082807D
:10B3700097B7FF1F938787C29C4303D5070182803D
:10B3800097B7FF1F938787C19C4303C5270182801E
:10B3900097B7FF1F938787C09C4303D547018280DF
:10B3A00097B7FF1F938787BF9C4303D567018280B0
:10B3B00097B7FF1F938787BE9C4303D58701828081
:10B3C00097B7FF1F938787BD9C4303C5A701828062
:10B3D00097B7FF1F938787BC9C4303C5B701828043
:10B3E00097B7FF1F938787BB9C4303C5C701828024
:10B3F00097B7FF1F938787BA9C4303C5D701828005
:10B4000097B7FF1F938787B99C438857828097B768
:10B41000FF1F9387A7B89C4303D5C702828097B7C5
:10B42000FF1F9387A7B79C4303D5E70219E11305D4
:10B43000800C828097B7FF1F938747B69C4303C554
:10B440000703828097B7FF1F938747B59C43C85B6C
:10B45000828097B7FF1F9387E7B38843828097B7AF
:10B46000FF1F938767B38843828019E17D558280EF
:10B47000F5DE984265DFFDD917B7FF1F130707D523
:10B480001847AA877155058B631D072403C507005C
:10B490001547E37DA7FC03C737001305F0057D17AB
:10B4A0001377F70FE364E5FC03C35700E30003FCE5
:10B4B00083C86700E38C08FA03C77700494579170A
:10B4C0001377F70FE364E5FA03C7A70011481305E4
:10B4D000F7FF1375F50FE36BA8F803CE97000D483F
:10B4E0001305FEFF1375F50FE362A8F803C8B70054
:10B4F0006309080065181378F80F1305600DE367FA
:10B5000005F703C5C700794879151375F50FE36F83
:10B51000A8F403C8D7000D457D181378F80FE3672A
:10B5200005F503D80701930E401751184208135828
:10B530000801E3ED0EF303C8E7007D181378F80F58
:10B54000E36605F303C827017D181378F80FE36F4E
:10B5500005F103C88700C54E75181378F80FE3E7A7
:10B560000EF103D86701856E938EBEE06D18420818
:10B5700013580801E3EC0EEF03D847016D18420899
:10B5800013580801E3E40EEF03D887017918420845
:10B5900013580801E36C05ED03C8A7017D18137863
:10B5A000F80FE36505ED03C5B7011D487D1513755B
:10B5B000F50FE36DA8EA03C5D70171487915137536
:10B5C000F50FE365A8EA03D5E7011308E00F7D1541
:10B5D00042054181E36CA8E803C507024948791593
:10B5E0001375F50FE364A8E8C85301C937C83400E0
:10B5F0005915130858BFE36BA8E603A8870237C59F
:10B600003400130555BF5918E36205E717B5FF1F4E
:10B610002324C59803C6050117B5FF1F2320F598FD
:10B620000545E375C5E403D82501D0493376060303
:10B63000E31E06E203C61501E30A06E217B6FF1F82
:10B64000232AB69483C5270001466387A50003C655
:10B650001700F1453306B60283C707039305C002FE
:10B6600072971A071307C70516031A979608469785
:10B67000B387B70241553E973297420741836362D1
:10B68000E8061773FFFFE70203A5368597800000E1
:10B69000E780A06897000100E78020482A8497A0EF
:10B6A0000000E780805A2A9497F00000E780602627
:10B6B0002A9497900000E780A0812A9497F0FFFFDA
:10B6C000E780E06F2A9497400000E78060932A9417
:10B6D00097700000E780A09C22951773FFFF67001A
:10B6E000C3A182801773FFFFE702E39E4111A30706
:10B6F000A10097A00000E780A0C59305F100170501
:10B7000000001305E5B597F0FFFFE780802F0145A6
:10B7100041011773FFFF6700439E1773FFFFE702A6
:10B72000039917B4FF1F130464AA032884007959EE
:10B730009368180097B4FF1F23AE14A9137818005C
:10B7400063100802BA84BE89368B328A2E89AA8A8F
:10B7500097F0FFFFE780E0A77D15269519E53159A1
:10B760004A851773FFFF6700039897F0FFFFE78094
:10B7700040A67D152695A167E353F5FE97B7FF1FF9
:10B780009387C7DB98433E8C814B01CB014597F0F3
:10B790000000E7802044933B15004A85DA865686F0
:10B7A000D28597900000E780C04D2A8911CD1C44B6
:10B7B000F99B17B7FF1F232FF7A083270C00CDD3CA
:10B7C000E3800BFA829769BF268597B7FF1F23A1F5
:10B7D00007A097F0FFFFE780809C4146CE8517B514
:10B7E000FF1F130525A897300100E780C05697D0AA
:10B7F0000000E78040990325040B97D00000E78004
:10B80000009D054597D00000E78000A405459700FE
:10B810000000E78060EDA9B797B7FF1F9387079BEC
:10B820009C47858BEDC71773FFFFE702C38A17B5E7
:10B83000FF1F130565A197B7FF1F23A9079897B7A7
:10B84000FF1F23A7079897B7FF1F23A507989720E7
:10B850000100E780208197500000E780E0F5971015
:10B860000100E780A04C97100100E780A05297B735
:10B87000FF1F938727949C4391C70545978000003D
:10B88000E780402097A7FF1F9387877C9C4399C739
:10B8900041657D1597700000E78040A297F0000099
:10B8A000E780E03D97D00000E780808F97B7FF1FCB
:10B8B0009387C7A69C43139717016356070097F019
:10B8C0000000E78000AD97B7FF1F23AD079897B73B
:10B8D000FF1F23AB079897B7FF1F23A9079897B7B8
:10B8E000FF1F23A7079897000000E780008C9700B0
:10B8F0000000E780007297F0FFFFE780401897F0A4
:10B900000000E78040D61763FFFF6700037F828057
:10B9100097B7FF1F9387878B884382801763FFFF4A
:10B92000E702637B97800000E780607597800000E6
:10B93000E780C0771763FFFF6700237C1763FFFF73
:10B94000E702C3772A849304140201112E85B28979
:10B95000A685214636C63A8997300100E780403DEA
:10B960000DE9B24638082686CE8513059404975013
:10B970000000E780604121462C084A85973001008D
:10B98000E780003B1335150005611763FFFF670073
:10B9900023760145D5BF1763FFFFE702C373930505
:10B9A000450617A5FF1F1305A55F97100100E78047
:10B9B00020691763FFFF670043741763FFFFE70207
:10B9C000837141112EC697F0FFFFE780601BB245DF
:10B9D00088C141011763FFFF670023721763FFFFF0
:10B9E000E702C36DAA842E8497800000E780006C74
:10B9F000AA898545228597000000E780E07D83C7FE
:10BA0000E4011389940899E313890403CE85228500
:10BA100097000000E780407C2146930519022285AB
:10BA200097000000E780607897A7FF1F9387077A49
:10BA30008C43228597100000E780C08221469385C1
:10BA40008402228597000000E78020761763FFFFBD
:10BA50006700036A1763FFFFE7026365397197F0B8
:10BA60000000E780E0B49305400661E9978000009C
:10BA7000E78000606302051497A7FF1F83C7075480
:10BA800013B7170097A6FF1F238AE652014499CFE8
:10BA9000C16417A9FF1F130969739309400EFD14B0
:10BAA00097000000E780C0866342A40A97F0FFFF7A
:10BAB000E780000D4169B7290900096AFD7A2A8BE0
:10BAC00081447D199389F97B130A0A71938A8AC785
:10BAD00097000000E780C08363D7A4041304400EDE
:10BAE000B387840217A7FF1F1307476E0324070BB2
:10BAF0003E948357C4016382270B18403307EB4001
:10BB000063EAE900834744008507B3874703D69774
:10BB10006365F70801468145094597F0FFFFE78017
:10BB2000604EAA8B29E597400000E7808083854717
:10BB30006317F50689659385057117A5FF1F130522
:10BB4000254697100100E780A04F95A0B307340366
:10BB50000327090BBA9703D7C7016308970003C7E8
:10BB60005700A38207002382E700050415BF930551
:10BB7000C500228597000000E78080E65E8522866A
:10BB8000976501009385856F97F0FFFFE780E0528E
:10BB90005E8597100000E780608A850415BF97A72F
:10BBA000FF1F9387A7629C478D83858BC1F7216117
:10BBB0001763FFFF6700235301468545094502D0FF
:10BBC00002D202D402D697F0FFFFE780A043AA84F6
:10BBD00079DD97F00000E780E09C1389C4002A8497
:10BBE00081454A8597000000E780005F0C40414690
:10BBF0004A8597000000E780405B83294400638505
:10BC0000090C4E8502D802DA02DC02DE9730010010
:10BC1000E78000482ACE141005462C0808184ECCA0
:10BC200097500000E780E00A1375F50F51ED83553A
:10BC3000840093E525004A8597000000E780E05ED8
:10BC400011460C104A8597000000E7800056014617
:10BC50009765010093850563268597F0FFFFE780D0
:10BC6000C045268597000000E780407D5C40A1D359
:10BC7000014685450D4597F0FFFFE780A038AA846F
:10BC80001DD548401389C40097300100E78040402B
:10BC90002AC64A8597000000E780404C3246636F11
:10BCA000C5004C404A8597000000E78000500146DF
:10BCB0008145268597F0FFFFE78020402685970085
:10BCC0000000E780A077E5B583558400ADB7176322
:10BCD000FFFFE702434097A7FF1F9387274F9C472B
:10BCE0001DC193E7870017A5FF1F1305652B17A735
:10BCF000FF1F2321F74E97100100E78040321763A2
:10BD0000FFFF6700833FDD9B17A7FF1F2324F74C2E
:10BD100097300000E780E0647DF117A5FF1F130551
:10BD2000252897100100E780E033D1BF1763FFFF9C
:10BD3000E702E3374169AA892E8AB28A368BBA8B29
:10BD4000814417ACFF1F130C6C48930C400E7D19F7
:10BD500097F0FFFFE780C05B63C4A40001443DA0EF
:10BD60003384940383270C0B3E948357C40163866A
:10BD700027055A87D6865286CE8513050403970079
:10BD80000000E780E0BB01C923800B002285176318
:10BD9000FFFF670043358347F40185C35A87D68682
:10BDA0005286CE851305940897000000E78040B9BD
:10BDB00009C585472380FB00D1BF850451BF835748
:10BDC00045006380071E1763FFFFE702232F011161
:10BDD0002A8497000000E780C04D09C985476309A0
:10BDE000F50605611763FFFF6700833097E00000E9
:10BDF000E780007C7DF5835744004947ED9BE39243
:10BE0000E7FEC145228597000000E7804033AA8401
:10BE1000228597000000E780204F0357440002CEA0
:10BE200091472A89631AF700228597000000E7806E
:10BE3000A0513C082ACC3ECE97E00000E7808076F7
:10BE40005C55C5D374084A86A6850545829751BFBF
:10BE500003574400D147E3F6E7F8032A0400C16919
:10BE6000014997AAFF1F938A6A36130B400EFD19EA
:10BE700097F0FFFFE780C049634FA90E2285032A90
:10BE8000040097000000E780C042A1452A8922856E
:10BE900097000000E780A02AAA842285970000006E
:10BEA000E780804A14402A86AA8978082685CA85B0
:10BEB00097000000E780C0E7AA8405D503C7F40116
:10BEC00089476315F7008347C10181DF5546D28555
:10BED0001385640097300100E780E0E70145978013
:10BEE0000000E780C01901C583D7C401A5E797A763
:10BEF000FF1F9387A72D9C4793551900858913D75A
:10BF00003700058B01CF8983858B6399B700014585
:10BF10002EC697000000E780C0DBB2454E859780B3
:10BF20000000E780601F0346C1012A849375190051
:10BF3000268597900000E780E03935C126859780F7
:10BF40000000E780E018268511C0014597800000B9
:10BF5000E780004C97300000E780A0408547E3125F
:10BF6000F5E883C754001307F00FE38CE7E6850775
:10BF7000A382F400BDB5B304690383A70A0BBE9482
:10BF800083D7C401638B37015546D285138564007E
:10BF900097300100E780C0D955DD0509D1BD5DD8D6
:10BFA0006DB782801763FFFFE7024311978000009F
:10BFB000E780000C05C1C164014417A9FF1F1309E4
:10BFC000E9209309400EFD1497F0FFFFE78040340D
:10BFD000634EA40017A5FF1F130585FC97100100F1
:10BFE000E780E0031763FFFF670083103305340326
:10BFF0008327090B3E958357C50163889700231259
:10C00000050097800000E780A00C050475BF97A786
:10C01000FF1F9387A71B9C478D83858B8DE3176339
:10C02000FFFFE702430B17A5FF1F130565F79710E6
:10C030000100E78020031763FFFF6700030C828085
:10C040001763FFFFE7022309970500009385C5A04A
:10C0500017A5FF1F1305C5F497100100E78020EE18
:10C060001763FFFF670063091763FFFFE702A3067B
:10C070008841B7E70400BC5B050542054181829712
:10C0800009C585472300F50005051763FFFF670015
:10C09000C30683C7F5FF2E858507A38FF5FE828033
:10C0A00083C7F5FFFD1793F7F70FA38FF5FE99EF01
:10C0B0001763FFFFE7022302B7E70400BC571385AD
:10C0C000F5FF82971763FFFF6700230382801C41FF
:10C0D000035745008D8FBA951CC12312B5003E85CC
:10C0E000828093D78500A2051441DD8D83574500DA
:10C0F0001387E6FF18C189072312F50013D68500C0
:10C100004111238FB6FEA38FC6FE410182801841E4
:10C110009307F7FF1CC18357450085072312F500DD
:10C12000A30FB7FE8280835745008D8F2312F50041
:10C130001C41BE950CC12E858280AA8703D747007B
:10C1400008410D8FAA952392E7008CC38280184185
:10C1500008453305A7408280835745000357650093
:10C160001D8F1C4108453385A7403305A7408280B9
:10C170001763FFFFE70223F641112EC62A849700BA
:10C180000000E780A0FDB2456373B50001A08357AE
:10C1900044000840BE952312B4003E954101176348
:10C1A000FFFF670083F51763FFFFE702C3F241114A
:10C1B0002E84B28532C697000000E780A0FB32468D
:10C1C000A28597300100E78000B941011763FFFFA6
:10C1D0006700A3F21763FFFFE702E3EF2E848545B4
:10C1E00097000000E78000F9230085001763FFFF38
:10C1F0006700A3F01763FFFFE702E3ED4111231788
:10C20000B100894597000000E780C0F68347E10050
:10C210002300F5008347F100A300F50041011763F7
:10C22000FFFF670083ED1763FFFFE702C3EA93D7C1
:10C230008500A2054111DD8D2317B10089459700C6
:10C240000000E78020F38347E1002300F5008347E7
:10C25000F100A300F50041011763FFFF6700E3E968
:10C260001763FFFFE70223E71397850193D7850143
:10C27000C166938606F0D98F13D78500758FD98F45
:10C28000A2053707FF00F98D4111DD8D2EC69145BE
:10C2900097000000E78000EE6C0011469730010027
:10C2A000E78060AB41011763FFFF670003E5176399
:10C2B000FFFFE70243E21C41854503C407009700E6
:10C2C0000000E78080E622851763FFFF6700E3E256
:10C2D0001763FFFFE70223E01C414111894503C7B3
:10C2E000070083C717002307E100A307F1009700A9
:10C2F0000000E78080E30355E10041011763FFFF81
:10C300006700A3DF1763FFFFE702E3DC1C41411175
:10C31000894503C7070083C717002307E100A30768
:10C32000F10097000000E78040E08357E100410101
:10C3300013D58700A2075D8D420541811763FFFF7A
:10C340006700A3DB1763FFFFE702E3D80C4141114D
:10C350002A841146680097300100E780C09F91450C
:10C36000228597000000E78040DCB247C1669386D3
:10C3700006F01397870113D58701598D13D78700CE
:10C38000758F598DA2073707FF00F98F5D8D410129
:10C390001763FFFF670063D61C45BE950CC1828002
:10C3A000AE87944391E6584101EF0CC15CC1828095
:10C3B00003C7570013671700A382E700B687D5B7F6
:10C3C0000CC3EDB7AA87084119CD1841D44398C3CF
:10C3D0006313D500D8C32A87034657009376160007
:10C3E00081E6232007008280944381CA8C4203A8FF
:10C3F00047008CC363930601CCC3799A14C3A3028C
:10C40000C7003687D1BF1C45DC471D8DB777DBB62B
:10C41000938777DB09853305F502420541818280E8
:10C42000F147B385F50248452E9582808347450044
:10C4300085072302F50082801763FFFFE702A3C987
:10C440002A8409E41763FFFF670023CB8347440076
:10C45000F5DBFD1793F7F70F2302F400E5F71C4413
:10C4600003D7270005072391E700DC4399C3228502
:10C4700082974C4889CD83475400898B99E71C44A7
:10C4800022859C479C439C478297232A04000040B6
:10C49000232004007DB71763FFFFE702C3C3835760
:10C4A000250041112EC681EB01442285410117630D
:10C4B000FFFF670083C4035705008147F146E3058A
:10C4C000F7FEB385D702404585072E948345440087
:10C4D00008C4F5F5B247AA8481E7232A040009A815
:10C4E0001C456C0022859C439C43829748C84DDDC7
:10C4F00085472312F400B2472320040023180400C8
:10C500002319F4005C485CC483D72400FD172391F1
:10C51000F40061BF1763FFFFE702E3BB97A7FF1FAC
:10C52000938707AA88432326050023240500410595
:10C5300097100100E78000B31763FFFF6700E3BBBC
:10C540001763FFFFE70223B917A4FF1F130444A7D3
:10C550001C40411199CF9C472300B5002AC65CC1FD
:10C5600097000000E78040FB1C40DC4399C3324544
:10C57000829741011763FFFF670023B80347450017
:10C5800029E3584DAA877D551DCF1763FFFFE702AA
:10C5900083B41CC3DC4797A6FF1F23A3E6A2F15672
:10C5A000130507012390D700970500009385050226
:10C5B00097100100E780A09801451763FFFF67000F
:10C5C000C3B37D55828082801763FFFFE702A3B06B
:10C5D00001116146814528009760FFFFE780A0B206
:10C5E00097A7FF1F9387C79D9C4328009305F00FD3
:10C5F000DC473EC697000000E780C0F40561176382
:10C60000FFFF670083AF97A7FF1F9387679B9C433C
:10C61000D847A1679387C702631EF70A397106DE00
:10C6200022DC26DA80004AD84ED652D456D2328541
:10C63000B28497000000E780C0C7AA8926859700CA
:10C640000000E78020C92318A4FC2685970000007D
:10C65000E78040C82319A4FC268597000000E780E6
:10C6600060C783D744000A8A231AA4FC858393F702
:10C67000F70F230EF4FC8607BD0793F7073F33013E
:10C68000F1408A8A01498347C4FD6367F902CE8578
:10C69000130584FC232C54FD97000000E78080EAFA
:10C6A0005281130104FCF2506254D2544259B259DF
:10C6B000225A925A21618280268597000000E780E5
:10C6C00060C193171900D69705092390A700137925
:10C6D000F90F55BF828097A7FF1F9387678E9C43F2
:10C6E000D847A1679387A702631AF70A397106DE54
:10C6F00022DC26DA80004AD84ED652D456D2328571
:10C70000B28497000000E780C0BAAA892685970006
:10C710000000E78020BCFD572318A4FC26852319C0
:10C72000F4FC97000000E780E0BA83D744000A8A4F
:10C73000231AA4FC858393F7F70F230EF4FC8607D6
:10C74000BD0793F7073F3301F1408A8A01498347C8
:10C75000C4FD6367F902CE85130584FC232C54FDC8
:10C7600097000000E78000DE5281130104FCF250C4
:10C770006254D2544259B259225A925A216182804B
:10C78000268597000000E780E0B493171900D6973C
:10C7900005092390A7001379F90F55BF828097A749
:10C7A000FF1F9387E7819C43D847A16789076310E0
:10C7B000F70A397106DE22DC26DA80004AD84ED626
:10C7C00052D456D23285328997000000E78060AE9D
:10C7D000AA894A8597000000E780C0AF83574900C7
:10C7E0000A8A2318A4FC858393F7F70F230CF4FC23
:10C7F0008607BD0793F7073F3301F1408A8A8144DA
:10C80000834784FD63E7F402CE85130584FC232A65
:10C8100054FD97000000E780E0D25281130104FC30
:10C82000F2506254D2544259B259225A925A21615A
:10C8300082804A8597000000E780C0A99397140082
:10C84000D69785042390A70093F4F40F55BF8280F8
:10C850009797FF1F9387C7769C43D847A167938715
:10C86000E704631EF70A397106DE22DC26DA80004F
:10C870004AD84ED652D456D23285B28497000000A0
:10C88000E78020A3AA89268597000000E78080A47E
:10C890002318A4FC268597000000E780A0A3231A94
:10C8A000A4FC268597000000E780C0A283D744003F
:10C8B0000A8A2319A4FC858393F7F70F230EF4FC4F
:10C8C0008607BD0793F7073F3301F1408A8A014984
:10C8D0008347C4FD6367F902CE85130584FC232CCE
:10C8E00054FD97000000E780E0C55281130104FC6D
:10C8F000F2506254D2544259B259225A925A21618A
:10C900008280268597000000E780C09C931719005D
:10C91000D69705092390A7001379F90F55BF828098
:10C920009797FF1F9387C7699C43D847A167938751
:10C93000C704631AF70A397106DE22DC26DA8000A2
:10C940004AD84ED652D456D23285B28497000000CF
:10C95000E7802096AA89268597000000E7808097C7
:10C96000FD572318A4FC2685231AF4FC9700000029
:10C97000E780409683D744000A8A2319A4FC858364
:10C9800093F7F70F230EF4FC8607BD0793F7073FD5
:10C990003301F1408A8A01498347C4FD6367F90284
:10C9A000CE85130584FC232C54FD97000000E780FE
:10C9B00060B95281130104FCF2506254D2544259BE
:10C9C000B259225A925A216182802685970000002E
:10C9D000E780409093171900D69705092390A70088
:10C9E0001379F90F55BF82809797FF1F9387475D93
:10C9F0009C43D847A167DD076317F7041753FFFF70
:10CA0000E702636D79713285328497000000E78018
:10CA1000408A2AC6228597000000E780A08B231158
:10CA2000A102228597000000E780A088B24523007C
:10CA3000A102280897000000E780C0B045611753A5
:10CA4000FFFF6700836B82809797FF1F938747578D
:10CA50009C43D847A167938787046317F70417534C
:10CA6000FFFFE70243677971328532849700000047
:10CA7000E78020842AC6228597000000E780808511
:10CA80002311A102228597000000E7808082B24531
:10CA90002300A102280897000000E780A0AA4561B2
:10CAA0001753FFFF6700636582809797FF1F938787
:10CAB00027519C43D847A1679387A7046312F702C5
:10CAC0001753FFFFE70223610111280081459700FA
:10CAD0000000E78020A705611753FFFF6700E361AF
:10CAE00082809797FF1F9387A74D9C43D847A167E4
:10CAF000938757026319F7021753FFFFE702A35DFD
:10CB00000111328597F0FFFFE780A07A2308A1008A
:10CB10008145280097000000E780C0A205611753F7
:10CB2000FFFF6700835D82809797FF1F93874749C8
:10CB30009C43D847A1679387E702631BF704175309
:10CB4000FFFFE702435901113285328497F0FFFF5E
:10CB5000E7804078AA84228597F0FFFFE7808077FE
:10CB6000854709E9228597F0FFFFE7808074420539
:10CB7000B337A00028008145231891003ECA9700D2
:10CB80000000E780209C05611753FFFF6700E35614
:10CB900082809797FF1F9387A7429C43D847994766
:10CBA0006313F7081753FFFFE702E35279713285E9
:10CBB000328497F0FFFFE780C06F2AC6228597F086
:10CBC000FFFFE78020712310A102228597F0FFFF6D
:10CBD000E780206E2301A102228597F0FFFFE78006
:10CBE000406DA301A102228597F0FFFFE780606CF2
:10CBF0002302A102228597F0FFFFE780806B2313B9
:10CC0000A102228597F0FFFFE780A06AB2452314B6
:10CC1000A102280897000000E780C09245611753E1
:10CC2000FFFF6700834D82809797FF1F93874739E7
:10CC30009C43D847A1679387C7036313F70817532B
:10CC4000FFFFE702434979713285328497F0FFFF95
:10CC5000E78020662AC6228597F0FFFFE78080677D
:10CC60002310A102228597F0FFFFE780A066231121
:10CC7000A102228597F0FFFFE780A0632302A102B3
:10CC8000228597F0FFFFE780C062A302A102228500
:10CC900097F0FFFFE780E0612303A102228597F070
:10CCA000FFFFE7800061B245A303A10228089700B7
:10CCB0000000E780208945611753FFFF6700E343C9
:10CCC00082801753FFFFE702034101112A8497F086
:10CCD000FFFFE780005EAA84228597F0FFFFE780D0
:10CCE000605F228597F0FFFFE780C05E0357440036
:10CCF0008D4763F7E700228597F0FFFFE780805DAF
:10CD0000228597F0FFFFE780E05C2800A68597006A
:10CD10000000E780208305611753FFFF6700E33DB4
:10CD20009797FF1F9387C7299C43D847A167FD07A3
:10CD3000631FF7001753FFFFE702E33932859700BF
:10CD40000000E78040F81753FFFF6700033B828035
:10CD50009797FF1F9387C7269C43D847A167E5078E
:10CD60006315F7081753FFFFE702E3367971328541
:10CD7000328497F0FFFFE780C0532AC6228597F0E0
:10CD8000FFFFE7802055228597F0FFFFE780805462
:10CD90002310A102228597F0FFFFE780A0535205E0
:10CDA00051812311A10222852302010297F0FFFF86
:10CDB000E7802050A302A102228597F0FFFFE780C1
:10CDC000404F2303A102228597F0FFFFE780604ECA
:10CDD000B245A303A102280897F0FFFFE780807601
:10CDE00045611753FFFF6700433182809797FF1F0C
:10CDF0009387071D9C43D847A1679387E703631F69
:10CE0000F7001753FFFFE702032D3285970000005C
:10CE1000E78060EB1753FFFF6700232E8280979710
:10CE2000FF1F9387E7199C43D847A167938747045F
:10CE3000631EF7021753FFFFE702E329797132857A
:10CE4000328497F0FFFFE780C0462AC6228597F01C
:10CE5000FFFFE7802048B245280897F0FFFFE780F2
:10CE6000606E45611753FFFF670023298280979703
:10CE7000FF1F9387E7149C43D847A16793878702D6
:10CE80006310F7041753FFFFE702E324797132853B
:10CE9000328497F0FFFFE780C0412AC6228597F0D1
:10CEA000FFFFE7800041B2452300A102280897F068
:10CEB000FFFFE780206945611753FFFF6700E32309
:10CEC00082801753FFFFE7020321011197F0FFFF54
:10CED000E780203EAA85280097F0FFFFE780806664
:10CEE00005611753FFFF670043219797FF1F938743
:10CEF000270D9C43D847A167D107631FF70017533D
:10CF0000FFFFE702431D328597000000E780A0FB8A
:10CF10001753FFFF6700631E82809797FF1F938759
:10CF2000270A9C43D847A167C507631FF70017531B
:10CF3000FFFFE702431A328597000000E780A0F860
:10CF40001753FFFF6700631B82809797FF1F93872C
:10CF500027079C43D847A167B907631FF7001753FA
:10CF6000FFFFE7024317328597000000E780A0F536
:10CF70001753FFFF6700631882809797FF1F9387FF
:10CF800027049C43D847A167AD07631FF7001753D9
:10CF9000FFFFE7024314328597000000E780A0F20C
:10CFA0001753FFFF6700631582809797FF1F9387D2
:10CFB00027019C43D84789476318F7021753FFFF9F
:10CFC000E70263110111328532C897F0FFFFE78055
:10CFD000402EAA85280097F0FFFFE780A056056144
:10CFE0001753FFFF6700631182809797FF1F938796
:10CFF00027FD9C43D847A1678D076311F70417539A
:10D00000FFFFE702430D01113285328497F0FFFFE5
:10D01000E780202A13066100AA844C0022859730FD
:10D020000000E780C0232800A68597F0FFFFE78077
:10D03000605105611753FFFF6700230C82809797AB
:10D04000FF1F938727F89C4381CFDC4391CB175375
:10D05000FFFFE702430882971753FFFF6700E309CA
:10D0600082801753FFFFE702030779713C08AE8403
:10D070003ED2A165B7070A002A843ED448103C0876
:10D08000DD053ED636C432C63AC297D0FFFFE780F0
:10D09000E02F12474810BA8597F0FFFFE780C013D2
:10D0A00032464810B28597F0FFFFE780E014A246B1
:10D0B0004810B68597F0FFFFE78000125010014737
:10D0C0008146A685228597D0FFFFE7808051456184
:10D0D0001753FFFF670063021753FFFFE702A3FF29
:10D0E00001117C000329C501AE843ECAA165B707C2
:10D0F00007002A843ECC48087C00C5053ECE97D068
:10D10000FFFFE780A0288345D900480897F0FFFF7C
:10D11000E780800C500801478146A685228597D07C
:10D12000FFFFE780004C05611753FFFF6700E3FC3A
:10D130001753FFFFE70223FA83C7950093F7F7071A
:10D14000A384F50097000000E78040F91753FFFF24
:10D150006700A3FA1753FFFFE702E3F779713C0872
:10D16000AE843ED2A165B70709002A843ED4481098
:10D170003C08938545043ED632C636C497D0FFFF9F
:10D18000E780C020A2464810B68597F0FFFFE780F1
:10D19000A00432464810B28597F0FFFFE780C00533
:10D1A000501001478146A685228597D0FFFFE78072
:10D1B000404345611753FFFF670023F41753FFFFF8
:10D1C000E70263F183C7950041112A8493F7F707BB
:10D1D000A384F50032852EC697F0FFFFE780800F0D
:10D1E00085672AC46370F50297700000E78020E924
:10D1F0002246B24509ED114781462285970000007D
:10D20000E78060E641011753FFFF670003EF014726
:10D210008346F501DDB71753FFFFE70223EA01114B
:10D220003C003ECAB7070A003ECC3C003ECE83C756
:10D230009500AA89328593F7F707A384F5002E8419
:10D2400097F0FFFFE78000098567637DF504A1651E
:10D25000AA8493858504480897D0FFFFE7800013D0
:10D26000268597700000E78080E12A8929E19145B1
:10D27000480897F0FFFFE78020F6A685480897F05A
:10D28000FFFFE78060F7CA85480897F0FFFFE78057
:10D29000A0F4014781465008A2854E8597D0FFFF34
:10D2A000E780203405611753FFFF670063E4814581
:10D2B000480897F0FFFFE78020F20349090275BF95
:10D2C0001753FFFFE70283DF79711C103ECAB707CF
:10D2D0000F003ECC404D1C10AA84AE8948089945E9
:10D2E00032C636893ECE97D0FFFFE780200A32460D
:10D2F0004808B28597F0FFFFE78000EE630C090253
:10D30000A545480897F0FFFFE780C0E62546CA8597
:10D3100097200100E78020A4500801478146CE8570
:10D32000268597D0FFFFE780C02B45611753FFFF8D
:10D33000670003DC8355C402480897F0FFFFE780CD
:10D34000A0EB0355E402814505C58547854563018A
:10D35000F502C167FD179305F00F630BF5007D150E
:10D3600097700000E780208E9305150093F5F50F68
:10D37000480897F0FFFFE78020E68345040348084C
:10D3800097F0FFFFE78040E583451403480897F0D6
:10D39000FFFFE78060E483552403480897F0FFFF10
:10D3A000E78080E583554403480897F0FFFFE78056
:10D3B000A0E49DB71753FFFFE702E3D183C79500B1
:10D3C0008146014693F7F707A384F5009700000014
:10D3D000E78040EF1753FFFF670023D21753FFFF8B
:10D3E000E70263CF79713E841C103ECA2E89B707CD
:10D3F0000F00A1653ECCFD051C10AA84480842C060
:10D400003AC23ECE36C432C697D0FFFFE78000F85E
:10D4100032464808B28597F0FFFFE780E0DBA2467E
:10D420004808B68597F0FFFFE78000DD12474808FF
:10D43000BA8597F0FFFFE78020DC0248630C080202
:10D440009145480897F0FFFFE780C0D21146A285BA
:10D4500097200100E7802090500801478146CA8547
:10D46000268597D0FFFFE780C01745611753FFFF60
:10D470006700A3C88945480897F0FFFFE78080CF81
:10D48000834704002300F50083471400A300F50040
:10D49000E1B71753FFFFE70263C283C7950001118D
:10D4A0002A8A93F7F707A384F5003285AE8432C643
:10D4B00097F0FFFFE78000E232462A89328597F035
:10D4C000FFFFE78000DF85676373F902AA894A8559
:10D4D00097700000E780A0BA2A8419ED11478146B1
:10D4E0004A86A685528597000000E780C0B705618F
:10D4F0001753FFFF6700C3BF9387E9FF93F7F70F49
:10D500000547E366F7FE8347F50195EB8947E3801E
:10D51000F9FE8346F401528501474A86A6859700A5
:10D520000000E78040B4A167D90748083ECC230A31
:10D53000010002CE97000000E780A0B04DBF639EBF
:10D54000E7008947639EF90093071020231FF50029
:10D5500097700000E780C0B76DBF0947E39BE7FA0B
:10D560008D47E398F9FA228597700000E78080DF05
:10D570009797FF1F938707C49C4399E79797FF1FCF
:10D58000938707AD9C4399C703D50400978000009B
:10D59000E780A0CE231F040022855DBF1753FFFF45
:10D5A000E70263B301113C003ECAB7070B003ECC53
:10D5B0003C003ECE83C795002A89328593F7F70752
:10D5C000A384F500AE8497F0FFFFE780A0D0931707
:10D5D0000501C187635AF006A1652A849385E50297
:10D5E000480897D0FFFFE78060DAA285480897F0E7
:10D5F000FFFFE78060C09797FF1F938767A59C4355
:10D60000A9EB01449375F40F480897F0FFFFE780FA
:10D61000A0BC9355844093F5F50F480897F0FFFFA1
:10D62000E78080BB9355044193F5F50F480897F0C8
:10D63000FFFFE78060BA014781465008A6854A850A
:10D6400097D0FFFFE780E0F905611753FFFF670000
:10D65000C3AA416585460546A2857D159750000001
:10D66000E78060BD59DD510597000100E780808F9C
:10D67000130440063344850271B71753FFFFE702D6
:10D6800083A50111B70706003EC683C79500216434
:10D690002A8993F7F707A384F500AE842800930541
:10D6A000A4040AC40AC897D0FFFFE78020CE300048
:10D6B00001478146A6854A8597D0FFFFE78060F243
:10D6C00097E0FFFFE780801513049404480822CCFC
:10D6D000230A010002CE97000000E78080960561D2
:10D6E0001753FFFF670063A11753FFFFE702039D76
:10D6F000C1642A8901449799FF1F938929AD130AB0
:10D700008002FD1497E0FFFFE78080C16347A4001B
:10D7100001451753FFFF6700A39DB307440303A709
:10D72000C90ABA9703D707006306970083D7270073
:10D73000638427010504F9B70545E1BF1753FFFFCF
:10D74000E702C3972A8A2E8999C123A0050081493F
:10D750008144979AFF1F938A2A87614B97E0FFFFC6
:10D76000E78040C263C7A4004E851753FFFF6700E0
:10D7700023983384640383A70A003E9483570400EC
:10D7800099E763040900232089008504C1BF41464D
:10D79000D2851305440097100100E780605975F5A4
:10D7A000A289E5B71753FFFFE702439139717C085F
:10D7B0003ED4B7070A003ED67C083ED883C7950002
:10D7C0002A8A328593F7F707A384F5002E8932C69B
:10D7D00097F0FFFFE78000B085676373F508324676
:10D7E000AA84328597F0FFFFE780A0AC8547AA891D
:10D7F00063E8A706A16593858504281097D0FFFFED
:10D80000E780C0B8268597700000E78040872A84AB
:10D8100029ED9145281097F0FFFFE780E09BA68552
:10D82000281097F0FFFFE780209DCE85281097F005
:10D83000FFFFE780609A014781463010CA85528514
:10D8400097D0FFFFE780E0D9A16793877704481856
:10D850003EDC230A010202DE97F0FFFFE780607ED4
:10D8600021611753FFFF6700A3888145281097F0B7
:10D87000FFFFE7806096A685281097F0FFFFE780FE
:10D88000A0979797FF1F938727CB9C4381CB228537
:10D890006389090097D00000E78040248345040293
:10D8A00071B797D00000E780C022CDBF1753FFFFAC
:10D8B000E702C38083C795004111AA8993F7F70750
:10D8C000A384F5003285AE84328A97F0FFFFE780AB
:10D8D00060A08567637FF5022A8997600000E78072
:10D8E000007A2A84914631C58347F501054763874D
:10D8F000E70291C70D476366F704AD461DA893057F
:10D90000050303250A00414697100100E7804042C5
:10D910000DE941011743FFFF6700837D93059508DB
:10D9200003250A00414697100100E78060408146C8
:10D9300069F54A86A6854E8597000000E780C0817C
:10D94000C9BF83250A001305940897700000E7807B
:10D95000A02919C1C146F1BF9797FF1F93878785FB
:10D960009C4399E79787FF1F9387876E9C4399C7CE
:10D97000228597800000E780208A69FD8547A30FF4
:10D98000F400228597B00000E780608422859760CC
:10D990000000E780E0734E8581464A86A68597F0B1
:10D9A000FFFFE780607BA1679387570448003EC470
:10D9B0002302010002C697F0FFFFE780806891BF55
:10D9C0001743FFFFE702A36E83C795004111AA89A1
:10D9D00093F7F707A384F50032852E89B28A97F072
:10D9E000FFFFE780208F85676374F50EAA84976038
:10D9F0000000E780C0682A840DED416B014A978BD7
:10DA0000FF1F938BAB7C130C400E7D1B19A83304B6
:10DA10008A0383A70B0B3E948357C4016383670576
:10DA2000050A97E0FFFFE780A08EE342AAFE954635
:10DA30000DA08357C501639697029305050303A5BF
:10DA40000A00414697100100E780802E994611E1B7
:10DA500081462686CA854E8597F0FFFFE780C06F16
:10DA600085A883A50A001305040397700000E780CA
:10DA7000A017C14679FD2285231E940097A00000BF
:10DA8000E780E074228597600000E78060649797E4
:10DA9000FF1F938767AA9C43A9C323000402228522
:10DAA00097D00000E78040F04E8581462686CA85E3
:10DAB00097F0FFFFE780406AA1679387070448005B
:10DAC0003EC42302010002C697F0FFFFE7806057C3
:10DAD00041011743FFFF6700036189472300F402F8
:10DAE000E1B7397106DE22DC4AD8800052D456D222
:10DAF0005AD026DA4ED65ECE2E8A32892A8B97D01D
:10DB0000FFFFE780E07D0605710541998A8A3301B0
:10DB1000A140232224FC231404FC97D0FFFFE780BC
:10DB2000207C83479A000605350593F7F7072315F0
:10DB3000A4FCA304FA004A85232624FC97E0FFFFF7
:10DB4000E780407993170501C1876340F002568151
:10DB5000130104FCF2506254D2544259B259225A71
:10DB6000925A025BF24B21618280AA844A8597E037
:10DB7000FFFFE7802076AA894A8597E0FFFFE780CC
:10DB80006075A1659385C5022A89130544FC97C079
:10DB9000FFFFE780A07F268597C0FFFFE780E07347
:10DBA000854511C94A86CE8597C0FFFFE780606D25
:10DBB000AA8B21E98945130544FC97E0FFFFE78024
:10DBC000A061A685130544FC97E0FFFFE780C062D3
:10DBD000CE85130544FC97E0FFFFE780E061CA852E
:10DBE000130544FC97E0FFFFE78000610147814691
:10DBF000130644FCD2855A8597D0FFFFE780609ECC
:10DC0000B9B78145130544FC97E0FFFFE780C05C8E
:10DC1000A685130544FC97E0FFFFE780E05DCE8515
:10DC2000130544FC97E0FFFFE780005DCA851305FC
:10DC300044FC97E0FFFFE780205C814497D0FFFF22
:10DC4000E780006AE3D4A4FA83A70B0113971400BA
:10DC5000BA9783D5070099C5130544FC97E0FFFFE9
:10DC6000E78080598504D9BF797106D622D44AD07D
:10DC700000184ECE52CC56CA26D25AC8AE89328926
:10DC8000AA8A97D0FFFFE780A0650605690541993C
:10DC90000A8A3301A140232A24FC231C04FC97D0C8
:10DCA000FFFFE780E06383C7990006052D0593F722
:10DCB000F707231DA4FCA384F9004A85232E24FC26
:10DCC00097E0FFFFE780006193170501C187634F6D
:10DCD000F0005281130104FDB250225492540259B3
:10DCE000F249624AD24A424B45618280AA844A85FF
:10DCF00097E0FFFFE780005EA1659385A5022A8972
:10DD0000130544FD97C0FFFFE7804068268597C054
:10DD1000FFFFE780805C854509C9CA8597C0FFFF82
:10DD2000E78020592A8B29E18945130544FD97E0B6
:10DD3000FFFFE780604AA685130544FD97E0FFFFDB
:10DD4000E780804BCA85130544FD97E0FFFFE7801D
:10DD5000A04A01478146130644FDCE85568597D0DB
:10DD6000FFFFE7800088B5B78145130544FD97E0C4
:10DD7000FFFFE7806046A685130544FD97E0FFFF9F
:10DD8000E7808047CA85130544FD97E0FFFFE780E1
:10DD9000A046814497D0FFFFE7808054E3DBA4FADC
:10DDA00083270B0113971400BA9783D5070099C5F1
:10DDB000130544FD97E0FFFFE78000448504D9BFC9
:10DDC0001743FFFFE702233183474500404DD5EF5E
:10DDD000FD575DC48346940009476363D70A034631
:10DDE000B400854663EEC6088306E40063CA0608ED
:10DDF0005C45F9562390D7009787FF1F83C7071DFF
:10DE000099E3A304E4009787FF1F938767249C434B
:10DE100081E78947A306F4009787FF1F9387C7719F
:10DE20009C4381E789472306F4009705000093850A
:10DE30004506AA841305040197F00000E78020102E
:10DE4000FD57231AF40281471CDC01489787FF1F06
:10DE500023AA87169787FF1F93870717232E04038C
:10DE600004C0804397D0FFFFE780C051614633066E
:10DE7000C502814522859740FFFFE780C028814782
:10DE80003E851743FFFF67004327FD57D5BF174364
:10DE9000FFFFE70243242A840355450297600000F0
:10DEA000E780E01D19E5231E04001743FFFF67000C
:10DEB000C3248357E401F5DB930504FF17450100F4
:10DEC0001305057697E00000E780E014F9BF1743DB
:10DED000FFFFE70243202E89A16541119385E503E9
:10DEE0002A8436C432C6BE843AC297C0FFFFE78098
:10DEF000E04912472285BA8597E0FFFFE780C02DF1
:10DF000032462285B28597E0FFFFE780E02EA246E9
:10DF10002285B68597E0FFFFE780002E63030902A4
:10DF20009145228597E0FFFFE780C0241146A68532
:10DF300097100100E78020E241011743FFFF6700CF
:10DF4000C31B8945228597E0FFFFE780A02283C796
:10DF500004002300F50083C71400A300F500E9BF07
:10DF60001743FFFFE702231783C79500444D05477A
:10DF700093F7F707A384F5001C42411183C70700FC
:10DF80006367F7062E842A89B1C003C7D400630FE4
:10DF9000F7021787FF1F1307A70B184305C3A386B4
:10DFA000F40097A00000E780404A83C7D40099E7B7
:10DFB00041657D1597400000E780403083D72403FA
:10DFC000918B89C797E00000E780C0134A85A2853E
:10DFD00097F0FFFFE7808010A167C10748003EC4AB
:10DFE0002302010002C697F0FFFFE7808005410190
:10DFF0001743FFFF670063101743FFFFE702A30DFE
:10E0000003D745008D47AA8441112E8432892E857D
:10E0100063E3E70297E0FFFFE780C02BAA852300B8
:10E020000900268597C0FFFFE780A028410117431C
:10E03000FFFF6700830C97E0FFFFE780A0292AC657
:10E04000228597E0FFFFE780E028B24585472A86D2
:10E050002300F900268597C0FFFFE7808022F9B7EB
:10E06000397106DE22DC26DA80004ED652D456D232
:10E070004AD85AD05ECEAE89B284AA8A97D0FFFF22
:10E08000E780002506051305250241990A8A330118
:10E09000A140232224FC231404FC97D0FFFFE78037
:10E0A000202383C7990006054D0593F7F70723152D
:10E0B000A4FCA384F9002685232624FC97E0FFFF17
:10E0C000E780402193170501C1876340F002528128
:10E0D000130104FCF2506254D2544259B259225AEC
:10E0E000925A025BF24B21618280AA8B03AB04003F
:10E0F00097C0FFFFE780601E51E583D744000149C8
:10E100008544F11793B71700A301F4FC834734FC4F
:10E11000A165C9C79385E504130544FC97C0FFFFBB
:10E12000E780C026A685130544FC97E0FFFFE78043
:10E13000A00ADE85130544FC97E0FFFFE780C00BD3
:10E14000834734FC114691E30946DA85130544FC04
:10E1500097E0FFFFE78060058144630A0900416B97
:10E160007D1B97D0FFFFE780A01663CCA402014778
:10E170008146130644FCCE85568597C0FFFFE78095
:10E180004046B1B7A685130634FC97000000E7802F
:10E19000E0E6933415002A8986048DBF9385C50473
:10E1A000A5BF8327C90013971400BA9783D507002A
:10E1B00063886501130544FC97E0FFFFE780C00317
:10E1C000850445B71743FFFFE70263EE79711C1022
:10E1D0003EC4B7070F003EC61C103EC883C795005B
:10E1E000AA8A328593F7F707A384F500AE893284B3
:10E1F00097E0FFFFE780000E93170501C187635A80
:10E20000F0062A8A228597E0FFFFE780A00C2A8982
:10E210005285032B040097C0FFFFE780000C39ED07
:10E220008357440081440544F11793B71700A303B3
:10E23000F10083457100DA872287CA86528628005A
:10E2400097000000E780E0C8014781463000CE8596
:10E25000568597C0FFFFE780C038A1679387D70333
:10E2600048083ECC230A810026CE97F0FFFFE780C6
:10E2700040DD45611743FFFF6700E3E6A285130613
:10E28000710097000000E78060D7AA84094455D147
:10E290003544E30055FB4A8597F0FFFFE7800045D2
:10E2A0000D4441D9014497D0FFFFE7806002634DE0
:10E2B000A400C16B0144FD1B97D0FFFFE780400124
:10E2C000634EA4001544B5B7DC4413171400BA9785
:10E2D00083D70700638327030504F1B7D844931756
:10E2E0001400BA9703D70700631B77012390270117
:10E2F000268597A00000E78080DB01441DBF050450
:10E3000065BF1743FFFFE70263DB83C79500411139
:10E310002A8A93F7F707A384F50032852E89328481
:10E3200097E0FFFFE78000FB93170501C187635368
:10E33000F006AA89228597E0FFFFE780A0F9231164
:10E34000A1004E85832A040097C0FFFFE780E0F814
:10E3500039E58357440085440144F11793B717000A
:10E36000A300F1000348110003572100D68752850E
:10E37000CE862686CA8597F0FFFFE7806006A167F4
:10E38000F10748003EC42302910022C697F0FFFF28
:10E39000E78020CB41011743FFFF670063D5A285CB
:10E3A0001306110097000000E78040C52A848944C5
:10E3B00055D98357210011678544BA97C207116761
:10E3C000C1831307F7EFE36FF7F89787FF1F938772
:10E3D00067DE9C4381CB85451305210097500000E3
:10E3E000E7802075835521002285814497C0FFFF77
:10E3F000E78040E525D923100500228597A000007D
:10E40000E78040CD85B71743FFFFE70243CA83C7C4
:10E41000950041112A8B93F7F707A384F500328505
:10E420002E8A328497E0FFFFE780C0EA9317050148
:10E43000C1876351F006AA8A228597E0FFFFE78033
:10E4400060E92A895685832B040097C0FFFFE78087
:10E45000C0E831E58357440081440544F11793B780
:10E460001700A301F10003483100DE875A854A876F
:10E47000D6862286D28597F0FFFFE78060F6A167F7
:10E48000ED0748003EC42302810026C697F0FFFF37
:10E49000E78020BB41011743FFFF6700C3C4A2858B
:10E4A0001306310097000000E78040B5AA840944B4
:10E4B0005DD99167CA97C2071167C1831307F7EF48
:10E4C0000544E362F7FACA8597C0FFFFE78080D76B
:10E4D000014451F9814997D0FFFFE78060E063DB99
:10E4E000A900984893971900BA9703D7070005EF3A
:10E4F0002390270197D0FFFFE78080DE1544E38457
:10E50000A9F6268597A00000E780C0BC9787FF1F6B
:10E51000938747CA9C430144B9D74A859750000066
:10E52000E780C05889B785097DB71743FFFFE70229
:10E53000E3B879713E847C083EC82E8AB707140080
:10E54000A1653ECAE5057C08AA89080836C4428947
:10E5500032C6BA8AC6843ECC97C0FFFFE78000E38C
:10E56000CA85080897E0FFFFE78000C73246080821
:10E57000B28597E0FFFFE78020C8A246630A09043E
:10E580009D45080897E0FFFFE780C0BE1D46814516
:10E590009740FFFFE78020B763890A089145080884
:10E5A00097E0FFFFE78000BD1146A68597000100B8
:10E5B000E780607A100801478146D2854E8597C072
:10E5C000FFFFE780000245611743FFFF670043B28A
:10E5D000B685080897E0FFFFE78000C21C400808E6
:10E5E000D8439355C701858912075183B205D98D48
:10E5F00097E0FFFFE78040C01C40080883C5870004
:10E6000097E0FFFFE78040BD1C40080883C5A700D6
:10E6100097E0FFFFE78040BC1C40080883C59700D7
:10E6200097E0FFFFE78040BB85BF8945080897E07A
:10E63000FFFFE78020B483C704002300F50083C7F1
:10E640001400A300F500BDB71743FFFFE70203A7BF
:10E6500083C795004111AA8993F7F707A384F500B2
:10E660003285AE84328497E0FFFFE780A0C693171F
:10E670000501C187635DF0042A89032A040097C05D
:10E68000FFFFE78080C519E9835744000548F1176B
:10E6900093B71700A307F100814631A81306F100D4
:10E6A000A28597000000E78060951DC51C459DC7A9
:10E6B00083D6470001480347F10093078500D288BD
:10E6C0004A86A6854E8597000000E78040E6410116
:10E6D0001743FFFF6700C3A109487DBF1D486DBFF9
:10E6E0001743FFFFE702839D65715C083EC4B707CF
:10E6F0007B013EC65C083EC883C795002A8A3285E6
:10E7000093F7F707A384F500AE8997E0FFFFE78052
:10E7100040BA8357E100E1C78945280097C0FFFF51
:10E72000E780C0C68145280097E0FFFFE780C0AAC8
:10E7300097C0FFFFE780A0CC9787FF1F9387C7DFB5
:10E740009C431784FF1F03446488AA8433348000E9
:10E7500099C3136424009787FF1F9387678F9C4397
:10E7600099C3136444009787FF1F9387A7A49C4312
:10E7700099C31364840083D504002800014997E0FD
:10E78000FFFFE78060A783D52400280097E0FFFF04
:10E79000E78080A683D54400280097E0FFFFE7804C
:10E7A000A0A597D0FFFFE780A0AE93150501C1811A
:10E7B000280097E0FFFFE78020A4A285280097E0CB
:10E7C000FFFFE78060A39C446360F9020147814634
:10E7D0003000CE85528597C0FFFFE78080E0596109
:10E7E0001743FFFF6700C390DC441314490028005F
:10E7F0003E9497E0FFFFE78060968347440003471D
:10E80000540089070607BA978607E36AF5FC835523
:10E8100024002800814A97E0FFFFE780E09D8345C0
:10E820004400280097E0FFFFE780009B83455400E9
:10E83000280097E0FFFFE780209A8347440063C9E0
:10E84000FA00814A8347540063C1FA020509A5BF53
:10E850001C4413975A002800BA9783D50700850AED
:10E8600097E0FFFFE7804099C9BF032BC40093974F
:10E870005A0028003E9B83552B00850A97E0FFFF36
:10E88000E780809783550B00280097E0FFFFE78023
:10E89000A0964DBF1743FFFFE702E3835C4993E770
:10E8A00017005CC997A00000E78020B61743FFFF60
:10E8B0006700A3841743FFFFE702E3812E848145AD
:10E8C00097F0FFFFE780C0E705C583570500FD17F8
:10E8D0002310F50009C4835725002310F400970086
:10E8E0000000E78060FB01451743FFFF6700E380FE
:10E8F00031457DD823100400C5BF1733FFFFE70261
:10E90000E37B83C7950041112A8A93F7F707A38415
:10E91000F50032852E89328497E0FFFFE780809BE7
:10E9200093170501C1876356F006AA89C145228560
:10E9300097E0FFFFE780A0802A8B4E85832A0400A2
:10E9400097C0FFFFE780609931E9835744002311A6
:10E9500001000544F11793B71700A300F1008144AB
:10E960000348110003572100D6875285CE862286A0
:10E97000CA8597F0FFFFE780A0A6A16793871702DB
:10E9800048003EC42302810026C697E0FFFFE780CF
:10E99000406B41011733FFFF6700837513061100B9
:10E9A000A28597F0FFFFE7806065AA8409E523113F
:10E9B0000100094475B7930521005A8597000000AE
:10E9C000E78080EF835721002A84D9DB9777FF1FE8
:10E9D0009387477E9C4381CB854513052100975043
:10E9E0000000E7800015835521002685314497C03B
:10E9F000FFFFE78020852DD5231005002685979001
:10EA00000000E780206D0144A1BF1733FFFFE7023C
:10EA1000836C41112E896C00AA8402C697F0FFFF17
:10EA2000E78000D20DC10357050005072310E5005C
:10EA300097000000E78040E681473E85410117339B
:10EA4000FFFF6700836B3247954765DBCA852685E4
:10EA500097300000E780400DC147E34005FE324497
:10EA6000854741462310F40083570900A685130506
:10EA700044002311F40097000100E780C02D228597
:10EA800045BF1733FFFFE702636383C7950041115A
:10EA9000AA8A93F7F707A384F5003285AE893284FA
:10EAA00097E0FFFFE780008393170501C187635656
:10EAB000F0062A8AC145228597D0FFFFE7802068AB
:10EAC000AA845285032B040097C0FFFFE780E080F3
:10EAD00031E983574400231101008544F11793B7AE
:10EAE0001700A300F100014403481100035721005F
:10EAF000DA875685D2862686CE8597F0FFFFE78097
:10EB0000208EA1679387070248003EC4230291002C
:10EB100022C697E0FFFFE780C05241011733FFFF95
:10EB20006700035DA2851306110097F0FFFFE780E1
:10EB3000E04C2A8409E523110100894475B7268534
:10EB40009305210097000000E78060ECAA8449FD4E
:10EB500083552100228597B0FFFFE780A06E49F51D
:10EB6000014997C0FFFFE780A077635DA9001848BF
:10EB700093171900BA9703D707000DEF0357210029
:10EB80002390E70097C0FFFFE780807563062503A9
:10EB90009777FF1F938707629C4399C7035521000E
:10EBA00097500000E78080F0228597900000E78072
:10EBB00060521DBF050975B795443DB705C1930760
:10EBC000F00F630FF500C547630CF5009307F5FFE1
:10EBD00005453315F500420541818280014582805B
:10EBE00041657D158280B9E91733FFFFE702A34E27
:10EBF00003450603328497000000E78060FC93051C
:10EC0000803EB305B502C205C18181CD0357E40240
:10EC1000854763F8E7001305040197E00000E780EB
:10EC200020428357E40241677D176385E700FD17A3
:10EC30002317F4021733FFFF6700234C828017333A
:10EC4000FFFFE702C346004283C79500444D0349D6
:10EC5000140093F7F707A384F50083470400220903
:10EC600011673369F900A167B347F90041112A8B95
:10EC7000AE8A63ECE70E834724001307C00EB91772
:10EC800093F7F70F6373F71003473400C14763EE40
:10EC9000E70E834744001307E00793C70708637133
:10ECA000F70C8349840083477400A209B3E9F90093
:10ECB000856763F7F90A034A6400834754004E8569
:10ECC000220A336AFA0097500000E780403B61C196
:10ECD00023962403834B3400137AFA00239A3403D7
:10ECE000238874032399440393890401631C090056
:10ECF00023A60402239804024E8597E00000E780D3
:10ED000060363DA0034924004A8597000000E78053
:10ED100020EB2397A402834744004E85A388F40286
:10ED2000E38D0BFCE30B09FC97E00000E780202F4C
:10ED300097900000E780007381460146D6855A858A
:10ED400097E0FFFFE7800058A167938797033EC4D1
:10ED500023020100480002C697E0FFFFE780602E13
:10ED600041011733FFFF670003388544A2862686DA
:10ED7000D6855A8597E0FFFFE780C054A167938747
:10ED800097033EC423029100F1B7BD44C5B7914437
:10ED9000F1BF1733FFFFE702633201111C08404D3A
:10EDA0003EC2B7070F003EC41C083EC62A89AE8982
:10EDB00097C0FFFFE780A0DA585C1C5C6346B70E83
:10EDC0006394E50063E2A70E3385A740B3B7A700BD
:10EDD000B305B7401306803E81469D8D9700010024
:10EDE000E78080B793140501C180A1659385C503B1
:10EDF000480097B0FFFFE78060598145480097D0F1
:10EE0000FFFFE780603D83550404480097D0FFFF73
:10EE1000E780803E83552404480097D0FFFFE780B9
:10EE2000A03D814589CCC167FD179305F00F63882C
:10EE3000F400268597500000E780E0E0AA854800AE
:10EE400097D0FFFFE780403903554404814501CD49
:10EE5000C167FD179305F00F6307F5009750000099
:10EE6000E78060DEAA85480097D0FFFFE780C036C4
:10EE700083456404480097D0FFFFE780E035834571
:10EE80007404480097D0FFFFE78000355000014729
:10EE90008146CE854A8597B0FFFFE7808074056183
:10EEA0001733FFFF6700C324814481B71733FFFF87
:10EEB000E702632283C7950093F7F707A384F50061
:10EEC00097000000E78020ED1733FFFF6700E32283
:10EED0001733FFFFE702831E83C795004111404DA2
:10EEE00093F7F707A384F5002A8A3285B284AE89A6
:10EEF00097D0FFFFE780003E2A8B268597D0FFFF43
:10EF0000E780403D2A89268597D0FFFFE780603A59
:10EF100093170B0163CA0702E177CA97C207C1833F
:10EF2000116763E3E70293070910C207C183130760
:10EF3000B00F637BF70093170901C187AA8A634A60
:10EF4000F000C54763FE570141011733FFFF67001B
:10EF5000231A97B0FFFFE780C028E31725FFD5B736
:10EF600063080B0263060902814463890A02B7073A
:10EF70007F0023106405231124057CC0568597006B
:10EF80000000E780E0C39304803EB304950239A0FB
:10EF9000B7077F00232004047CC081440355240468
:10EFA00097E00000E780A0A3A1C497C0FFFFE7801F
:10EFB00000BB269593D7F44133379500AE97BA97A7
:10EFC00008DC5CDCCE85528597000000E780A0DC81
:10EFD00099E023220404A1679387B70348003EC445
:10EFE0002302010002C697E0FFFFE7808005A9BF6A
:10EFF000814701481CDC232E0403E9B71733FFFFC8
:10F00000E702630D97C0FFFFE780C037E147330594
:10F01000F502914597500000E78000C5E55711C5FE
:10F020009777FF1F23A2A7FA81473E851733FFFF7B
:10F030006700A30C85471777FF1F2309F7F8828025
:10F040001733FFFFE70223099777FF1F938787F79F
:10F0500080433DC0835704046390A706835724046C
:10F06000639CB7043689B28497C0FFFFE78020AF66
:10F070005C5C63C3B7046395B7001C5C63EEA702D6
:10F080008347640463F3F400A6872303F4048347EF
:10F09000740463F39700A687A303F404835744041E
:10F0A00041677D176385E70085072312F4043C441C
:10F0B00081C7CA85268582971733FFFF6700E30360
:10F0C0009777FF1F938707F09C43014599C303C5BA
:10F0D000870082801733FFFFE702E3FF0111B707C4
:10F0E00007003EC683C79500584D0AC493F7F7073B
:10F0F0000AC8A384F5002A89AE8411CB1C4283C7B9
:10F1000007002304F70097900000E7800034216493
:10F1100093055402280097B0FFFFE780202797004F
:10F120000000E78020FAAA85280097D0FFFFE7803B
:10F13000A00A300001478146A6854A8597B0FFFFA7
:10F14000E780204A13044402480822CC230A010025
:10F1500002CE97E0FFFFE780C0EE05611733FFFFA7
:10F160006700A3F91733FFFFE702E3F601117C0004
:10F170003ECAB70707003ECC7C003ECE83C7950051
:10F180002E84AA8493F7F707A384F500A1659385DD
:10F190005502480897B0FFFFE780401F9700000026
:10F1A000E78040F2AA85480897D0FFFFE780C002B9
:10F1B000500801478146A285268597B0FFFFE7806A
:10F1C000404205611733FFFF670023F39777FF1F66
:10F1D000938747DF9C43094599C303C59700828005
:10F1E0009777FF1F938707DE9C43094599C303C5A3
:10F1F000D70082809777FF1F9387C7DC9C43014528
:10F2000099C303C5A70082801733FFFFE70203EB12
:10F210000111B70708003EC683C79500404D0AC4D8
:10F2200093F7F7070AC8A384F5002A89AE8429C496
:10F230001442854703C7060063E0E70A834794004A
:10F24000094681496380C702B307F740A304E4007D
:10F25000B339F00083C716002305F400979000002F
:10F26000E780A01E03572403058B19C76386090096
:10F2700097D00000E78000E921649305840228000C
:10F2800097B0FFFFE780801097000000E78040F410
:10F29000AA85280097D0FFFFE78000F497000000C0
:10F2A000E78080F5AA85280097D0FFFFE780C0F2AD
:10F2B000014781463000A6854A8597B0FFFFE78069
:10F2C000403213047402480822CC230A010002CE03
:10F2D00097E0FFFFE780E0D605611733FFFF670087
:10F2E00023E11733FFFFE70203DF01117C003ECA71
:10F2F000B70708003ECC7C003ECE83C795002E8425
:10F30000AA8493F7F707A384F500A1659385850286
:10F31000480897B0FFFFE780600797000000E7808C
:10F3200020EBAA85480897D0FFFFE780E0EA970026
:10F330000000E78060ECAA85480897D0FFFFE780CF
:10F34000A0E9500801478146A285268597B0FFFFB6
:10F35000E780202905611733FFFF670003DA9777FD
:10F36000FF1F938727C69C43014599C303C5B70078
:10F3700082801733FFFFE70203D60111B7070700AA
:10F380003EC683C79500404D0AC493F7F7070AC8E5
:10F39000A384F5002A89AE8405C81C42054783C7AB
:10F3A00007006368F7060347B400630FF700A3057F
:10F3B000F40097900000E78040098347B400B9CF7C
:10F3C00097D0FFFFE78040BE21649305B40028007A
:10F3D00097B0FFFFE78080FB97000000E78060F8B0
:10F3E000AA85280097D0FFFFE78000DF014781460C
:10F3F0003000A6854A8597B0FFFFE780801E29046C
:10F40000480822CC230A010002CE97E0FFFFE780E4
:10F4100040C305611733FFFF670023CE97D0FFFF7E
:10F42000E78020BF55B71733FFFFE702C3CA0111BA
:10F430007C003ECAB70707003ECC7C003ECE83C7A7
:10F4400095002E84AA8493F7F707A384F500A1659D
:10F45000AD05480897B0FFFFE78040F39700000034
:10F46000E78020F0AA85480897D0FFFFE780C0D644
:10F47000500801478146A285268597B0FFFFE780A7
:10F48000401605611733FFFF670023C79777FF1FFB
:10F49000938747B39C43094599C303C5C70082803E
:10F4A0001733FFFFE70223C301117C00AE843ECA7D
:10F4B000A165B70707002A843ECCD1057C00480827
:10F4C0003ECE97B0FFFFE78060EC97000000E7803A
:10F4D00020FCAA85480897D0FFFFE780E0CF5008BE
:10F4E00001478146A685228597B0FFFFE780600F20
:10F4F00005611733FFFF670043C01733FFFFE702C3
:10F5000083BD83C7950093F7F707A384F5009700A1
:10F510000000E78020F91733FFFF670003BE1733B1
:10F52000FFFFE702A3B983C795000329C501411175
:10F5300093F7F707A384F5001C4283C907008547AA
:10F5400063E637079777FF1F938707FF9C432E8457
:10F55000AA8485CF97000000E78080F3894763067F
:10F56000F502630409028347C90063803703230659
:10F57000390197900000E78040ED83572903898B7C
:10F5800089C797D00000E780E0B72685A28597005D
:10F590000000E78020F1A167CD0748003EC42302A8
:10F5A000010002C697E0FFFFE780A0A941011733E1
:10F5B000FFFF6700E3B39777FF1F9387A7A09C43E4
:10F5C0001D4599C303C5E70082801733FFFFE7029B
:10F5D00083B00111B70707003EC683C79500584D99
:10F5E0000AC493F7F7070AC8A384F5002A89AE84F2
:10F5F00015C71C4283C7070093968701E18663C441
:10F60000060685466381D7068346E7006388F600D1
:10F610002307F70097900000E78020E3216493051B
:10F62000E400280097B0FFFFE78040D69700000075
:10F63000E780A0F8AA85280097D0FFFFE780C0B92F
:10F64000014781463000A6854A8597B0FFFFE780D5
:10F6500040F93504480822CC230A010002CE97E085
:10F66000FFFFE780009E05611733FFFF6700E3A8F7
:10F670001733FFFFE70223A601117C003ECAB7073C
:10F6800007003ECC7C003ECE83C795002E84AA8422
:10F6900093F7F707A384F500A165B905480897B06B
:10F6A000FFFFE780A0CE97000000E78000F1AA8569
:10F6B000480897D0FFFFE78020B2500801478146F5
:10F6C000A285268597B0FFFFE780A0F1056117337B
:10F6D000FFFF670083A21733FFFFE702239EAA8480
:10F6E00001441779FF1F1309298EE14997C0FFFFD5
:10F6F000E78040C96344A400014519A833053403D9
:10F70000832709003E9583572500639797001105CD
:10F710001733FFFF6700C39D0504C9BF032E850093
:10F72000630A0E121773FF1F1303C3A803230300FA
:10F730006315030029436390061203234E016315EA
:10F7400003001D43639907101733FFFFE702239659
:10F75000C689428A3E89BA8AB684328BAE8B2A84A5
:10F76000B5E103554E0019E501431A851733FFFF34
:10F7700067006397A167A98F116763FBE700970094
:10F780000000E78080F5814597F0FFFFE780C01219
:10F790000844B70700E05841F98F18455CC1B70726
:10F7A000001FF98F1CC55C4991C7610597E00000F7
:10F7B000E780408BE38A09FA228597900000E78072
:10F7C00060C65DB7328597C00000E78040430D43B7
:10F7D00049DD1C44116703D54700A167A98F63FB6E
:10F7E000E70097000000E78040EF814597F0FFFFBA
:10F7F000E780800C0323840093164B01D18283475A
:10F80000B300035663008588FD8BA305F300FD77E5
:10F810007D8E558EFD76FD16B204F18E8327430151
:10F82000C58E231273012313D30023045301230530
:10F830002301A3044301BDDF228597B0FFFFE780CA
:10F8400020CDAA850844B5D1610597D00000E78096
:10F85000207F8DB71D431A8582801733FFFFE70293
:10F86000E3850569AA84AE89328A0144FD5A7D196F
:10F8700097C0FFFFE780C0A56347A4000145173389
:10F88000FFFF6700E386D84493171400BA9703D7A5
:10F890000700631F37032390570163070A0026857B
:10F8A00097900000E780A0809C449DC383D76700A9
:10F8B000B3F72701639E3701D2880148814701478A
:10F8C000814601468145268597000000E78040E596
:10F8D000050479BF1723FFFFE702437E79711C10EF
:10F8E0003EC4B7070F003EC61C103EC883C7950034
:10F8F000AA8A328593F7F707A384F5002E8932840C
:10F9000097D0FFFFE780009D93170501C187635AD9
:10F91000F006AA89228597D0FFFFE780A09B2A8A5C
:10F920004E85032B040097B0FFFFE780009B39ED65
:10F930008357440081440544F11793B71700A3038C
:10F94000F10083457100DA872287D2864E8628002F
:10F9500097E0FFFFE780E057014781463000CA8506
:10F96000568597B0FFFFE780C0C7A1679387F7036D
:10F9700048083ECC230A810026CE97D0FFFFE780BF
:10F98000406C45611723FFFF67008376A28513064D
:10F99000710097E0FFFFE7806066AA84094455D1B3
:10F9A000528597E0FFFFE78060D40D4459D90546A2
:10F9B000D285268597000000E78060EA2A8451B747
:10F9C0001723FFFFE7022371835507000346270033
:10F9D00041112A842E8532C62EC497E0FFFFE780AE
:10F9E000E0D001C93246A245228597000000E78099
:10F9F00000E741011723FFFF670023701723FFFF74
:10FA0000E702E36A83C795004111AA8A93F7F707D3
:10FA1000A384F5003285AE89328497D0FFFFE7805A
:10FA2000608B93170501C1876357F00AC1452A8A85
:10FA3000228597C0FFFFE78080702A8D228597D0AE
:10FA4000FFFFE78020892A89228597D0FFFFE78082
:10FA50004086930705F893F7F70F1307E007AA8B83
:10FA6000637BF706228597D0FFFFE78080842A8C8E
:10FA7000228597D0FFFFE780C083AA8C5285032B95
:10FA8000040097B0FFFFE780408539E983574400C1
:10FA9000231101008144F11793B71700A300F1006F
:10FAA000054403471100835621009387840056853F
:10FAB000DA8822885286CE8597F0FFFFE78020A75C
:10FAC000A167E90748003EC42302810026C697D0FB
:10FAD000FFFFE780005741011723FFFF6700A36086
:10FAE00013061100A28597E0FFFFE7802051AA844A
:10FAF00009E52311010009446DB7930521006A85CA
:10FB000097F0FFFFE780A0F02A8441FD8355210094
:10FB10009356C9001316490185486688E2875E87B7
:10FB2000858A5182268597000000E78060BF2A847D
:10FB30008DBF1723FFFFE702835783C7950041114D
:10FB40002A8B93F7F707A384F5003285AE893284B8
:10FB500097C0FFFFE780007893170501C1876352C4
:10FB6000F00A2A8A228597C0FFFFE780A076AA8A3A
:10FB7000228597C0FFFFE780E0752A89228597C01C
:10FB8000FFFFE7800073930705F893F7F70F13075C
:10FB9000E0072A8C6377F706228597C0FFFFE7808E
:10FBA0004071AA8C228597C0FFFFE78080702A8D64
:10FBB0005285832B040097A0FFFFE780007239E590
:10FBC0008357440085440144F11793B71700A301FC
:10FBD000F10003473100930784005A85DE882688A8
:10FBE000D6865286CE8597F0FFFFE78040948D47FA
:10FBF00048003EC42302910022C697D0FFFFE78051
:10FC0000404441011723FFFF6700E34DA28513061F
:10FC1000310097E0FFFFE780603E2A84894455D990
:10FC20009356C9001316490185486A88E68762879A
:10FC3000858A5182D68597000000E78060AEAA844D
:10FC400049BF1723FFFFE70263472A898144014424
:10FC5000617A916A176BFF1F130BCB5597B0FFFFAB
:10FC6000E780006863C7A40022851723FFFF6700B1
:10FC700023488327090093991400CE9703D50700E2
:10FC800033074501420741836364570305C10327D6
:10FC90000B0019C785453E8597400000E78060E965
:10FCA000832709000504CE972390070085047DB7BC
:10FCB00097000000E78060A2832709000504CE9723
:10FCC0002390070065D5814597F0FFFFE780C0BE10
:10FCD000F1BF1723FFFFE702633E83C79500411181
:10FCE0002A8A93F7F707A384F50032852E89328498
:10FCF00097C0FFFFE780005E93170501C187635A35
:10FD0000F004AA89832A040097A0FFFFE780E05C43
:10FD100031E58357440085440144F11793B7170038
:10FD2000A301F10003483100D68752850147CE86F2
:10FD30002686CA8597D0FFFFE780806AA167F5070E
:10FD400048003EC42302910022C697D0FFFFE780FF
:10FD5000402F41011723FFFF67008339A285130657
:10FD6000310097E0FFFFE78060292A8489445DD94C
:10FD70009767FF1F938707449C4381CF044997B03F
:10FD8000FFFFE780E055AA85268597400000E780C1
:10FD900040DA1305040197000000E780C0EA2285DD
:10FDA00097800000E78000338144ADBF1723FFFF39
:10FDB000E702E32F83C795004111AA8A93F7F7075B
:10FDC000A384F5003285AE8932842311010097C0E7
:10FDD000FFFFE780205093170501C1876354F006A9
:10FDE0002A8AC145228597C0FFFFE7804035AA8B4C
:10FDF0005285032B040097A0FFFFE780004E21E906
:10FE00008357440085440144F11793B71700A300BA
:10FE1000F1000348110003572100DA875685D28686
:10FE20002686CE8597D0FFFFE780805BA16793870A
:10FE3000270248003EC42302910022C697D0FFFF4C
:10FE4000E780202041011723FFFF6700C329A28517
:10FE50001306110097E0FFFFE780401A2A848944C7
:10FE60004DD99767FF1F9387E73498433E8901CFA9
:10FE7000044997B0FFFFE780A046AA8526859740F2
:10FE80000000E78000CB1305040197000000E78025
:10FE900080DB97B0FFFFE780A04495443DD99305F0
:10FEA00021005E8597F0FFFFE78060B6AA8435F1F8
:10FEB0001C480357210022852390E700978000000B
:10FEC000E780402183270900A9D7035521009740E7
:10FED0000000E780A0BD35BF1723FFFFE702231D09
:10FEE00083C795004111AA8A93F7F707A384F50009
:10FEF0003285AE89328497C0FFFFE780A03D93171B
:10FF00000501C1876351F0062A8A228597C0FFFF49
:10FF1000E780403C2A895285032B040097A0FFFF0D
:10FF2000E780A03B31E58357440085440144F11745
:10FF300093B71700A301F10003483100DA87568513
:10FF40004A87D2862686CE8597D0FFFFE780404934
:10FF5000A167F90748003EC42302910022C697D04A
:10FF6000FFFFE780000E41011723FFFF6700A31783
:10FF7000A2851306310097E0FFFFE78020082A845E
:10FF800089445DD99167CA97C2071167C183130776
:10FF9000F7EF8544E362F7FA9767FF1F938787219E
:10FFA0009843BE8B01CF044997B0FFFFE7804033F1
:10FFB000AA85268597400000E780A0B713050401B5
:10FFC00097000000E78020C897B0FFFFE78040312E
:10FFD00095443DD11C482285814423902701978078
:10FFE0000000E780200F83A70B00B9D74A85974010
:10FFF0000000E780A0AB89B71723FFFFE702A30D3E
:020000040001F9
:100000002A844105B28497000000E780C0C311C56F
:10001000228597800000E780E00B81460146A68597
:10002000228597800000E780C04E1C4C89C7DC47C2
:1000300099C3228582971723FFFF6700030C9767F8
:10004000FF1F938727F89C43014599C31385070138
:1000500082809767FF1F9387E7F688438280172384
:10006000FFFFE70243079317C600DD8DC20541116C
:10007000C1812A8432C697C0FFFFE780E01732466D
:10008000228511829375F60F97C0FFFFE780C01499
:1000900041011723FFFF670043061723FFFFE70215
:1000A000E30179713C083ED2B7070C003ED43C080E
:1000B0003ED683C79500AE842A8993F7F707A384B9
:1000C000F500A16593853504481097A0FFFFE780F0
:1000D000E02BC165FD150144176AFF1F130A0A0FC3
:1000E000930A400EAE892E8B2EC697B0FFFFE78095
:1000F00020224205931704014181C183B24563E97F
:10010000A702C167FD176387F500481097C0FFFF7E
:10011000E780800E501001478146A6854A8597A04A
:10012000FFFFE780004C45611723FFFF670043FC9A
:100130003307540383270A0BBA9703D6C701630A10
:100140003601638A3501481097000000E78060F1AE
:10015000DA85050451BFB285EDBF1723FFFFE70223
:1001600003F579717C083EC8B70711003ECA7C08C8
:100170003ECC83C79500AA89328593F7F707A384FD
:10018000F5002E8997C0FFFFE780C014856763786C
:10019000F504A165AA848905080897A0FFFFE780F8
:1001A000E01E268597400000E78060ED13341500BF
:1001B0000A04A285080897C0FFFFE780E001A68532
:1001C000080897C0FFFFE780200325CC0147814640
:1001D0001008CA854E8597A0FFFFE78080404561E3
:1001E0001723FFFF670023F0B30754030327CA0A4E
:1001F000BA9703D70700631C970003D627006380D4
:100200006505080897000000E780A0E5DE85050485
:100210002EC697B0FFFFE780A01042059317040198
:100220004181C183B245E3E1A7FCC167FD17E38FBC
:10023000F5F8080897C0FFFFE78000FC41BFB285D2
:10024000F9B7C165FD150144176AFF1F130A0AF8C3
:10025000930A80022E8BAE8B65BF1723FFFFE70248
:1002600083E718418347170083460700A207D58F0D
:10027000D207D1832390F500834727000347170057
:100280008D45A207D98F91832310F60097C0FFFFF9
:10029000E780A0E91723FFFF670023E61723FFFF8E
:1002A000E702C3E1C16401441769FF1F130909F2A2
:1002B00093098002FD1497B0FFFFE7806006634753
:1002C000A40001451723FFFF670083E233053403D1
:1002D0008327C90A3E9583570500E38597FE0504E9
:1002E000D9BF1723FFFFE70263DD2A8AAE89B284F4
:1002F000B68A97400000E78080D819E591473E858F
:100300001723FFFF6700C3DE2A894E8597C00000D0
:10031000E780E08E2A84638E0A048D476DD10357EF
:100320000500C547E31D47FD0347F9018546AD4775
:10033000E317D7FC8347450081CF4146A6855D057D
:1003400097F00000E780C09E814755D9AD4745BF73
:10035000130965012302E500CA8526859710000070
:10036000E780606231C1A547E38B0AF823020400ED
:1003700079B705C183570500E39247F94146A68541
:10038000190597F00000E780A09A81472DD9994779
:10039000BDB74E8597000000E78080F02A8495471E
:1003A00039DD130955004DBF4146A6852310440190
:1003B000231134011305190097F00000E780A0997C
:1003C000228597800000E780A0EA81470DBF1723B0
:1003D000FFFFE70243D079717C003ECCB7070A00EB
:1003E0003ECE7C003ED083C79500B2842E8493F726
:1003F000F707A384F5001306A1002A892C0026859F
:1004000097000000E780A0E5A16528088D0597A06A
:10041000FFFFE780A0F790408355A10003558100BE
:10042000854697000000E78000ECAA84AA8528088A
:1004300097C0FFFFE78040DA0356A1008355810093
:10044000280897000000E780C0C1300801478146B6
:10045000A2854A8597A0FFFFE780A018854748102E
:100460003ED42302910202D697D0FFFFE78060BD01
:1004700045611723FFFF670043C81723FFFFE7020B
:1004800083C579717C003ECCB7070A003ECE7C0064
:100490003ED083C79500B2842E8493F7F707A384D8
:1004A000F5001306A1002A892C002685970000007C
:1004B000E780E0DAA16528088D0597A0FFFFE780B7
:1004C000E0EC90408355A1000355810081469700E0
:1004D0000000E78040E1AA84AA85280897C0FFFFB2
:1004E000E78080CF0356A10083558100280897003C
:1004F0000000E78000B7300801478146A2854A85A1
:1005000097A0FFFFE780E00D48102302910202D47C
:1005100002D697D0FFFFE780C0B245611723FFFFE7
:100520006700A3BD1723FFFFE702E3BA97000000AF
:10053000E78060DB1723FFFF670023BC9767FF1F7F
:10054000938787A8884382801723FFFFE702A3B819
:10055000835725004111AE842A842307B10017F583
:10056000FFFF130525466C002316F10097A0FFFF3F
:10057000E780204991C4228597800000E780E0D67B
:10058000FD572310F4001306200281451305540083
:100590009720FFFFE78020B741011723FFFF670087
:1005A000C3B51723FFFFE70263B179717C003ECC2E
:1005B000B7070A003ECE7C003ED083C79500AA89CB
:1005C000AE8493F7F7073285A384F5001306A100E4
:1005D0002C0097000000E78080C80355810011447B
:1005E00097400000E780A0A915C50355A10001446C
:1005F00097B00000E780A06011CD03570500835736
:10060000810045446318F700854597000000E780A6
:10061000E0F30144216993053900280897A0FFFF02
:10062000E780C0D6A285280897C0FFFFE780C0BA40
:100630000356A10083558100280897000000E78039
:1006400040A2300801478146A6854E8597A0FFFF4E
:10065000E78020F948104AD42302810202D697D0BD
:10066000FFFFE780009E45611723FFFF670043A857
:100670001723FFFFE70283A49767FF1F93878794E1
:100680002A8488432E8915C5035745038357C4011F
:100690006311F7022326050223180502410597D0AE
:1006A0000000E780209C6306090097800000E78037
:1006B00060DB81449769FF1F938949B1130A800267
:1006C00097B0FFFFE780C0C563C4A4049767FF1F0E
:1006D000938707989C4399C70355C401972000004E
:1006E000E780C0BD63070900228597800000E7808E
:1006F000C0A01306400E814522859720FFFFE780AA
:1007000080A0FD57231EF4001723FFFF6700439EC0
:100710003385440383A7C90A3E95035705008357D1
:10072000C4016317F700CA8597000000E78000E264
:10073000850479B71723FFFFE702439883C7950025
:100740004111AA8993F7F707A384F5003285AE8497
:1007500097C0FFFFE78000B885676378F5042A89B2
:1007600097400000E780A091014401CD83D70400A9
:10077000314463882701854597000000E78080EFBA
:1007800001444E85A2864A86A68597D0FFFFE78062
:10079000A09CA1679387170448003EC423028100F0
:1007A00002C697D0FFFFE780C08941011723FFFFF2
:1007B000670003941723FFFFE70243909767FF1F2B
:1007C00093874780804329C4014597C00000E78094
:1007D000002181470148C1641CDC232E040323202F
:1007E00004041769FF1F1309699E01449309400E11
:1007F000FD1497B0FFFFE780A0B1634FA4008145CF
:1008000017F5FFFF1305857F97A0FFFFE780601FA7
:100810001723FFFF6700C38D330534038327090BBC
:100820003E958357C5016387970085459700000073
:10083000E78040E4050475BF9357050113D787008F
:10084000A380F50093170501C183A1832380E500F0
:100850002381F500A381A50082801723FFFFE70213
:1008600083872300050083C71500A300F50083C715
:1008700025002301F50083C73500A301F50083C7D8
:1008800045002302F50083C75500A302F50083C786
:10089000650093059500A30305002303F5002304D9
:1008A0000500328597000000E78040F91723FFFF1D
:1008B0006700A3841723FFFFE70243804111E95437
:1008C0000DCD85CD93F9C5FF2E842A89AA84338A5C
:1008D000A900B7EA040063189A020D88854411CC78
:1008E000B7E704009C5F82972AC622866C00330516
:1008F000390197E00000E780004626854101171383
:10090000FFFF6700E37E83A78A0391048297931712
:100910000501C183A183A38EF4FE93570501238FA4
:10092000F4FEA183238EA4FEA38FF4FE6DB763E6CD
:10093000D5021713FFFFE702037AB287411136860B
:10094000BE8536C697E00000E780E040B246410130
:1009500036851713FFFF6700437A8146368582800C
:10096000838705001387F5003D05FD8793F777081A
:10097000834607007D158606B58FA300F500630743
:10098000B7007D17834717009D83DDB7828017135B
:10099000FFFFE7024374B7E7040083A70709328724
:1009A0002A863A858297133515001713FFFF6700D3
:1009B000C37415C181478DC11713FFFFE702A371EF
:1009C000414697E00000E780003985473E851713D0
:1009D000FFFF6700837281473E8582801DCD17131C
:1009E000FFFFE702436F414681452A849710FFFFCE
:1009F000E780607141468145130504039710FFFFAE
:100A0000E78060700147C1672322040438C87CC8AE
:100A100005451713FFFF6700436E0145828081473C
:100A20003DCDB5CD1713FFFFE702E36AB2842E89EF
:100A30001306800581452A849710FFFFE780A06C8C
:100A4000CA8524C4268597000000E780C0F6414689
:100A5000814522859710FFFFE780E06A3044A28538
:100A6000228597000000E780C0F293040401A2856C
:100A7000268597000000E780E0EEA68513050402B6
:100A800097000000E78000EE228597000000E780D5
:100A900020F585473E851713FFFF670003663E85F7
:100AA00082801713FFFFE70263614111E9540DCD06
:100AB00085CD93F9C5FF2E842A89AA84338AA9009B
:100AC000B7EA0400639844030D88814411CCB7E76A
:100AD00004009C5F82972AC622866C003305390188
:100AE00097E00000E7802027268541011713FFFFCC
:100AF0006700036083A78A03910482979317050117
:100B0000C183A183A38EF4FE93570501238FF4FEC6
:100B1000A183238EA4FEA38FF4FE6DB765CD1713BA
:100B2000FFFFE702A359B28411E605451713FFFF43
:100B30006700035C2A842E890145EDD93C4878483A
:100B4000B3E6E700E5D69386F7FFB3B7F6007D1767
:100B5000032A4404BA9734C87CC863050A06C1490D
:100B600013050A03B38949412295637D3601B28694
:100B70002E86A68597000000E780A0DB7C40BE940F
:100B800064C065B7CE862E86CE8597000000E780CC
:100B900040DAC114D2944E9923220404A28793060A
:100BA000040103C7070003C607038507318FA38F1E
:100BB000E7FEE398F6FE3044A28522859700000008
:100BC000E78020DD2699C1493306994063EC9900FE
:100BD000A9DCA686A6851305040397000000E7801C
:100BE00040D579BF8147B306F4003307F6000347C9
:100BF000070083C5060085072D8F2380E600E39458
:100C000037FF3044A285228597000000E78060D836
:100C1000C1145DBF014582800DC11713FFFFE702BC
:100C2000834B1306800581459710FFFFE780A04D99
:100C300005451713FFFF6700434C0145828081473C
:100C400049C5C1C51713FFFFE702E348FC41414610
:100C50002E84AA846399C70413860501A28781465E
:100C6000C14503C7070003C507038507298F33055F
:100C7000D600034505008506298FA38FE7FEE39282
:100C8000B6FE3044A285268597000000E78060D03C
:100C9000228597000000E78060F885473E8517139E
:100CA000FFFF67008345138507031D8E814522954D
:100CB0009710FFFFE78020457C40130700F81306DC
:100CC0000402A2972388E70251BF3E858280171352
:100CD000FFFFE70243406D712E84B284AA85901015
:100CE0002800368997000000E780A0D309EDD5578A
:100CF00025A050400C40280097000000E78040E20B
:100D00007DD5FD142104F5F42C004A8597000000E0
:100D1000E78020F3814761DD3E8551611713FFFFB6
:100D20006700A33D1713FFFFE702E33A41112EC40A
:100D300032C62C00054697000000E78080F941018B
:100D40001713FFFF6700633B1713FFFFE702A3388A
:100D500001112A842EC602C802CA02CC02CE97E034
:100D60000000E780E032B2462A86A2850808970094
:100D70000000E78060FB1375F50F05611713FFFF97
:100D80006700A3371713FFFFE702E3347971B287D7
:100D90002A8421462308B10013051101BE853AC4F7
:100DA00036C697E00000E78000FBB246930591014C
:100DB000368597000000E78060A82285141035462C
:100DC0000C0897000000E78020F62A84224701E9FA
:100DD00021460C103A8597E00000E780C0F7228595
:100DE00045611713FFFF670043311713FFFFE70249
:100DF000832E7171AE84AA850A8532849700000023
:100E0000E78060BB11C90A86A6852285970000008D
:100E1000E78020B8814711E1C5473E854D61171332
:100E2000FFFF6700832D1713FFFFE702C3271D7124
:100E30002A8AB289BE8435468547130511012E8C56
:100E4000B68A3A8BC28C468D2308F10097E00000E9
:100E5000E78060F010100C085285231F01009700F6
:100E60000000E780C0F82A843DEDA1476313FD0828
:100E70009307900591E0E5473546E285130511019A
:100E800013990A012308F1001359090197E00000A2
:100E9000E78060EC1357890093978A00D98F9008F8
:100EA0000C085285231FF10097000000E78020F412
:100EB0002A8415E9A1E49387FA0091831379F90054
:100EC0003EC6631309004149668B8144C14B854D81
:100ED000B247639F970C6A868C0033855C0197E06C
:100EE0000000E78040E7228525611713FFFF6700B8
:100EF000431F93079004C9F0A547BDBF8347010571
:100F00000947C14B2308F10083471105A58FA308AA
:100F1000F10093872400814463E1FB040147140836
:100F20003386E6008C08B386E400BA95DA9683C669
:100F3000060083C505000507AD8E2300D600E390AB
:100F4000E7FE4147639CE70490080C085285970030
:100F50000000E780C0E925D181A0B3069B00BA87D5
:100F60001008B305F60090083E9603C50600034638
:100F7000060085078506298E2380C500E39277FF4A
:100F8000998F90080C085285BE9497000000E78066
:100F900000E68947014749D12A84B1B790083E96B7
:100FA000034606001408BE962380C600850759BF75
:100FB000B24785046387971481471808B306F70082
:100FC00098083E973386F90003470700034606005A
:100FD0008507318F2380E600E39177FF90080C08A6
:100FE000528597000000E78080E05DF53546E28598
:100FF000130511012308B10197E00000E780A0D597
:10100000139704014183939784002183D98F10188B
:101010000C085285231FF10097000000E78020DDB7
:1010200025FD814710183387F9003E9603470700D6
:1010300003460600B306FB008507318F2380E600D8
:10104000E39277FF65A81808B306F70098083E9763
:101050003386F90003470700034606008507318FF2
:101060002380E600E3E127FFCA87639E77099008A3
:101070000C08528597000000E78060D711FD81477A
:101080009800B306F700900818103E973E96034765
:101090000700034606008507318F2380E600E391B1
:1010A00077FF3546E285130511012308B10197E06A
:1010B0000000E78040CA139704014183939784009E
:1010C0002183D98F10180C085285231FF100970037
:1010D0000000E780C0D1E31105EC81471018338789
:1010E000F9003E960347070003460600B306FB00DF
:1010F0008507318F2380E600E3E227FFC109410B1A
:10110000C1BB814785B79408BE9683C60600180800
:101110003E972300D700850789BF638006321713E7
:10112000FFFFE70243F859712A84BE89B28B8547D5
:101130003546130511022E8B468C4289BA8A368AAF
:101140002300F10297E00000E780E0C010180C10C7
:1011500022852317010297000000E78040C9631829
:101160000512A147631FFC069307900563930900CE
:10117000E5473546DA851305110293140A01230069
:10118000F102C18097E00000E780E0BC93178A007D
:1011900013D78400D98F90080C1022852317F102F1
:1011A00097000000E780A0C47DE1639209049307E3
:1011B000FA00BD88918391E0C144C207C183DE8CEF
:1011C000814A3EC6414DB24763E2FA0E6286B3855C
:1011D0004B01881097E00000E78080B54DC93D5570
:1011E0007DA093079004E39609F8A54759B7834774
:1011F00001050947C14C2300F10283471105B3C71C
:10120000F900A300F10293872900814963E1FC04FE
:10121000814618103306D7008C083387D900B6955D
:1012200056970347070083C5050085062D8F2300C9
:10123000E600E390D7FE41476390E70690080C1064
:10124000228597000000E78080BA35D189A0B38657
:101250003A01BA871010B305F60090083E9603C510
:1012600006000346060085078506298E2380C500F3
:10127000E39297FF3387EC4090080C102285BA99CF
:1012800097000000E780A0B68947014741D165611A
:101290001713FFFF6700E3E490083E96034606003D
:1012A0001410BE962380C600850779B7B247850A19
:1012B00093990A01939D8A0093D909016391570F6D
:1012C00085473546DA85130511022300F10293D9CB
:1012D000890097E00000E78000A8B3ED3D01900091
:1012E0000C1022852317B10397000000E78020B07F
:1012F00059FD8147A68963EA970626860C084A8528
:1013000097E00000E78020A581471810B306F7009A
:10131000100898083E973E960347070003460600CC
:101320008507318F2380E600E3E197FE639FA905DF
:1013300090080C10228597000000E78040AB21F94F
:1013400081479810B306F700900818183E973E960C
:1013500003470700034606008507318F2380E60018
:10136000E391A7FF4109C10CB9BD18089000B3066D
:10137000F7003E963387FC0003470700034606004C
:101380008507318F2380E600B5B798084E9703474D
:1013900007001C10CE972380E700850941BF8547D1
:1013A0003546DA85130511022300F10293D989002D
:1013B00097E00000E780209AB3ED3D0190000C100B
:1013C00022852317B10397000000E78040A2E310B5
:1013D00005EC814718089000B306F7003E96338766
:1013E000FC0003470700034606008507318F238072
:1013F000E600E391A7FF41460C084A8597E000000C
:10140000E780609581471810B306F7001008980828
:101410003E973E9603470700034606008507318F37
:101420002380E600E391A7FF90080C102285970027
:101430000000E780C09B1DD599BD7D5582801713A4
:10144000FFFFE70243C901112A842E85930551004D
:10145000328902C002C202C402C69304740097F02B
:10146000FFFFE780A03D1D46A6851305910097E08C
:101470000000E780408E10088A854A8597000000AA
:10148000E780E09619ED93071400180883C607005B
:101490000346070085070507B18EA38FD7FEE397A4
:1014A000F4FE05611713FFFF670023C51713FFFF45
:1014B000E702C3C02E848C414111AA89838715009D
:1014C0003289914463D30700A1449757FF1F938744
:1014D000A7069C43A1C7C1CA8D472310F10083C74B
:1014E00025004A852301F10083C73500A301F100DF
:1014F00083C745002302F10083C75500A302F10012
:1015000083C7650093059100A30301002303F10045
:101510002304010097F0FFFFE78040320C404A8629
:101520000A8597F0FFFFE780803303280400835685
:101530004400A6881D0881470147E51642868A8532
:101540004E8597000000E780408E2A8919E5A68520
:10155000228597B0FFFFE780E0C14A85410117135C
:10156000FFFF6700E3B84A860A8597F0FFFFE78030
:10157000002F6DB71713FFFFE70243B42E848C4191
:101580004111AA89838715003289914463D30700EA
:10159000A1449757FF1F938727FA9C43A1C7C1C651
:1015A0008D472310F10083C725004A852301F100F0
:1015B00083C73500A301F10083C745002302F10072
:1015C00083C75500A302F10083C76500930591000E
:1015D000A30301002303F1002304010097F0FFFFA0
:1015E000E780C0250C404A860A8597F0FFFFE78018
:1015F000002783564400032804008A85858EC2068E
:101600001D08C1822312D400A68881470147E51630
:1016100042864E8597000000E78060B041011713B5
:10162000FFFF6700E3AC4A860A8597F0FFFFE7807B
:1016300000234DBF1713FFFFE702E3A9B335B00046
:10164000011185052A891315F60133651501230853
:10165000B1009305110136843AC632C03EC442C27D
:1016600097F0FFFFE780801DA2471248425593D6AE
:101670008700230BF1009305910193578800A30A7B
:10168000D100A30BF100230C010197F0FFFFE780CD
:10169000E01A3247024603280400B337E0008356BD
:1016A00044009207914411C2A1444A85A68842860B
:1016B0000C0897F0FFFFE78040772A8919E5A68597
:1016C000228597B0FFFFE780E0AA4A8505611713DE
:1016D000FFFF670083A21713FFFFE702239E01119C
:1016E0003EC68647B335B0008505AA891315F601B5
:1016F0005D8D2308B1009305110136843A89B284C7
:1017000042C446C297F0FFFFE78040132248924848
:10171000164593578800A30AF1009305910193D7CA
:101720008800230B0101A30BF100230C110197F09A
:10173000FFFFE780A0103247104083564400B337C4
:10174000E000920703280900914891C0A1480C08C5
:101750004E8597000000E780809CAA8401E98355AC
:1017600044004A8597B0FFFFE780C0A02685056149
:101770001713FFFF6700C397AA959307F00F17177A
:101780000100130767ED6317B50013C5F7FF137565
:10179000F50F828005058346F5FFB58FBA9783C79D
:1017A0000700D5B70357450014419307F00F1716EC
:1017B0000100130666EA3697420741831395060136
:1017C0004181631BE500AD8FB29703C50700130588
:1017D00015F3133515008280850603C5F6FFA98F22
:1017E000B29783C70700D9BF1713FFFFE702A38E85
:1017F000B28736842E86BA86AA853E85BA8497F04B
:10180000FFFFE7806052634F0500228597E00000EC
:10181000E78000882A86A686A285268597F0FFFFA6
:10182000E78080501713FFFF6700238D1713FFFF1A
:10183000E702C3885D712A8BAE8A17150100130574
:1018400025DF2C00B284368ABA893E8997F0FFFFE3
:10185000E780C04F2A845DE134104146DA852800D4
:1018600097F0FFFFE780404C2A8449E98547A303AE
:10187000F100A6C2930771002408BEC4A68685475E
:101880000D462C18281002DC02DED6C0BEC697F02A
:10189000FFFFE78000442A8435E183477102A68672
:1018A0000D4693F7F7072300FA00C1473EDE2C18D8
:1018B0008947281026DCA303F10097F0FFFFE7809B
:1018C00040412A8405ED4146A6854E8597D000000B
:1018D000E78060488D47A6860D462C182810A30384
:1018E000F10097F0FFFFE780C03E2A8401E94146FE
:1018F000A6854A8597D00000E780E0452285616192
:101900001703FFFF6700C37E1703FFFFE702A37CF7
:1019100097F7000093870713984383C747007971AF
:101920002A89AE8417150100130505D10C083AC4A5
:101930002306F10097F0FFFFE78040412A8405ED80
:1019400014104146CA85080897F0FFFFE780C03DA4
:101950002A8415E1140815462C00081097F0FFFFA3
:10196000E780803C2A8401E921462C08268597D00F
:101970000000E780403E228545611703FFFF6700B6
:10198000C3771703FFFFE702037597F700009387FC
:10199000670B9C477971AA842E84171501001305E3
:1019A00025CA0C083EC697F0FFFFE780203A0DE9F4
:1019B00014104146A685080897F0FFFFE780C0365F
:1019C00005E1140811466C00081097F0FFFFE7804E
:1019D000A03519E58347F10193F7F7032300F400DD
:1019E00045611703FFFF670043711703FFFFE7021D
:1019F000836E3688A14881470147E54697F0FFFF8F
:101A0000E780A0421703FFFF6700236F1703FFFF64
:101A1000E702636C3688A14881470147E54697F0A5
:101A2000FFFFE780C06F1703FFFF6700036D170319
:101A3000FFFFE702436A01112A842E850C0832C693
:101A400097F0FFFFE780803009ED324797160100DD
:101A5000938686BD1008C145228597000000E78067
:101A6000E0D805611703FFFF670023691703FFFF35
:101A7000E70263664111C1472EC032C48A85094618
:101A80003EC23EC697F0FFFFE780A0244101170346
:101A9000FFFF670083661703FFFFE702C36341117F
:101AA000AE8613061009AA850A8502C002C202C4C6
:101AB00002C697F0FFFFE780202741011703FFFFD1
:101AC0006700A3631703FFFFE702E36032879716FF
:101AD0000100938666B72E869305000297000000EA
:101AE000E780C0D01703FFFF670023611703FFFFE4
:101AF000E702635E7971C1472ACC2ED032D42C081C
:101B00000D4628003ECE3ED23ED602C402C602C8D2
:101B100002CA97F0FFFFE780C01B45611703FFFF74
:101B20006700A35D1703FFFFE702E35A0111AA84D0
:101B30002E84171501001305A5B18A8597F0FFFFC4
:101B4000E780C02015E514084146A6850A8597F070
:101B5000FFFFE780601D09ED8347E1010347F101C5
:101B6000A207D98FCA07C9836177D98F2310F400E0
:101B700005611703FFFF6700435815CD1703FFFFEB
:101B8000E70263559747FF1F938787489043974520
:101B9000FF1F938525481745FF1F1305654397D001
:101BA0000000E78000C51745FF1F130565421703B6
:101BB000FFFF670083541745FF1F130565418280AF
:101BC0008DCD1703FFFFE70203519747FF1F938750
:101BD0002744944301112E840A869745FF1F93855D
:101BE000654397D00000E78040C60A85029401450E
:101BF00005611703FFFF670043507D55828017037F
:101C0000FFFFE702434D97D00000E78080D1974760
:101C1000FF1F23AFA73E17F5FFFF1305E5C997B0D8
:101C20000000E780C0741703FFFF6700034D1747EC
:101C3000FF1F130727409317150008433E95FD57D4
:101C40002310F50082801703FFFFE702C3482A84B0
:101C5000084009E51703FFFF6700234A1C4158406D
:101C60001CC06313E5005CC08347550023200500BA
:101C7000F99BA302F50097A0FFFFE780207CC9BF76
:101C80001703FFFFE70283439747FF1F9387873CB4
:101C900098432A8411CB8347350093F7070289C7FD
:101CA00003550500894502971305440197B00000CC
:101CB000E780403B835504000355E4009730000063
:101CC000E780A00C485819C597A0FFFFE780007770
:101CD000232A04021305840397000000E780E0F63E
:101CE0008144B1499790FFFFE780C06D63CBA402A8
:101CF000834734002320040493F727FCA301F40056
:101D000000489790FFFFE780E06C131615008145AF
:101D100022859700FFFFE780003F1703FFFF670062
:101D2000233DB38734030329040385043E994A8580
:101D300097000000E78060F12304090065B783473E
:101D4000350093F7070299E3014582808357E50048
:101D5000E39CB7FEC167FD176316F6000545828058
:101D6000054599A81703FFFFE702E336931706011D
:101D7000C187B2842A8401496359F0028357050060
:101D80009DCB01456367F600034584003E953325EE
:101D9000A6001375F50F0DA01C4813171900BA976C
:101DA00083D70700E38E97FA05099790FFFFE78036
:101DB0006062E343A9FE01451703FFFF6700E333B9
:101DC0001703FFFFE702832FAE89AA849790FFFFD6
:101DD000E78000562A8497D0FFFFE780A02EAA86CE
:101DE00001471306840197050000938585E4174594
:101DF000FF1F130565249790FFFFE780801C2A8949
:101E000025C98C441304C50022859E0593F5050859
:101E100097A0FFFFE780403CCC4083877400E181BE
:101E200063DD070493E50508228597A0FFFFE7809F
:101E3000A03A0D4693854400228597A0FFFFE780D6
:101E4000C03683D50400228597A0FFFFE780E03DE0
:101E500083D52400228597A0FFFFE780003D03D6AD
:101E6000490083A50900228597A0FFFFE780E033A2
:101E70004A851703FFFF6700A32793F5F5076DB7A2
:101E80001703FFFFE702232501112A84328532C69A
:101E900097A0FFFFE780E0279780FFFFE78060348F
:101EA000835704001747FF1F130747323246231B8F
:101EB000F100930700F8A30DF1001C471843231A03
:101EC000A1008983858BB307F740B28548083ECED1
:101ED000231C0100230D010097000000E78080EE25
:101EE00005611703FFFF670043211703FFFFE702A8
:101EF000E31C004101453DC49304C400268532899A
:101F0000AE8997A0FFFFE780C02495452A8A2685E1
:101F1000035B040197A0FFFFE7802021268597A09F
:101F2000FFFFE780603E8D45AA8A268597A0FFFFC8
:101F3000E780A01F268597A0FFFFE780E03C5C4874
:101F4000420A135A0A01D2975CC4231864018147DC
:101F500063983A0146054D813306254193371600B3
:101F600013F5F70F1703FFFF670083181703FFFF31
:101F7000E702E31389692A8BAE8B328AB68A8144E1
:101F80000144314CFD199790FFFFE780A04363CDDA
:101F9000A4009790FFFFE780E045018D33B5AA00CC
:101FA0001703FFFF670023143389840383270B0083
:101FB0003E9963170A008347890085043E94E1B780
:101FC00003560A00DE854A8533F6C90097000000F3
:101FD000E780E0F16DD10545E1B71703FFFFE702A8
:101FE000830F01112A847C000355E5003ECAB70720
:101FF00007003ECC7C003ECE97200000E780200802
:102000002A898545480897A0FFFFE7802039994530
:10201000480897A0FFFFE780E015AA844A8597202B
:102020000000E780A0082380A4009747FF1F938744
:10203000E7199C434166130606F09396870113D770
:102040008701558F93D68700F18E558FA207B7066B
:10205000FF00F58FD98F11462C00138514003EC464
:1020600097D00000E78020CF5008A3820400894564
:10207000228597000000E780E0E019C9AA851305D2
:10208000840397A0FFFFE780E0313C4085073CC018
:1020900005611703FFFF670043061703FFFFE70211
:1020A00083039790FFFFE780E0342A84050497902C
:1020B000FFFFE78020333305A402F1479145330544
:1020C000F50297200000E78020BA11E56555170357
:1020D000FFFF670083029747FF1F23A5A7F697908E
:1020E000FFFFE78020312A8405049790FFFFE780F7
:1020F000602F3305A4028945060597200000E7807C
:10210000A0B669D59747FF1F23A6A7F29790FFFFB8
:10211000E780402E2A8405049790FFFFE780802CFB
:102120003304A4029747FF1F239887F09790FFFF7F
:10213000E780402C2A849790FFFFE780A02A93072E
:1021400014003385A7029747FF1F2398A7EE970730
:1021500001009387A7131747FF1F2323F7EE0145BD
:10216000BDB71703FFFFE70263F5AA842E89014478
:102170009749FF1F93898905130A80069790FFFFEF
:10218000E78040266347A40001451703FFFF67006F
:1021900023F63305440383A709024A86A6853E95A4
:1021A00097000000E780E0B919E10504C1BF0545CB
:1021B000E9BF1703FFFFE70283EFAA8A2E8BB28BDA
:1021C000368C3A8A814401448149974CFF1F938C95
:1021D000ECFF130D80069790FFFFE780A02063C9F6
:1021E000A40011E085494E851703FFFF6700A3EFA8
:1021F0003389A40383A70C025E86D6853E994A855F
:1022000097000000E780E0B31DC19790FFFFE780D3
:10221000601E0544636D4501D2866286DA8513052A
:10222000090397000000E780A0D411C18549850407
:102230005DB71703FFFFE70263E8C16441112A8914
:1022400001449749FF1F938969F8130A8006FD141A
:1022500036C632C42EC29790FFFFE780A018924581
:102260002246B2466348A400014541011703FFFF1F
:10227000670003E83305440383A709023E9509C6B6
:1022800083473500C18B9DC791C68347350093F7BF
:1022900007028DC3630699008357E500639C2701FD
:1022A0000357050001CB63E7E50083478500BA9734
:1022B000E3CDF5FA050469BF1703FFFFE70203E06A
:1022C000C1642A8901449749FF1F938929F0130AA1
:1022D0008006FD149790FFFFE780C0106346A400BE
:1022E0001703FFFF6700C3E03305440383A7090218
:1022F0003E958357E500638A9700630499006396CF
:10230000270197000000E780E0970504E1B7170375
:10231000FFFFE70243D989692A8AAE8A328BB68BDE
:102320008144174CFF1F130C6CEA930C8006314D4F
:10233000FD199790FFFFE780E00A63C6A40017032A
:10234000FFFF670003DA3389940383270C02835568
:10235000CA015A863E994A8597000000E780609E30
:1023600031C1814D15A03384AD038327090303D602
:102370000B00D68533F6C9003E94228597000000F5
:10238000E780E0B609E9850D9790FFFFE7808003BD
:10239000E3CBADFC01A8228597000000E780E08A2E
:1023A00023040400850471B71703FFFFE70223D05D
:1023B0004169AA8A014A174BFF1F130B2BE17D19B4
:1023C000C14B054C9790FFFFE780C0016346AA0010
:1023D0001703FFFF670023D193098006B3073A0371
:1023E00083290B02BE9983D7E900638E270163849A
:1023F0002A01639A570103A4890301E84E859700D7
:102400000000E780C0BD050A75BF835704016399CA
:1024100077099304C400268597A0FFFFE78060D367
:1024200085452A8D2685835C040197A0FFFFE78000
:10243000C0CF268597A0FFFFE780A0E762056185F2
:10244000635905048D45268597A0FFFFE780E0CD01
:102450008945268597A0FFFFE78020CD8945268501
:1024600097A0FFFFE78060CC8545268597A0FFFFFA
:10247000E780E0CC83470500094793F7F707639AA5
:10248000E7009945268597A0FFFFE78040CBA30290
:1024900085014848337D2D01231894016A9548C46D
:1024A0000040A1BF1703FFFFE702E3C237E40400C7
:1024B0008327041D82979747FF1F83C727BE1715E1
:1024C000FF1F1305E505A300F5008327441C829731
:1024D0008327841C81461306F00F814501458297AE
:1024E0001703FFFF670063C11747FF1F130707AB01
:1024F00018439745FF1F83C565BA9747FF1F93870A
:1025000067B883468703034697036397D5009747C9
:10251000FF1F2385C7B8828083C587010347A703B0
:102520006317B6009747FF1F238AE7B6828003C66A
:1025300087016317C7009747FF1F2381D7B68280A3
:1025400083C68701130750026319D70093076002FF
:102550001747FF1F2304F7B4828083C68701130641
:1025600060026315D60093077002DDB783C7870149
:1025700055BF9747FF1F9387E7B0D44B0947638D3B
:10258000E6081703FFFFE70203B51749FF1F13090A
:10259000A9AC3E8483470900918B9DCFB7E404002A
:1025A00083A7041D829783A7441C1745FF1F1305AB
:1025B00025AB829783A7841C81461746FF1F0346DD
:1025C00026AC81450145829721C583470900ED9BD3
:1025D0001747FF1F2302F7A88347040093F7F70F5D
:1025E00085CB91471747FF1F2328F7AA97000000C4
:1025F000E78080EB97000000E78040EFB7E704003A
:10260000BC4F414691451745FF1F034525A88297BA
:102610001703FFFF670063AE82801703FFFFE70227
:1026200083AB8D4741116306F504C5476308F50286
:1026300085476310F5029747FF1F2383A7A6B7E7D7
:102640000400BC4B930500101745FF1F034505A46C
:10265000829741011703FFFF670023AA85471747A9
:10266000FF1F230FF7A2B7E70400BC4B9305002020
:10267000E1BF9747FF1F9387E7A0D44B1147638DB6
:10268000E600B7E7040083A7071D8297B7E70400B9
:10269000BC4B930500044DBF05491747FF1F232D71
:1026A000279F83C7070032C62E8493F7F70FD5D331
:1026B000B7E4040083A7041D7D141374F40F8297FC
:1026C000E37689FCB245994703C61500E3F0C7FCE1
:1026D000FC4409061745FF1F1305C59C8297BC489B
:1026E000930500081745FF1F0345459A829779BF58
:1026F0001703FFFFE702239E1747FF1F1307879863
:102700004047184B1C409746FF1F23A3F6986316BB
:10271000E4001747FF1F232FF796130584FE9790B9
:10272000FFFFE78000AA035564FF9780FFFFE78063
:10273000807297A0FFFFE78060D01703FFFF67005C
:10274000C39B1703FFFFE70203999747FF1F938778
:102750006793D84BDC4789C797000000E78080F972
:1027600085471747FF1F2329F7929747FF1F938736
:10277000E7829C43930500021745FF1F034505911F
:1027800083C787031747FF1F230AF790B7E70400A3
:10279000BC4B82971703FFFF670023969747FF1FE5
:1027A00023A4A78E82801703FFFFE702239137E45B
:1027B00004007C4CA1451745FF1F0345258D8297DA
:1027C0007C48A1451745FF1F0345458C9744FF1FD3
:1027D0009384448B8297DC4489EB97000000E78068
:1027E00080D91703FFFF6700A39003D567FF978089
:1027F000FFFFE7804066AA896DD1D84891476310F2
:10280000F7027C4C91451745FF1F034525888297A9
:102810007C4891451745FF1F03454587829703A9CB
:10282000490103D409018947B7E904001747FF1F8D
:102830002324F78683A7091D21044204829783C7B6
:1028400084011715FF1F1305A5CD61191717FF1F69
:10285000A308F7CC83A7491C418082979747FF1FA5
:102860002380078483A7C91C814609469375F40F0A
:102870004A85829711E99747FF1F83C7A79289C7A7
:102880009700FF1FE7806036B7E70400BC4F214682
:10289000A1451735FF1F0345657F829799B7170339
:1028A000FFFFE702438393F7052001112E8481CFB8
:1028B00097000000E78020E9134504200561170315
:1028C000FFFF6700838393F70510A9CF9734FF1F9D
:1028D0009384447BDC4897000000E78020C11737D1
:1028E000FF1F1307A76B184383C7840103478703A0
:1028F0006318F700DC4489C797000000E78080DF99
:1029000085471737FF1F2329F778B7E70400BC4B2B
:10291000930500021735FF1F03454577829713453E
:10292000041069BF93F70508BDC79737FF1F83C71A
:102930007777E91719469735FF1F9385C5761305F5
:10294000D10093F4F70F1739FF1F0349A97597C0FA
:102950000000E780404093970401C1831737FF1FB1
:102960001307C774231DF100231CF1009737FF1FC5
:10297000938747713ACE3ACAD8432306010009CB60
:10298000DC439315890154080D46E1856800829760
:102990001345040825B793F72500A5C39737FF1FF4
:1029A0009387476ED84B89476306F7029737FF1F17
:1029B00083C7876A13F7270011EF918B99CFB7E789
:1029C0000400BC4F1306000A89451735FF1F034555
:1029D000E56B829713452400D5B59737FF1F938782
:1029E000E75B9C4383C787031737FF1F2308F76AFA
:1029F00097000000E78060DBF1BF93F7050281CB11
:102A000097000000E78060DA1345040245BD93F7A4
:102A1000850081CB97000000E780E0D21345840059
:102A200071BD93F7150081CB97000000E780A0B43B
:102A30001345140061B593F7450081CB9700000062
:102A4000E78060B31345440095BD93F7050495C333
:102A50009737FF1F83C7076391CB97000000E7807C
:102A6000A0A491471737FF1F2328F76213450404DA
:102A7000B1B593F705010145E38207E49737FF1FDE
:102A800093874760D84B91476310F7049737FF1F30
:102A90009387875C9C4313D727008583D98F858BC9
:102AA00091E7B7E7040083A7071D8297B7E7040003
:102AB000FC4F91451735FF1F0345455D82978547BC
:102AC0001737FF1F232AF75C13450401C5BB97374F
:102AD000FF1F2389A76C828017F3FEFFE702A35F25
:102AE0009737FF1F23A6075A9737FF1F23A4075ABC
:102AF00085471734FF1F1304644A1737FF1F232D20
:102B0000F7581C4083C787031737FF1F2308F75860
:102B10009790FFFFE780409329C59717FF1F23A5D4
:102B2000A7A01C40170500001305A5D783C787037E
:102B30001737FF1F2304F7561717FF1FA302F79E2F
:102B40009737FF1FA3800754B7E7040083A7070840
:102B500082979737FF1F238BA75217F3FEFF67005B
:102B6000C359B7C7898E938767ED1717FF1F232DAA
:102B7000F79A45BF1737FF1F0347C750795555E7E9
:102B80009737FF1F9387075003C71700050797362E
:102B9000FF1FA389E64E03C717008D463377D70280
:102BA0009736FF1FA380E64E83C617001737FF1F17
:102BB0001307C73E184393F6F60FA9EE8347870322
:102BC0001737FF1F230CF74C85471737FF1F230BC1
:102BD000F74A9737FF1F938727489C430145998BF6
:102BE000A9E717F3FEFFE702034F37E404007C4830
:102BF000C1451735FF1F0345654982973C48854508
